:1000000000000320D501000055020000953C0100CE
:10001000590200005B0200005D02000000000000C9
:100020000000000000000000000000005F0200006F
:100030006102000000000000630200006502000091
:100040007D1B0100851B0100ED8E00008D1B010052
:10005000951B01009D1B0100A51B0100AD1B0100AC
:10006000B51B0100BD1B0100C51B0100CD1B01001C
:10007000D51B0100DD1B0100E51B0100ED1B01008C
:10008000F51B0100FD1B0100051C01000D1C0100FA
:10009000151C01001D1C0100251C01002D1C010068
:1000A000351C01001D9200003D1C0100451C010093
:1000B0004D1C0100551C01005D1C0100651C010068
:1000C0006D1C0100751C01007D1C0100851C0100D8
:1000D0008D1C0100951C01009D1C0100A51C010048
:1000E000AD1C0100B51C0100BD1C0100C51C0100B8
:1000F000CD1C0100D51C0100DD1C0100E51C010028
:100100000582000069810000DD810000ED1C010016
:10011000F51C0100FD1C0100051D01000D1D010065
:10012000151D01001D1D0100251D0100A9800000F5
:100130002D1D0100351D01003D1D0100451D010063
:100140004D1D0100551D01005D1D0100651D0100D3
:100150006D1D0100751D01007D1D0100851D010043
:100160008D1D0100951D01009D1D0100A51D0100B3
:10017000AD1D0100B51D0100BD1D0100C51D010023
:10018000CD1D0100D51D0100D1CC000059CC0000CF
:1001900081CC0000A9CC00005869010000000020BB
:1001A000A0010000586901000000FF1F00000000CE
:1001B000586901000000001400000000A0010020A8
:1001C000002B00000000FF1F0000000000000014D2
:1001D0000000000010B572B60EF022FA0E4B0F4A66
:1001E000934208D203F10C049A685968186800F029
:1001F00019F82346F3E70A4A934207D21C46596886
:1002000054F8080B00F01DF82346F4E70FF030FE19
:1002100062B607F08FFAFEE798010000BC0100000B
:10022000D4010000002393420AD210B450F8044BCA
:1002300041F8044B04339342F8D35DF8044B704704
:10024000704700238B4204D2002240F8042B043371
:10025000F8E77047FEE7FEE7FEE7FEE7FEE7FEE7AA
:10026000FEE7FEE7FEE7FEE7FFFFFFFFFFFFFFFF02
:10027000FFFFFFFFFFFFFFFFFFFFFFFFFFFFFFFF8E
:10028000FFFFFFFFFFFFFFFFFFFFFFFFFFFFFFFF7E
:10029000FFFFFFFFFFFFFFFFFFFFFFFFFFFFFFFF6E
:1002A000FFFFFFFFFFFFFFFFFFFFFFFFFFFFFFFF5E
:1002B000FFFFFFFFFFFFFFFFFFFFFFFFFFFFFFFF4E
:1002C000FFFFFFFFFFFFFFFFFFFFFFFFFFFFFFFF3E
:1002D000FFFFFFFFFFFFFFFFFFFFFFFFFFFFFFFF2E
:1002E000FFFFFFFFFFFFFFFFFFFFFFFFFFFFFFFF1E
:1002F000FFFFFFFFFFFFFFFFFFFFFFFFFFFFFFFF0E
:10030000FFFFFFFFFFFFFFFFFFFFFFFFFFFFFFFFFD
:10031000FFFFFFFFFFFFFFFFFFFFFFFFFFFFFFFFED
:10032000FFFFFFFFFFFFFFFFFFFFFFFFFFFFFFFFDD
:10033000FFFFFFFFFFFFFFFFFFFFFFFFFFFFFFFFCD
:10034000FFFFFFFFFFFFFFFFFFFFFFFFFFFFFFFFBD
:10035000FFFFFFFFFFFFFFFFFFFFFFFFFFFFFFFFAD
:10036000FFFFFFFFFFFFFFFFFFFFFFFFFFFFFFFF9D
:10037000FFFFFFFFFFFFFFFFFFFFFFFFFFFFFFFF8D
:10038000FFFFFFFFFFFFFFFFFFFFFFFFFFFFFFFF7D
:10039000FFFFFFFFFFFFFFFFFFFFFFFFFFFFFFFF6D
:1003A000FFFFFFFFFFFFFFFFFFFFFFFFFFFFFFFF5D
:1003B000FFFFFFFFFFFFFFFFFFFFFFFFFFFFFFFF4D
:1003C000FFFFFFFFFFFFFFFFFFFFFFFFFFFFFFFF3D
:1003D000FFFFFFFFFFFFFFFFFFFFFFFFFFFFFFFF2D
:1003E000FFFFFFFFFFFFFFFFFFFFFFFFFFFFFFFF1D
:1003F000FFFFFFFFFFFFFFFFFFFFFFFFFFFFFFFF0D
:10040000FFFFFFFFFFFFFFFFFFFFFFFFFEFFFFFFFD
:1004100001F0FF01102A2BDB10F0070F08D010F8B5
:10042000013B013A8B422DD010F0070F42B3F6D1B9
:10043000F0B441EA012141EA014122F007047FF0D2
:1004400000070023F0E80256083C85EA010586EA29
:10045000010685FA47F5A3FA87F586FA47F6A5FA65
:1004600087F68EB9EED1F0BC01F0FF0102F0070271
:1004700032B110F8013B013A83EA010313B1F8D11C
:100480000020704701387047002D06BF35460338FD
:10049000073815F0010F07D1013015F4807F02BF36
:1004A000013015F4C03F0130F0BC0138704700BF87
:1004B000B0B586B000AF87ED030AC7ED020A87ED3D
:1004C000011AB8680FF06EF802460B4620A1D1E978
:1004D00000010FF0E9F902460B4614461D4697ED60
:1004E000037AD7ED017A37EE677AD7ED036AD7ED55
:1004F000017A76EEE77A67EE277AB1EE677AD7ED82
:10050000027A77EEA76AD7ED027A66EEA77AC7EE8F
:10051000276AB0EE660A12F0C1F910EE103A1846DA
:100520000FF040F802460B46204629460FF092F89D
:1005300002460B46104619460FF09EFA03467B61B1
:100540007B6907EE903AB0EE670A1837BD46B0BD3A
:100550002BF697DD9387D93F80B483B000AF7860E6
:100560001A4BD3F81031C3F38063DBB2002B17D0E2
:100570007B68DB889BB201339AB27B68DA807B6848
:10058000DB889BB24EF6602293428CBF012300238E
:10059000DBB2002B14D07B684FF47A72DA800FE064
:1005A0007B68DB889BB2142B8CBF01230023DBB25A
:1005B000002B02D07B6801229A727B680022DA80CD
:1005C00000BF0C37BD465DF8047B704700F00F405C
:1005D00080B582B000AF78607B68DB78DBB2002B3F
:1005E0000CBF01230023DBB2002B00F040817B68AD
:1005F0001B79DBB20133DAB27B681A717B681B7935
:10060000DBB2802B0CBF01230023DBB2002B02D016
:100610007B6800221A717B681B79DBB2002B0CBF50
:1006200001230023DBB2002B18D07B681B7ADBB2DE
:1006300083F00103DAB27B681A727B681B78DBB245
:10064000002B14BF01230023DBB2002B06D07B68F4
:100650001B78DBB2013BDAB27B681A707B681B79CE
:10066000DBB2402B0CBF01230023DBB2002B10D0E8
:100670007B681B78DBB2002B14BF01230023DBB2A5
:10068000002B06D07B681B78DBB2013BDAB27B68BB
:100690001A709C4AB2F8403043F40063A2F840302C
:1006A000984AB2F8403043F48063A2F840307B6847
:1006B0005B79DBB2934A03F00F03D9B2D2F88030F2
:1006C00061F34813C2F880307B685B8A9BB21A469C
:1006D0007B685B79DBB242FA03F303F00103002B82
:1006E00014BF01230023DBB2002B10D07B681B7AE0
:1006F000DBB283F00103DBB2824A03F00103D9B21B
:10070000B2F8403061F38A23A2F8403018E07B68E9
:100710001B8A9BB21A467B685B79DBB242FA03F311
:1007200003F00103002B14BF01230023DBB2002BD5
:1007300006D0744AB2F840306FF38A23A2F84030F2
:100740007B68DB7ADBB2002B30D07B685B79DBB275
:10075000082B0CBF01230023DBB2002B0FD07B68DA
:100760001B7ADBB283F00103DBB2664A03F00103BC
:10077000D9B2B2F8403061F38A23A2F840307B68E6
:100780005B79DBB20A2B0CBF01230023DBB2002B09
:100790000CD07B681B7ADBB25A4A03F00103D9B252
:1007A000B2F8403061F38A23A2F840307B68DB89DD
:1007B0009AB27B689B8A9BB213439BB21A467B68B2
:1007C0005B79DBB242FA03F303F00103002B14BFA1
:1007D00001230023DBB2002B06D04A4AB2F8403096
:1007E0006FF3CB23A2F840307B68DB8A9BB21A46BA
:1007F0007B685B79DBB242FA03F303F00103002B61
:1008000014BF01230023DBB2002B2DD07B681B7AA1
:10081000DBB283F00103DBB23A4A03F00103D9B241
:10082000B2F8403061F3CB23A2F840307B68DB891B
:100830009AB27B689B8A9BB213439BB21A467B6831
:100840005B79DBB242FA03F303F00103002B14BF20
:1008500001230023DBB2002B06D02A4AB2F8403035
:100860006FF3CB23A2F840307868FFF775FE7B6802
:10087000DB78DBB2022B0CBF01230023DBB2002BA1
:1008800000F08280204B5B68C3F38103DBB2032B53
:100890000CBF01230023DBB2002B1ED07B689B8A98
:1008A0009BB21A467B685B79DBB242FA03F303F032
:1008B0000103002B04D07B689B7EDBB2002B01D1AF
:1008C000012300E00023002B2AD00E4AB2F840306A
:1008D00043F40063A2F8403022E07B68DB899BB2DE
:1008E0001A467B685B79DBB242FA03F303F001033B
:1008F000002B04D17B689B7EDBB2002B06D1012349
:1009000005E000BF00F00F40F40100200023002BA1
:1009100006D08C4AB2F8403043F40063A2F840306D
:100920007B68DB8A9BB21A467B685B79DBB242FA52
:1009300003F303F00103002B13D07B689B8A9AB268
:100940007B68DB899BB213439BB21A467B685B7959
:10095000DBB242FA03F303F00103002B01D00123C1
:1009600000E00023002B0FD07B681B7ADBB283F002
:100970000103DBB2734A03F00103D9B2B2F840308D
:1009800061F3CB23A2F840307B681B78DBB2002BED
:1009900014BF01230023DBB2002B00F0A6807B688C
:1009A0005B79DBB21A467B685B78DBB2013B9A422B
:1009B0000CBF01230023DBB2002B43D07B681B78E4
:1009C000DBB2082B0CBF01230023DBB2002B06D0C7
:1009D0005C4AB2F840306FF38A23A2F840307B685B
:1009E0001B78DBB2062B0CBF01230023DBB2002BEC
:1009F00006D0544AB2F8403043F48063A2F8403045
:100A00007B681B78DBB2042B0CBF01230023DBB215
:100A1000002B06D04B4AB2F840306FF38A23A2F87D
:100A200040307B681B78DBB2022B0CBF0123002314
:100A3000DBB2002B06D0434AB2F8403043F4806367
:100A4000A2F840307B685B79DBB21A467B689B7802
:100A5000DBB2013B9A420CBF01230023DBB2002B27
:100A600043D07B681B78DBB2072B0CBF012300232C
:100A7000DBB2002B06D0334AB2F840306FF3CB2301
:100A8000A2F840307B681B78DBB2052B0CBF01233A
:100A90000023DBB2002B06D02A4AB2F8403043F4E0
:100AA0000063A2F840307B681B78DBB2032B0CBFDD
:100AB00001230023DBB2002B06D0224AB2F84030DB
:100AC0006FF3CB23A2F840307B681B78DBB2012B9D
:100AD0000CBF01230023DBB2002B06D0194AB2F869
:100AE000403043F40063A2F840307B68DB78DBB22F
:100AF000072B0CBF01230023DBB2002B0ED07B6839
:100B00005B79DBB20133DAB27B685A717B685B795F
:100B1000DBB203F00F03DAB27B685A717B68DB78D3
:100B2000DBB20133DAB27B68DA707B68DB78DBB288
:100B300003F00703DAB27B68DA7000BF0837BD46FE
:100B400080BD00BF00F00F4080B485B000AF78607A
:100B5000554AB2F840306FF38A23A2F84030524A27
:100B6000B2F8403043F40063A2F840300023FB8128
:100B7000FB899BB20F2B94BF01230023DBB2002B18
:100B800037D0FB899BB2484A03F00F03D9B2D2F8A1
:100B9000803061F34813C2F880300023BB81BB89E9
:100BA0009BB240F28F12934294BF01230023DBB229
:100BB000002B18D000237B817B899BB240F28F12DF
:100BC000934294BF01230023DBB2002B05D07B8925
:100BD0009BB201339BB27B81EEE7BB899BB20133B1
:100BE0009BB2BB81DBE7FB899BB201339BB2FB81EC
:100BF000BEE72D4AB2F8403043F48063A2F840309B
:100C0000294AB2F840306FF3CB23A2F840300023DA
:100C1000FB81FB899BB20F2B94BF01230023DBB226
:100C2000002B3BD0FB899BB2DBB2C3F10F03DBB2DD
:100C30001D4A03F00F03D9B2D2F8803061F3481394
:100C4000C2F880300023BB81BB899BB240F28F1277
:100C5000934294BF01230023DBB2002B18D0002362
:100C60007B817B899BB240F28F12934294BF012318
:100C70000023DBB2002B05D07B899BB201339BB2F2
:100C80007B81EEE7BB899BB201339BB2BB81DBE783
:100C9000FB899BB201339BB2FB81BAE700BF1437DB
:100CA000BD465DF8047B704700F00F4080B582B010
:100CB00000AF78600A4BB3F840207B685A807B68AD
:100CC0005A887B681B889A4202D0786800F01AF82C
:100CD0007B685A887B681A8000BF0837BD4680BD94
:100CE000A001002080B483B000AF7860044BB3F85B
:100CF000403018460C37BD465DF8047B704700BF96
:100D0000A001002080B586B000AF78607B685B886A
:100D1000BB827B685A887B681B8853409BB27B826E
:100D20000023FB75FB7D0F2B00F2E9817B8A9BB2D0
:100D300003F00103002B14BF01230023DBB2002BBF
:100D400000F0CF81FB7D03F00F03DAB23B7B62F34F
:100D500003033B73BB8A9BB203F00103DAB23B7B14
:100D600062F304133B733B7B6FF345133B733B7B95
:100D70006FF386133B733B7B6FF3C7133B73A14B3E
:100D80001B78DBB20E2B14BF01230023DBB2002B38
:100D900000F097819C4B1B69C3F34333DBB2042BF8
:100DA00000F0E980042B00F38581022B02D0032B95
:100DB0007CD07FE13B7BC3F30303DBB2022B4CD03F
:100DC000022B00F38981002B02D0012B22D083E17A
:100DD0003B7B03F01003DBB2002B61D0894A13790F
:100DE0006FF383031371874B5B68C3F38103DBB23B
:100DF0001A46864B1A70864B0022DA813B7BC3F37E
:100E00000303DBB20133DBB21A460221804811F042
:100E1000B4FA45E03B7B03F01003DBB2002B41D07A
:100E2000784A1379012161F383031371754B5B6871
:100E3000C3F38103DBB21A46744B1A70744B002261
:100E4000DA813B7BC3F30303DBB20133DBB21A4627
:100E500002216F4811F091FA24E03B7B03F010036C
:100E6000DBB2002B20D0674A1379022161F38303A0
:100E70001371644B5B68C3F38103DBB21A46634BA7
:100E80001A70634B0022DA813B7BC3F30303DBB2AE
:100E90000133DBB21A4602215D4811F06EFA03E01D
:100EA00000BF19E100BF17E100BF15E13B7BC3F3B1
:100EB0000303DBB2022B40D0022B00F30F81002B87
:100EC00002D0012B1CD009E14E4A13796FF3830342
:100ED00013714C4B5B68C3F38103DBB21A464B4B77
:100EE0005A704B4B0022DA813B7BC3F30303DBB226
:100EF0000133DBB21A460321454811F03EFA39E0CE
:100F0000404A1379012161F3830313713D4B5B6800
:100F1000C3F38103DBB21A463C4B5A703C4B0022B0
:100F2000DA813B7BC3F30303DBB20133DBB21A4646
:100F30000321374811F021FA1CE0324A13790221CB
:100F400061F3830313712F4B5B68C3F38103DBB23F
:100F50001A462E4B5A702E4B0022DA813B7BC3F38C
:100F60000303DBB20133DBB21A460321284811F038
:100F700004FA00BFB2E03B7BC3F30303DBB2022BF6
:100F800048D0022B00F3AC80002B02D0012B1CD0E8
:100F9000A6E01C4A13796FF383031371194B5B6846
:100FA000C3F38103DBB21A46184B9A70184B002228
:100FB000DA813B7BC3F30303DBB20133DBB21A46B6
:100FC0000421134811F0D9F973E00E4A1379012175
:100FD00061F3830313710B4B5B68C3F38103DBB2D3
:100FE0001A460A4B9A700A4B0022DA813B7BC3F304
:100FF0000303DBB20133DBB21A460421044811F0CB
:10100000BCF956E0F401002000F00F40F405002088
:10101000C01D00203C4B1B78DBB20B2B0CBF012307
:101020000023DBB2002B28D0374A137943F00C039E
:101030001371354B5B68C3F38103DBB21A46334B44
:101040009A70314A13796FF3041313712E4A13798E
:101050006FF3471313712E4B01229A762C4B072204
:10106000DA813B7BC3F30303DBB20133DBB21A4605
:101070000421274811F081F91BE0234A13796FF30B
:1010800083031371204B5B68C3F38103DBB21A4601
:101090001E4B9A701E4B0022DA813B7BC3F3030385
:1010A000DBB20133DBB21A460421194811F065F9AD
:1010B00000BF15E07B689B68F968184610F0B9FE20
:1010C0000FE0144B1B69C3F343337B689B68F968DB
:1010D000184610F0AEFE04E000BF02E000BF00E0E2
:1010E00000BF7B8A9BB25B109BB27B82BB8A9BB2A8
:1010F0005B109BB2BB82FB7D0133FB7512E600BF28
:101100001837BD4680BD00BFF4010020F405002063
:10111000C01D002000F00F4080B483B000AF7860A5
:101120000B46FB701346BB70BB78032B32D801A271
:1011300052F823F045110000591100006D11000014
:1011400081110000FB7803F00F03D9B2144A137821
:1011500061F3030313701DE0FB7803F00F03D9B2B2
:101160000F4A137861F30713137013E0FB7803F051
:101170000F03D9B20A4A537861F30303537009E0AD
:10118000FB7803F00F03D9B2054A537861F30713D4
:10119000537000BF00BF0C37BD465DF8047B70473D
:1011A000E401002080B483B000AF78600B46FB7090
:1011B0001346BB70BB78032B32D801A252F823F040
:1011C000D1110000E5110000F91100000D1200001E
:1011D000FB7803F00103D9B2144A937861F300035A
:1011E00093701DE0FB7803F00103D9B20F4A9378A6
:1011F00061F34103937013E0FB7803F00103D9B26C
:101200000A4A937861F38203937009E0FB7803F054
:101210000103D9B2054A937861F3C303937000BF09
:1012200000BF0C37BD465DF8047B7047E401002029
:1012300080B483B000AF78600B46FB701346BB7080
:101240007B68FA7883F824207B68BA7883F82520B5
:101250007B6893F82430DBB21A467B6893F825301C
:10126000DBB218467B681C499200024451F82220E8
:101270005A617B681B7D03F00703DBB2012B0CD1A5
:101280007B681B7D03F00803DBB2002B05D07B6875
:10129000DB7CDAB27B689A7417E07B681B7DC3F352
:1012A0000203DBB21A467B68DB7CDBB29A4206DAC9
:1012B0007B681B7DC3F30203DBB21A4602E07B6846
:1012C000DB7CDAB27B689A7400BF00BF0C37BD4686
:1012D0005DF8047B704700BF8454010090B585B071
:1012E00000AF78600B46FB707B687A6852699A6140
:1012F000994B1B78DBB2092B08D17B681B7E03F06E
:101300000703DBB2042B01D1012300E00023002BF3
:101310000ED07A68137E43F0080313767A68537E02
:1013200043F0010353767A68137E43F0100313767B
:101330007B685B7E03F00103DBB2002B23D17B686B
:101340005B7CDBB21A467B681B7EC3F30203DBB215
:1013500019467B68DB7CDBB2994205DA7B681B7E31
:10136000C3F30203DBB202E07B68DB7CDBB29342B7
:1013700094BF01230023DBB2002B01D00023FCE14A
:101380007B6800221A747B681B7E03F04003DBB28B
:10139000002B3AD07B681B6A184610F0B1FE03465A
:1013A00003F00F03D9B27A68137861F30303137063
:1013B0007B681B6A184610F075FE034603F00F03A6
:1013C000D9B27A68137961F3030313717A681378D9
:1013D00043F0100313707A68137943F0100313710C
:1013E00000220021786811F047F801220121786875
:1013F00011F042F8786811F065F87B6802225A749F
:10140000786800F0BFF90123B7E17B689B7CDAB212
:101410007B681B7CDBB29A4294BF01230023DBB2C2
:10142000002B02D07B6800221A747B685B7CDAB2E6
:101430007B689B7CDBB29A422CBF01230023DBB28A
:10144000002B54D00023FB737B689B7CDBB2FA7BC0
:101450009A4234BF01230023DBB2002B7ED07B688D
:101460001B7CDBB21A467B6853F82230C3F30303BC
:10147000DBB21C467B681A6A7B681B7EC3F30203DF
:10148000DBB219467B68DB7CDBB2994205DA7B680C
:101490001B7EC3F30203DBB202E07B68DB7CDBB2C2
:1014A0001946104610F0E1FD03469C4214BF01238B
:1014B0000023DBB2002B16D07B681B7CDBB2013330
:1014C000DAB27B681A747B689B7CDAB27B681B7C1F
:1014D000DBB29A4294BF01230023DBB2002B02D07F
:1014E0007B6800221A74FB7B0133FB73ACE700239B
:1014F000BB737B689B7CDBB2BA7B9A4234BF01230F
:101500000023DBB2002B29D07B681B7CDBB21A46A0
:101510007B6853F82230C3F30013DBB2002B16D0E4
:101520007B681B7CDBB20133DAB27B681A747B68A0
:101530009B7CDAB27B681B7CDBB29A4294BF0123AE
:101540000023DBB2002B02D07B6800221A74BB7B25
:101550000133BB73CDE700BFF40100207B681B7E25
:1015600003F01003DBB2002B23D000237B737B68D6
:101570009B7CDBB27A7B9A4234BF01230023DBB22F
:10158000002B16D07A7B7B6853F82230C3F3030319
:10159000DBB21A46FB789A420CBF01230023DBB270
:1015A000002B02D07B687A7B1A747B7B01337B73C0
:1015B000DDE77B681B7EC3F30203DBB21A467B6860
:1015C000DB7CDBB29A4206DA7B681B7EC3F3020344
:1015D000DBB21A4603E07B68DB7CDBB21A467B6831
:1015E0009B7CDBB29A4214BF01230023DBB2002BA9
:1015F00029D000233B737B689B7CDBB23A7B9A4209
:1016000034BF01230023DBB2002B1CD07B681B7C82
:10161000DBB23A7B9A4214BF01230023DBB2002BDA
:101620000DD0397B7A6812F821306FF3041302F879
:1016300021303B7B1A4600217868FFF7B3FD3B7BE6
:1016400001333B73D7E77B685B7E03F00203DBB2B9
:10165000002B0FD07B68FA781A747B681B7CDBB296
:10166000032B8CBF01230023DBB2002B02D07B684D
:1016700003221A747B681B7CDBB21946FB7803F0EB
:101680000F03D8B27A6812F8213060F3030302F82E
:1016900021307B681B7CDBB219467A6812F8213056
:1016A00043F0100302F821307B681B7CD9B27B68C1
:1016B0001B7CDBB21A46786810F0DEFE786810F00A
:1016C00001FF7B681B7E03F00803DBB2002B16D002
:1016D0007B681B7CDBB20133DAB27B681A747B68EF
:1016E0009B7CDAB27B681B7CDBB29A4294BF0123FD
:1016F0000023DBB2002B02D07B6800221A747B68C7
:101700005B7CDBB20133DAB27B68114659747B68CB
:101710001B7EC3F30203DBB219467B68DB7CDBB2C2
:10172000994205DA7B681B7EC3F30203DBB202E059
:101730007B68DB7CDBB2934234BF01230023DBB246
:10174000002B16D07B681B7EC3F30203DBB21A4664
:101750007B68DB7CDBB29A4206DA7B681B7EC3F3D4
:101760000203DBB21A4602E07B68DB7CDAB27B68FC
:101770005A74786800F006F8012318461437BD46FD
:1017800090BD00BF80B485B000AF7860814B1B78FE
:10179000DBB20B2B0CBF01230023DBB2002B3ED0AE
:1017A0007B681B7F002B02D07B4B00229A82002398
:1017B000FB737B68DB7CDBB2FA7B9A4234BF01238C
:1017C0000023DBB2002B69D0FA7B7B6853F8223010
:1017D000C3F30013DBB2012B05D17B681B7F002B09
:1017E00001D0012300E00023002B14D0FA7B7B689A
:1017F00053F82230C3F30303DBB21A46012303FA82
:1018000002F1654B9B8A9BB21AB20BB213431BB217
:101810009AB2614B9A82FB7B0133FB73C9E77B6809
:101820001B7F002B02D05C4B0022DA810023BB73AC
:101830007B68DB7CDBB2BA7B9A4234BF0123002396
:10184000DBB2002B2AD0BA7B7B6853F82230C3F37B
:101850000013DBB2012B05D17B681B7F002B01D06D
:10186000012300E00023002B14D0BA7B7B6853F8DF
:101870002230C3F30303DBB21A46012303FA02F159
:10188000454BDB899BB21AB20BB213431BB29AB21F
:10189000414BDA81BB7B0133BB73C9E73D4B5B68CE
:1018A000C3F38103DBB2032B0CBF01230023DBB2A4
:1018B000002B68D07B681B7F002B02D0364B0722A1
:1018C000DA817B681B7F002B02D0334B00229A8287
:1018D00000237B737B68DB7CDBB27A7B9A4234BF6C
:1018E00001230023DBB2002B4DD07A7B7B6853F8B9
:1018F0002230C3F30013DBB2002B40D07A7B7B682D
:1019000053F82230C3F30303DBB2022B05D97B6803
:101910001B7F002B01D0012300E00023002B15D0FA
:101920007A7B7B6853F82230C3F30303DBB21A4699
:10193000012303FA02F1184BDB899BB21AB20BB2F6
:1019400013431BB29AB2144BDA8118E07B681B7FF9
:10195000002B14D07A7B7B6853F82230C3F3030347
:10196000DBB21A46012303FA02F10B4B9B8A9BB2AE
:101970001AB20BB213431BB29AB2074B9A827B7B0B
:1019800001337B73A6E700BF1437BD465DF8047BC7
:10199000704700BFF4010020C01D002080B483B058
:1019A00000AF78607A6892F82420D2B202F0030285
:1019B000D2B262F301037A6892F82520D2B202F023
:1019C0000302D2B262F38303094A5268C2F30012DF
:1019D000D2B262F30413064A5268C2F34212D2B280
:1019E00062F3471318460C37BD465DF8047B704719
:1019F000F401002080B584B000AF7860396007F151
:101A00000C03042219460A4812F097FEFB68396855
:101A10007A688A1AB3FBF2F102FB01F29A1A7B6828
:101A20001344FB60FB6818461037BD4680BD00BFFD
:101A30000090024080B598B000AF0346FB800023C1
:101A400087F85F300023BB6407F14C0300221A6063
:101A50005A609A60002387F85E30002387F85D3073
:101A60004FF00003BB6507F1080340220021184630
:101A700013F089FAFB88002B00F0BF80FB88002B55
:101A80001ED0FB8803F00103002B10D097F85F30C5
:101A9000013387F85F3097F85D305A1C87F85D2076
:101AA00007F16002134497F85E2003F8182CFB88B6
:101AB0005B10FB8097F85E30013387F85E30DDE71E
:101AC000002387F85E3097F85E2097F85F309A42DF
:101AD0004ED2002387F85D3097F85D300F2B41D848
:101AE00097F85D3007EE903AB8EE677A97F85F3076
:101AF000C3F110034D4A9B001344D3ED007AB0EEBE
:101B0000006AC7EE866A97F85E3007F160021344F8
:101B100013F8183C07EE903AF8EE677AB0EE671AC1
:101B2000F0EE660AB0EE470AFEF7C2FCB0EE407A6D
:101B300097F85D309B0007F160021344583BD3EDEA
:101B4000007A97F85D3077EE277A9B0007F1600204
:101B50001344583BC3ED007A97F85D30013387F8A2
:101B60005D30B9E797F85E30013387F85E30AAE759
:101B7000002387F85D3097F85D300F2B14D897F865
:101B80005D309B0007F160021344583BD3ED007AAF
:101B900097ED167A77EE277AC7ED167A97F85D30CB
:101BA000013387F85D30E6E7DFED216A97ED167ABD
:101BB000C6EE877AC7ED167A002387F85D3097F86E
:101BC0005D300F2B2DD897F85D309B0007F1600238
:101BD0001344583B93ED007A97F85D30D7ED167AB1
:101BE00067EE277A134A9B001344C3ED007A97F8F7
:101BF0005D30013387F85D30E1E7002387F85D3021
:101C000097F85D300F2B0CD897F85D30094A9B0090
:101C10001344094A1A6097F85D30013387F85D3044
:101C2000EEE700BF6037BD4680BD00BFA0000020CA
:101C30000000C642600000200000C84080B588B0A7
:101C400000AFF860B9601346FB710023FB764FF0DC
:101C500000037B61FB79002B34D064210020FFF767
:101C6000C9FE03463B613B6907EE903AF8EE677A9E
:101C700097ED057AB4EEE77AF1EE10FA12D5FB7E15
:101C80005A1CFA76154A9B001344D3ED007A97ED5F
:101C9000057A77EE277AC7ED057AFB7E0F2B00D801
:101CA000E1E700BFFB7E013BB968FA688A1A02FBD4
:101CB00003F3002B00DA0F331B111A46FB681344A1
:101CC000FB6105E0B968F868FFF794FE0346FB6125
:101CD000FB6918462037BD4680BD00BF600000206C
:101CE00080B485B000AF78600B46FB707B689B7C4E
:101CF000DAB27B6893F86630DBB29A4234BF0123D4
:101D00000023DBB2002B36D07B689B7CDBB2013337
:101D1000DAB27B689A747B689B7CFB73FB7B002B3D
:101D20000BD0FB7B5A1EFB7B79688A5CD1B27A6848
:101D3000D154FB7B013BFB73F0E77B68FA781A70A8
:101D40007B68B3F864309BB21AB2FB78012101FAC8
:101D500003F31BB213431BB29AB27B68A3F864204F
:101D60007B6893F86830002B05D07B68B3F864304B
:101D70009AB2044B9A8200BF1437BD465DF8047BCB
:101D8000704700BFC01D002080B485B000AF7860F0
:101D90000B46FB700023FB737B689B7CDBB2FA7BFA
:101DA0009A4234BF01230023DBB2002B41D0FB7BDE
:101DB0007A68D35CDBB2FA789A420CBF0123002325
:101DC000DBB2002B31D0FB7BBB737B689B7CDBB22F
:101DD000BA7B9A4234BF01230023DBB2002B0BD025
:101DE000BB7B5A1CBB7B79688A5CD1B27A68D154C0
:101DF000BB7B0133BB73E8E77B689B7CDBB2013BB9
:101E0000DAB27B689A747B68B3F864309BB21AB21A
:101E1000FB78012101FA03F31BB2DB431BB2134031
:101E20001BB29AB27B68A3F86420FB7B0133FB737F
:101E3000B2E77B6893F86830002B05D07B68B3F875
:101E400064309AB2034B9A8200BF1437BD465DF8E6
:101E5000047B7047C01D002080B584B000AF78605F
:101E60000B46FB707B68DB7CDBB283F00103DBB2EB
:101E7000002B05D0FB7819467868FFF731FF01E1A8
:101E8000FB781946786810F0E3FF0346002B0CBF7F
:101E900001230023DBB2002B00F0B3807B6893F8B2
:101EA00069301A461346DB0013445B0013441833B1
:101EB0007A6813440633FA781146184610F03BF856
:101EC0007B6893F869301A461346DB0013445B00C5
:101ED000134418337A6813440633184610F0A9F8EF
:101EE00003461A467B6893F86630DBB29A428CBF91
:101EF00001230023DBB2002B7DD07B6893F8663092
:101F0000FB737B6893F869301A461346DB00134471
:101F10005B00134418337A6813440633184610F0F4
:101F200088F803461A46FB7B934234BF0123002303
:101F3000DBB2002B4AD07B6893F869301A4613460F
:101F4000DB0013445B00134418337A6813440633F0
:101F5000FA7B1146184610F088F80346194678684F
:101F6000FFF712FF7B6893F869301A461346DB00CF
:101F700013445B00134418337A6813440633FA7B26
:101F80001146184610F071F803461A460123934093
:101F900083F47F4383F0FF037A6892F86920114647
:101FA0007A680C3132F8112092B212B21BB213408F
:101FB00019B27B6893F869301A4689B27B680C3293
:101FC00023F81210FB7B0133FB739AE77B6893F8CD
:101FD00069301A461346DB0013445B001344183380
:101FE0007A6813449A1D7B6893F86630DBB2194611
:101FF000104610F02BF8FB7819467868FFF770FE52
:1020000016E07B6893F869301A461346DB001344E8
:102010005B00134418337A6813440633FA78114688
:1020200018460FF0BDFFFB7819467868FFF7ACFE45
:102030007B6893F869301A467B680C3233F81230AB
:102040009BB21AB2FB78012101FA03F31BB2534091
:1020500019B27B6893F869301A4689B27B680C32F2
:1020600023F812107B6893F86830002B0AD07B6845
:1020700093F869301A467B680C3233F812309AB202
:10208000024B9A8200BF1037BD4680BDC01D0020A4
:1020900090B587B002AF78600B46FB701346BB70FB
:1020A0007B689B7CDBB2002B0CBF01230023DBB2DF
:1020B000002B0CD0BB78052B00F0ED81F978BB78B4
:1020C00000930F230022786810F01EFDE3E1BB7837
:1020D000013B042B00F2DF8101A252F823F000BF84
:1020E000F52000001F2100008722000029230000A6
:1020F000C92300007B689B7CDBB2002219460020CC
:10210000FFF79CFD0346DBB21946FB787A68525C08
:10211000D1B27A6813440A4683F85720BBE17B6842
:102120009B7CDBB2012B8CBF01230023DBB2002B95
:1021300072D00023FB73FB7B0F2B78D87B68B3F83E
:1021400064309BB21946FB787A68134493F8573091
:10215000DBB21A4601239340013B0B40002B0CBF1E
:1021600001230023DBB2002B05D0FB787A681344EF
:10217000012283F85F207B68B3F864309BB2194674
:10218000FB787A68134493F85730DBB201330122AD
:1021900002FA03F3013B83F47F4383F0FF030B4018
:1021A000002B0CBF01230023DBB2002B05D0FB78F2
:1021B0007A681344FF2283F85F20FB787A6813441F
:1021C00093F85F3058B2FB787A68134493F857302D
:1021D000D9B2C2B2FB780A44D1B27A6813440A4633
:1021E00083F857207B68B3F864309BB21946FB78BC
:1021F0007A68134493F85730DBB241FA03F303F0E3
:102200000103002B14BF01230023DBB2002B0DD1EF
:10221000FB7B0133FB738EE7FB787A681278D1B2CF
:102220007A6813440A4683F8572000E000BF7B68B1
:1022300093F86730DBB2002B00F02681FB787A68D8
:10224000134493F85F305BB2012B0CBF01230023D2
:10225000DBB2002B0BD07B68FC7818460FF050FFE8
:1022600003461A467B68234483F857200CE17B68B9
:10227000FC7818460FF016FF03461A467B68234485
:1022800083F8572000E1FB787A681344FF2283F833
:102290005F200023BB73BB7B0F2B32D8FB787A689F
:1022A0001A4492F85720D2B2013AD1B27A68134454
:1022B0000A4683F85720FB7850337A681344073373
:1022C0001A78D2B202F00F02D2B21A707B68B3F859
:1022D00064309BB21946FB787A68134493F8573000
:1022E000DBB241FA03F303F00103002B14BF012317
:1022F0000023DBB2002B03D1BB7B0133BB73CAE7E6
:1023000000BF7B6893F86730DBB2002B00F0BE8023
:102310007B68FC7818460FF0C5FE03461A467B68BA
:10232000234483F85720B1E0FB787A6813440122F4
:1023300083F85F2000237B737B7B0F2B32D8FB78E5
:102340007A681A4492F85720D2B20132D1B27A6830
:1023500013440A4683F85720FB7850337A681344B5
:1023600007331A78D2B202F00F02D2B21A707B6829
:10237000B3F864309BB21946FB787A68134493F83B
:102380005730DBB241FA03F303F00103002B14BF13
:1023900001230023DBB2002B03D17B7B01337B7352
:1023A000CAE700BF7B6893F86730DBB2002B6FD0C1
:1023B0007B68FC7818460FF0A3FE03461A467B683C
:1023C000234483F8572063E0FB787A68134493F83A
:1023D0005B30DBB2002B0AD0FB787A68134493F8A9
:1023E0005B30DAB27B689B7CDBB29A4201D301237B
:1023F00000E00023002B08D0FB787A68927CD1B2F1
:102400007A6813440A4683F85B20FB787A681A449A
:1024100092F85B20D2B2013AD1B27A6813440A46EC
:1024200083F85B20FB787A68134493F85B30DBB267
:102430001946FB787A68525CD1B27A6813440A462E
:1024400083F857207B6893F86730DBB2002B21D0EC
:102450007B689B7CDAB2FB78013AD1B27A6813448C
:102460000A4683F85B20FB787A68134493F85B3064
:10247000DBB21946FB787A68525CD1B27A681344B1
:102480000A4683F8572005E000BF04E000BF02E0E1
:1024900000BF00E000BF00BF1437BD4690BD00BFC5
:1024A00090B587B002AF78600B46FB701346BB70E7
:1024B0007B689B7CDBB2032B00F2418101A252F8C6
:1024C00023F000BFD524000031250000B325000013
:1024D00027260000B978FB7800930F230022786844
:1024E00010F012FB0023FB73FB7B032B00F2228115
:1024F000FA7BBB789A4217D0BA78FB7B79680A449A
:1025000092F85720D1B27A6813440A4683F85720CC
:10251000BA78FB7B79680A4492F85F2051B27A68F6
:1025200013440A4683F85F20FB7B0133FB73DBE730
:10253000BB7803F00103002B0ED17B6818460FF027
:10254000B1FD03461A46B978FB7800931346002282
:10255000786810F0D9FA0DE07B6818460FF0A2FDFC
:1025600003460133DAB2B978FB7800930F23786819
:1025700010F0CAFABB78BA7882F00202D2B21146E1
:102580007A68134493F85730DAB27B680B4483F8C7
:102590005720BB78BA7882F00202D2B211467A682C
:1025A000134493F85F305AB27B680B4483F85F2082
:1025B000C5E07B6818460FF0A3FD03461C467B6808
:1025C00018460FF06FFD03461A46B978FB78009362
:1025D00013462246786810F097FA0023BB73BB7B42
:1025E000032B00F2A980BA7BBB789A4217D0BA7845
:1025F000BB7B79680A4492F85720D1B27A681344B9
:102600000A4683F85720BA78BB7B79680A4492F867
:102610005F2051B27A6813440A4683F85F20BB7B7F
:102620000133BB73DBE7BB78032B00F2878001A289
:1026300052F823F045260000632600008D26000096
:10264000EB2600007B6818460FF05AFD03461A4639
:10265000B978FB78009313460022786810F054FA9A
:1026600067E07B6818460FF04BFD03460133DCB290
:10267000786810F0FCF903461A46B978FB780093A5
:1026800013462246786810F03FFA52E07B681846FD
:102690000FF008FD03460E2B94BF01230023DBB28D
:1026A000002B14D0786810F0E2F903460133DCB255
:1026B0007B6818460FF0F6FC03461A46B978FB789B
:1026C000009313462246786810F01EFA31E07868CD
:1026D00010F0CDF903460133DAB2B978FB780093F4
:1026E0000E23786810F010FA23E07B6818460FF08C
:1026F000D9FC03460E2B94BF01230023DBB2002B31
:102700000ED07B6818460FF0CDFC03460133DAB2D9
:10271000B978FB7800930F23786810F0F5F90DE095
:10272000B978FB7800930F230F22786810F0ECF94A
:1027300004E003E000BF02E000BF00E000BF7B68F0
:1027400093F86730DBB2002B03D07B68002283F85C
:10275000672000BF1437BD4690BD00BF90B585B05F
:1027600002AF78600B46FB707B6893F86930012BF1
:1027700040F024817B689B7CDBB2032B00F2248138
:1027800001A252F823F000BF99270000FF270000A4
:1027900071280000EF280000FB7800930F2300222F
:1027A0000021786810F0B0F97B6893F85730DAB2FE
:1027B0007B6883F858207B6893F85730DAB27B68DF
:1027C00083F859207B6893F85730DAB27B6883F836
:1027D0005A207B6893F85F305AB27B6883F8602098
:1027E0007B6893F85F305AB27B6883F861207B681E
:1027F00093F85F305AB27B6883F86220E4E07B682C
:1028000018460FF04FFC03461A46FB780093134618
:1028100000220021786810F077F97B6818460FF0E5
:1028200041FC03460133DAB2FB7800930F23012108
:10283000786810F069F97B6893F85730DAB27B68F2
:1028400083F859207B6893F85830DAB27B6883F8B4
:102850005A207B6893F85F305AB27B6883F8612016
:102860007B6893F860305AB27B6883F86220ABE0F3
:102870007B6818460FF044FC03461C467B681846EC
:102880000FF010FC03461A46FB78009313462246CD
:102890000021786810F038F97B6893F85730DAB285
:1028A0007B6883F858207B6893F85730DAB27B68EE
:1028B00083F859207B6893F85730DAB27B6883F845
:1028C0005A207B6893F85F305AB27B6883F86020A7
:1028D0007B6893F85F305AB27B6883F861207B682D
:1028E00093F85F305AB27B6883F862206CE07B68B3
:1028F00018460FF005FC03461A46FB780093134672
:1029000000220021786810F0FFF87B6818460FF06D
:10291000F7FB03460133DCB2786810F0A8F80346F1
:102920001A46FB780093134622460121786810F07E
:10293000EBF87B6818460FF0B5FB03460E2B94BFEF
:1029400001230023DBB2002B22D0786810F08FF82F
:1029500003460133DCB27B6818460FF0A3FB034645
:102960001A46FB780093134622460221786810F03D
:10297000CBF87B6818460FF095FB03460133DAB2BB
:10298000FB7800930F230321786810F0BDF81BE05B
:10299000786810F06CF803460133DAB2FB780093E4
:1029A0000E230221786810F0AFF8FB7800930F2314
:1029B0000F220321786810F0A7F805E0FB781A468B
:1029C00000217868FFF764FB7B6893F86730DBB21F
:1029D000002B03D07B68002283F8672000BF0C37F0
:1029E000BD4690BD90B585B000AF78607B68DB7C5C
:1029F000DBB2002B0CBF01230023DBB2002B00F065
:102A0000A2807B680122DA747B689B7CDBB2002B9E
:102A100014BF01230023DBB2002B4AD0786810F0EA
:102A2000F6F97B689B7CFB73FB7B002B00F08B80B3
:102A30007B6893F869301A461346DB0013445B0049
:102A4000134418337A6813449C1D7A68FB7B013B5E
:102A5000DBB2194610460FF008FB03461946204624
:102A60000FF069FA7A68FB7B013BDBB2194610462E
:102A70000FF0FBFA03461A46012303FA02F17B68C2
:102A800093F869301A467B680C3233F812309BB2E7
:102A90001AB20BB2134319B27B6893F869301A4625
:102AA00089B27B680C3223F81210FB7B013BFB736D
:102AB000BAE77B6893F869301A461346DB00134483
:102AC0005B00134418337A681344063318460FF03A
:102AD000B0FA0346002B14BF01230023DBB2002B06
:102AE00031D07B6893F869301A461346DB001344F3
:102AF0005B00134418337A681344063318460FF00A
:102B000098FA0346BB73BB7B002B1CD07B6893F801
:102B100069301A461346DB0013445B001344183334
:102B20007A6813449A1DBB7B013BDBB21946104601
:102B30000FF09BFA034619467868FFF7D1F8BB7B84
:102B4000013BBB73DFE77B6893F86830002B0AD04A
:102B50007B6893F869301A467B680C3233F8123080
:102B60009AB2034B9A8200BF1437BD4690BD00BF96
:102B7000C01D002090B585B000AF78607B68DB7C1D
:102B8000DBB2012B0CBF01230023DBB2002B59D099
:102B90007B6893F869301A461346DB0013445B00E8
:102BA000134418337A681344063318460FF041FA79
:102BB0000346FB73FB7B002B41D02848FEF792F8BD
:102BC00003461C467B6893F869301A461346DB00BF
:102BD00013445B00134418337A6813449A1DFB7B3B
:102BE000013BDBB2194610460FF03FFA034644FAA8
:102BF00003F303F00103002B0CBF01230023DBB21E
:102C0000002B18D07B6893F869301A461346DB0016
:102C100013445B00134418337A6813449A1DFB7BFA
:102C2000013BDBB2194610460FF01FFA0346194666
:102C30007868FFF7A9F8FB7B013BFB73BAE77B6879
:102C40000022DA747B6893F86830002B02D0044BC2
:102C500000229A8200BF1437BD4690BD601E00203E
:102C6000C01D0020B0B584B000AF78607B681E3313
:102C700018460FF0DEF903463B733B7B002B46D032
:102C80000023FB73FA7B3B7B9A4240D2FB7B03F031
:102C90000103002B1BD17B6803F11E003A7BFB7BF9
:102CA000D31ADBB2013BDBB219460FF0DEF9034663
:102CB0001A46FB7B5B1002F00F02D1B2584A023376
:102CC0009B0013441A7961F303021A711BE07B68BD
:102CD00003F11E003A7BFB7BD31ADBB2013BDBB274
:102CE00019460FF0C2F903461A46FB7B013B5B1005
:102CF00002F00F02D1B24A4A02339B0013441A7900
:102D000061F307121A71FB7B0133FB73BAE7444A84
:102D10003B7B82F82C307B6893F869309AB2404B49
:102D20001A867B68DB7CDAB23D4B83F854230023A0
:102D3000BB73BB7B022B6ED8BA7BBB7B79680A4422
:102D4000127DD1B2364A13440A4683F85523B97B23
:102D5000BB7B7A680C3132F8112091B2304A03F50E
:102D6000D4735B0013440A461A8100237B737B7B78
:102D7000102B1ED8B97B7C7BBA7B787B7D680B4699
:102D8000DB000B445B000B442B4423441E331B78B5
:102D9000DCB223491346DB0013445B0013440B44AD
:102DA000034403F25E3322461A707B7B01337B734C
:102DB000DDE7B97BBA7B78680B46DB000B445B0030
:102DC0000B4403442F331B78D8B215491346DB005C
:102DD00013445B0013440B4403F26F3302461A7032
:102DE000B97BBA7B78680B46DB000B445B000B4475
:102DF000034430331B78D8B209491346DB0013442F
:102E00005B0013440B4403F55C7302461A70BB7BF2
:102E10000133BB738DE700BF1037BD46B0BD00BFA7
:102E2000F4010020B0B584B000AF78604F4B93F848
:102E30002C307B7378680FF05DFD4C4B1B8E9BB282
:102E4000DAB27B6883F869207B7B002B03D00021FA
:102E500078680FF0ACFF454B1B8E9BB2002B14BF64
:102E600001230023DBB2002B03D0012178680FF08F
:102E70009EFF3E4B93F85433DAB27B68DA7400233A
:102E8000FB73FB7B022B6DD8FA7BFB7B37490A4433
:102E900092F85523D1B27A6813440A461A75FB7B1F
:102EA000FA7B324903F5D4735B000B441B8999B25A
:102EB0007B680C3223F812100023BB73BB7B102BF2
:102EC0001ED8F97BBC7BFA7BB87B284D0B46DB0018
:102ED0000B445B000B442B44234403F25E331B780A
:102EE000DCB279681346DB0013445B0013440B44E7
:102EF00003441E3322461A70BB7B0133BB73DDE7EC
:102F0000F97BFA7B19480B46DB000B445B000B4452
:102F1000034403F26F331B78D8B279681346DB00A1
:102F200013445B0013440B442F3302461A70F97BA1
:102F3000FA7B0E480B46DB000B445B000B4403445A
:102F400003F55C731B78D8B279681346DB00134431
:102F50005B0013440B44303302461A70FB7B013391
:102F6000FB738EE700BF1037BD46B0BDF4010020F3
:102F700080B582B000AF78607B6893F8783103F059
:102F80008103002B08D07B6893F8783183F002032B
:102F9000DAB27B6883F878217B6893F87931002B6B
:102FA0001CD17B6893F874311A467B68883233F8F9
:102FB0001230002B12D17B68B3F870311AB27B68E3
:102FC00093F87431194601238B401BB2DB431BB2CB
:102FD00013401BB29AB27B68A3F87021786800F0A6
:102FE0000FF87B6893F87831832B02D1034B0122D1
:102FF0001A7300BF0837BD4680BD00BFC01D00204A
:1030000080B582B000AF78607B6893F87831812B0F
:1030100002D0832B6FD096E07B6893F874311A4608
:10302000012393409AB24A4BDA827B6893F8743159
:103030001A46012393409AB2454BDA81444B5B8A8E
:103040009BB243F480539AB2414B5A82404B1B8A45
:103050009BB243F001039AB23D4B1A823D4A137969
:1030600043F0100313713C480FF0A6FC3A48FFF7F9
:10307000B9FC7B68B3F870217B68B3F872311340F8
:103080009BB21A467B6893F8743142FA03F303F05B
:103090000103002B06D07B6893F8743119467868D9
:1030A00000F0A0F87B68B3F870311A467B6893F89B
:1030B000743142FA03F303F00103002B07D12448D3
:1030C0000FF041F97B68FF2283F879213BE020482B
:1030D0000FF046F97B68B3F872311A467B6893F8B3
:1030E000743142FA03F3DBB203F00103DAB27B6816
:1030F00083F8792127E018480FF05EFC1648FFF7A7
:1031000039FD13480FF02CF9114B00229A82104B15
:103110000022DA820E4B0022DA810D4B1B8A9BB211
:1031200023F001039AB20A4B1A820A4A13796FF309
:1031300004131371064B5B8A9BB223F480539AB23B
:10314000034B5A8200BF00BF0837BD4680BD00BF99
:10315000C01D0020F4010020A81E0020B0B584B0DE
:1031600000AF78607B6893F874311C461C480EF001
:1031700060FF03461A467B68234483F800217B687E
:1031800093F874311A467B68134493F80031FB734B
:10319000FB7B002B20D07B6893F874311A467B6848
:1031A000134493F80021FB7BD31ADAB27B6893F8BF
:1031B00074311D46FB7B5C1E114609480EF055FF1D
:1031C000034619467A682B01134423440A461A70B1
:1031D000FB7B013BFB73DBE700BF1037BD46B0BD97
:1031E000A81E002080B582B000AF78600B46FB704F
:1031F0007B68FA7812019918FB787A68134493F87F
:1032000000311A4603480FF052FE00BF0837BD4692
:1032100080BD00BFA81E002090B585B000AF7860CB
:103220007B68B3F87021624BA3F8D4227B68B3F8B3
:1032300072215F4BA3F8D6220023FB73FB7B0F2B7D
:1032400000F2B180F97BFB7B7A684C3112F82120C7
:10325000C2F30102D1B2564AA4339B0013441A7937
:1032600061F301021A71F97BFB7B7A684C3112F829
:103270002120C2F38102D1B24D4AA4339B001344F2
:103280001A7961F383021A71F97BFB7B7A684C31FE
:1032900012F82120C2F30012D1B2454AA4339B0098
:1032A00013441A7961F304121A71F97BFB7B7A6873
:1032B0004C3112F82120C2F34212D1B23C4AA4335D
:1032C0009B0013441A7961F347121A71F97BFB7B57
:1032D0007A68883132F81110354A03F59C735B0027
:1032E00013440A469A80FB7BFA7B79680B4493F877
:1032F00000012F491346DB0013449B000B44543359
:1033000002461A700023BB7397F90E30072B3DDC81
:10331000FA7B97F90E305B00796812010A44134476
:103320001B78FA7B97F90E0003F00F03D9B2204CFB
:103330001346DB00134403440C339B0023441A79E7
:1033400061F303021A71FA7B97F90E305B000133C7
:10335000796812010A4413441B78FA7B97F90E002E
:1033600003F00F03D9B2124C1346DB00134403449D
:103370000C339B0023441A7961F307121A7197F9F1
:103380000E30DBB20133DBB2BB73BDE7002109486D
:103390000EF06BFE03461A46054B83F8D822FB7BE2
:1033A0000133FB734AE700BF1437BD4690BD00BF31
:1033B000F4010020A721002080B584B000AF786020
:1033C00078680FF0FFFD6C4BB3F8D4329AB27B688B
:1033D000A3F87021684BB3F8D6329AB27B68A3F891
:1033E00072210023FB73FB7B0F2B00F2AA80FB7B77
:1033F000F97B614AA4339B0013445B68C3F3010368
:10340000D8B27A684C3112F8213060F3010302F827
:103410002130FB7BF97B584AA4339B0013445B6843
:10342000C3F38103D8B27A684C3112F8213060F3CB
:10343000830302F82130FB7BF97B4F4AA4339B00C6
:1034400013445B68C3F30013D8B27A684C3112F8A6
:10345000213060F3041302F82130FB7BF97B464AEC
:10346000A4339B0013445B68C3F34213D8B27A6859
:103470004C3112F8213060F3471302F82130FB7B06
:10348000FA7B3D4903F59C735B000B449B8899B222
:103490007B68883223F81210FA7BF97B3648134692
:1034A000DB0013449B00034454331B78DAB27B687F
:1034B0000B4483F800210023BB7397F90E30072BD0
:1034C0003BDCFA7B97F90E102B481346DB001344C4
:1034D0000B440C339B0003445B68C3F30303D9B272
:1034E000FA7B97F90E305B000846796812010A44AE
:1034F000134402461A70FA7B97F90E101E481346C1
:10350000DB0013440B440C339B0003445B68C3F3A0
:103510000313D9B2FA7B97F90E305B0001330846EA
:10352000796812010A44134402461A7097F90E3062
:10353000DBB20133DBB2BB73BFE7FB7B0133FB7351
:1035400051E70D4B93F8D832DBB2FF2B14BF0123A8
:103550000023DBB2002B0AD07B6803F28F13064AEC
:1035600092F8D822D2B2114618460EF0E4FC00BF01
:103570001037BD4680BD00BFF401002090B585B076
:1035800000AF78607B68012283F88E217B6803F2AC
:103590008F1318460EF04DFD0346002B0AD07B68B2
:1035A00003F27B1318460EF044FD0346002B01D1B5
:1035B000012300E00023002B39D000213D480EF00C
:1035C00054FD034603F00F03DAB23B7B62F30303BF
:1035D0003B733B7B43F010033B733B7B6FF3451323
:1035E0003B733B7B6FF386133B733B7B6FF3C713DC
:1035F0003B737B6803F28F1318460EF076FCF96874
:103600002D480EF016FC00212A480EF02EFD034630
:103610001A46012303FA02F1284BDB8A9BB21AB245
:103620000BB213431BB29AB2244BDA821CE07B68C4
:1036300003F27B1318460EF0FCFC0346002B14BF6C
:1036400001230023DBB2002B0ED07B6803F28F1422
:103650007B6803F27B13002118460EF006FD03463B
:10366000194620460EF067FC7B6803F28F1318465C
:103670000EF0DFFC0346002B14BF01230023DBB256
:10368000002B12D000210B480EF0EFFC03461A4627
:10369000012303FA02F1094BDB8A9BB21AB20BB287
:1036A00013431BB29AB2054BDA8200BF1437BD46F2
:1036B00090BD00BFBB210020DC1D0020C01D0020EC
:1036C00080B582B000AF78607B68002283F88E21DD
:1036D0007B68FF2283F87A211A48FFF74BFA1948D2
:1036E0000FF06AF97B6803F27B1318460EF0FDFBBE
:1036F000154800F04DF8154B1B8A9BB223F48073DC
:103700009AB2124B1A82114B1B8A9BB223F00E0302
:103710009AB20E4B1A8200210D480EF0A6FC034609
:103720001A4601239340D943084BDB8A9BB21AB255
:103730000BB213401BB29AB2044BDA8200BF0837B7
:10374000BD4680BDA81E0020141F0020C01D002003
:10375000BB21002080B582B000AF78607B68043365
:1037600018460EF0B6FB7B681A3318460EF0B1FB14
:10377000054B064A1A62786800F00AF87B6818461A
:103780000837BD4680BD00BF6C1E0020941E00207F
:1037900080B582B000AF786007480EF0A6FB0748FE
:1037A0000EF045FE064B00229A8278680FF00AFE62
:1037B00000BF0837BD4680BD941E00206C1E00204F
:1037C000C01D002080B485B000AF78607B681B7896
:1037D000DAB22E4B83F824237B685B889AB22B4B9A
:1037E000A3F826230023FB73FB7B102B0ED8FA7B58
:1037F000FB7B79680A441279D1B2244A13440A4601
:1038000083F82823FB7B0133FB73EDE77B685B7D4B
:10381000DAB21E4B83F839237B689B7DDAB21B4BEF
:1038200083F83A237B68DB7DDAB2184B83F83C23BC
:103830007B681B8B9AB2154BA3F83E230023BB7306
:10384000BB7B102B0ED8BA7BBB7B79680A44927E77
:10385000D1B20E4A13440A4683F84023BB7B01339E
:10386000BB73EDE77B6893F82B30DAB2074B83F834
:1038700051237B6893F82C30DAB2044B83F852233F
:1038800000BF1437BD465DF8047B7047F40100208B
:1038900080B485B000AF78602F4B93F82433DAB250
:1038A0007B681A702C4BB3F826339AB27B685A8027
:1038B0000023FB73FB7B102B0ED8FA7BFB7B264986
:1038C0000A4492F82823D1B27A6813440A461A713E
:1038D000FB7B0133FB73EDE71F4B93F83933DAB20F
:1038E0007B685A751C4B93F83A33DAB27B689A7549
:1038F000194B93F83C33DAB27B68DA75164BB3F8A0
:103900003E339AB27B681A830023BB73BB7B102BB8
:103910000ED8BA7BBB7B10490A4492F84023D1B23F
:103920007A6813440A469A76BB7B0133BB73EDE792
:10393000094B93F85133DAB27B6883F82B20064B9E
:1039400093F85233DAB27B6883F82C2000BF143727
:10395000BD465DF8047B7047F401002090B585B04A
:1039600000AF78607B6801221A705E480EF061FB40
:103970000346002B14BF01230023DBB2002B00F011
:1039800087807B6800225A807B68043318460EF0DB
:10399000ACFA54480EF04DFB0346FB73FB7B002B47
:1039A00027D07B681C1DFB7B013BDBB219464D48D1
:1039B0000EF05BFB0346194620460EF0BCFAFB7B7B
:1039C000013BDBB2194647480EF04FFB03461A464F
:1039D000012303FA02F17B685B889BB21AB20BB237
:1039E00013431BB29AB27B685A80FB7B013BFB738B
:1039F000D4E77B68043318460EF01BFB03461C46D5
:103A000039480EF0F9FE03469C428CBF0123002387
:103A1000DBB2002B58D034480EF0EEFE0346BB73E9
:103A20007B68043318460EF004FB03461A46BB7B42
:103A3000934234BF01230023DBB2002B1DD07B68EF
:103A40001C1D7B680433BA7B114618460EF00DFB33
:103A50000346194620460EF0A3FA7B680433BA7B6E
:103A6000114618460EF001FB03461946786800F02F
:103A7000B7F8BB7B0133BB73D2E77B681C1D1A48C8
:103A80000EF0BAFE0346194620460EF0DFFA1BE0A0
:103A90007B68043318460EF0CCFA03467B737B7BBD
:103AA000002B11D07B681A1D7B7B013BDBB21946D2
:103AB00010460EF0DAFA03461946786800F066F808
:103AC0007B7B013B7B73EAE77B6893F82D30002B0F
:103AD00004D07B685B889AB2044BDA8100BF14374C
:103AE000BD4690BD941E00206C1E0020C01D00200D
:103AF00090B585B000AF78607B68043318460EF04F
:103B000098FA0346FB73FB7B002B2BD01D48FDF777
:103B1000E9F803461C467B681A1DFB7B013BDBB2C0
:103B2000194610460EF0A1FA034644FA03F303F0D7
:103B30000103002B0CBF01230023DBB2002B0DD0AF
:103B40007B681A1DFB7B013BDBB2194610460EF069
:103B50008CFA03461946786800F042F8FB7B013B7B
:103B6000FB73D0E77B6800221A707B6893F82D30D6
:103B7000002B02D0044B0022DA8100BF1437BD466F
:103B800090BD00BF601E0020C01D002080B582B027
:103B900000AF78600B46FB700E4B5B68C3F381038C
:103BA000DBB2032B02D1FB78022B01D9012300E009
:103BB0000023002B04D0FB78194607480EF0BBF910
:103BC000FB7819460548FDF789FB00BF0837BD465D
:103BD00080BD00BFF4010020941E00206C1E002058
:103BE00080B582B000AF78600B46FB700E4B5B680F
:103BF000C3F38103DBB2032B02D1FB78022B01D983
:103C0000012300E00023002B04D0FB78194607486D
:103C10000EF0C6F9FB78194605480EF095FC00BF7A
:103C20000837BD4680BD00BFF4010020941E00206F
:103C30006C1E002090B585B000AF786039603B788D
:103C400003F01003DBB2002B00F0D8808C4B5B68D4
:103C5000C3F38103DBB2022B08D1894B5B68C3F34A
:103C60000103DBB2022B01D1012300E00023002B72
:103C70000BD03B78C3F30303DBB2194681480EF047
:103C80005AF981480EF06EFDE4E07B681B78DBB2E8
:103C900083F00103DBB2002B08D03B78C3F30303AE
:103CA000DBB219467868FFF771FFD3E03B78C3F3C6
:103CB0000303DBB2194678680FF001FC034683F07A
:103CC0000103DBB2002B6BD07B681A1D3B78C3F37A
:103CD0000303DBB2194610460EF02DF97B6804335E
:103CE00018460EF0A6F903461C4667480EF084FD00
:103CF00003469C428CBF01230023DBB2002B46D03D
:103D000061480EF079FD0346FB737B680433184667
:103D10000EF08FF903461A46FB7B934234BF012312
:103D20000023DBB2002B28D07B680433FA7B1146DA
:103D300018460EF09AF9034619467868FFF750FFC7
:103D40007B680433FA7B114618460EF08EF9034661
:103D50001A460123934083F47F4383F0FF037A687C
:103D6000528892B212B21BB213401BB29AB27B6855
:103D70005A80FB7B0133FB73C7E77B681C1D4248FD
:103D80000EF03AFD0346194620460EF05FF93B78E7
:103D9000C3F30303DBB219467868FFF7F7FE11E0BF
:103DA0007B681A1D3B78C3F30303DBB21946104648
:103DB0000EF0F6F83B78C3F30303DBB219467868DC
:103DC000FFF70EFF7B685B889BB21AB23B78C3F3A8
:103DD0000303DBB2194601238B401BB253401BB2D5
:103DE0009AB27B685A807B6893F82D30002B31D0D3
:103DF0007B685B889AB2254BDA812BE0204B5B68AD
:103E0000C3F38103DBB2022B06D11D4B5B68C3F306
:103E10000103DBB2022B01D0012300E00023002BC1
:103E200010D07B681B78DBB283F00103DBB2002B80
:103E300010D03B78C3F30303DBB219467868FFF771
:103E4000CFFE07E03B78C3F30303DBB219460D480E
:103E50000EF0A6F80E4B93F87931002B0BD10C4BDA
:103E600093F87831812B06D17B685B889BB2194629
:103E700007480FF0EBF900BF1437BD4690BD00BFF7
:103E8000F4010020941E00206C1E0020C01D0020A4
:103E90002C20002090B585B000AF78600846114610
:103EA0001A4603467B800B467B7013463B703B787B
:103EB000194620480FF02DFA0346C3F30103DBB285
:103EC0001C463B7819461B480FF023FA0346C3F300
:103ED0008103DBB21A4621461748FDF7A9F90023F2
:103EE000BB600023FB73FB7B0F2B1FD87B8803F089
:103EF0000103002B13D0FB7B03F00F03DAB23B7AF4
:103F000062F303033B727B7803F00103DAB23B7A7E
:103F100062F304133B72B9687868FFF78BFE7B8805
:103F20005B107B80FB7B0133FB73DCE700BF143746
:103F3000BD4690BD2C2000206C1E002080B582B0B4
:103F400000AF78607B68012283F82D2003480EF0D3
:103F50008BFC00BF0837BD4680BD00BF6C1E002033
:103F600080B582B000AF78607B68002283F82D2096
:103F700003480EF086FC00BF0837BD4680BD00BF79
:103F80006C1E002080B582B000AF78607B68144A58
:103F900004331146C022184610F0E7FF7B68002268
:103FA00083F8C5207B68002283F8C6207B68002246
:103FB00083F8C7207B68002283F8C8207B684FF015
:103FC0000002C3F8CC207B68002283F8D0207868F8
:103FD00000F008F87B6818460837BD4680BD00BF72
:103FE000C454010080B483B000AF78601C4B002241
:103FF0005A821C4B002283F898237B68002283F8A6
:10400000D1207B68032283F8D2207B6817221A70A4
:104010007B68012283F8C4207B684FF00002C3F85C
:10402000CC207B68012283F8D0207B68002283F8B3
:10403000C7207B68002283F8C8200A4B002283F83F
:104040009923084B0022C3F8A023064B0022C3F893
:10405000A42300BF0C37BD465DF8047B704700BF4A
:10406000C01D0020F401002080B483B000AF786050
:10407000064B00225A827B68052283F8D12000BFBC
:104080000C37BD465DF8047B704700BFC01D0020A3
:1040900080B582B000AF78607868FFF7E5FF0F4821
:1040A0000DF0A8FE0E48FFF773FB7B68002283F833
:1040B000C8200C4B0022C3F8A4237B684FF00002F9
:1040C000C3F8CC207B68012283F8D0207B680022D3
:1040D00083F8D12000BF0837BD4680BDDC1D00201D
:1040E000141F0020F401002080B582B000AF78607A
:1040F0007B6893F8D130023B032B40D801A252F8E1
:1041000023F000BF3F4100001541000023410000A3
:10411000514100007868FFF7BBFF786800F084F831
:104120002DE07868FFF7B4FF174BD3F8A033013BBD
:10413000154AC2F8A433786800F08EF81FE078685A
:10414000FFF750FF786800F021F801F05DFA16E003
:104150007B6893F8D230032B02D0042B07D00DE0FC
:104160007868FFF795FF786800F05EF806E07868F9
:10417000FFF78EFF786800F06FF800BF00BF00BF48
:104180000837BD4680BD00BFF401002080B582B075
:1041900000AF78600E48FFF7FBFA0E4B93F89833A8
:1041A000DBB2002B14BF01230023DBB2002B03D0B2
:1041B00078680FF0A3F907E07B68012283F8D1202B
:1041C000054B42F201025A8200BF0837BD4680BD4E
:1041D000141F0020F4010020C01D002080B483B013
:1041E00000AF78607B6817221A700D4B012283F8AC
:1041F00098237B6893F8C530002B03D07B6801229D
:1042000083F8C6207B68022283F8D120054B4FF447
:1042100000525A8200BF0C37BD465DF8047B7047E0
:10422000F4010020C01D002080B483B000AF78608E
:104230007B68032283F8D1207B68032283F8D22095
:10424000044B00225A8200BF0C37BD465DF8047B48
:10425000704700BFC01D002080B483B000AF7860FD
:104260007B68042283F8D1207B68042283F8D22063
:10427000044B00225A8200BF0C37BD465DF8047B18
:10428000704700BFC01D002080B483B000AF7860CD
:104290000B46FB70FB78002B0FD0FB780E2B0CD855
:1042A0007B6893F9C430DBB21B01DAB2FB781344AC
:1042B000DBB25AB27B681A7021E0FB78002B0FD179
:1042C0007B6893F9C430002B19D07B6893F9C43014
:1042D000DBB2013BDBB25AB27B6883F8C4200EE04C
:1042E0007B6893F9C430012B09DC7B6893F9C430F7
:1042F000DBB20133DBB25AB27B6883F8C420044BD3
:1043000001221A7000BF0C37BD465DF8047B704770
:104310007C2C002090B585B000AF7860AC4B9B78CA
:1043200003F00103DBB2002B14D1A94B9B7803F0FF
:104330000203DBB2002B0DD1A54B9B7803F00403E5
:10434000DBB2002B06D1A24B9B7803F00403DBB257
:10435000002B02D0786800F0D9FA9E480EF09DFD3F
:104360000023BB609C4B1B78DBB2093B042B00F2A3
:10437000BA8201A252F823F0D54600008D43000016
:10438000E748000085470000374800007B681B7C39
:10439000002B57D08F480DF04CFE0346012B02D066
:1043A000032B17D041E07B685C7A002189480DF02F
:1043B0005CFE03462344DBB203F00F03DAB27B68F2
:1043C0009A727B685A7A7B68DA727B689A7A7B6821
:1043D0001A7343E07B685C7A00217E480DF045FE4D
:1043E00003462344DBB203F00F03DAB27B689A7210
:1043F0007B685C7A012177480DF037FE0346234441
:10440000DBB203F00F03DAB27B68DA727B685C7AA6
:10441000022170480DF029FE03462344DBB203F06D
:104420000F03DAB27B681A7318E07B685A7A7B68EC
:104430009A727B685A7A7B68DA727B685A7A7B68F0
:104440001A730BE07B685A7A7B689A727B685A7A97
:104450007B68DA727B685A7A7B681A730023FB7375
:10446000FB7B032B00F2FB807B68DB881946FB7B20
:104470007A6813445B7A41FA03F303F00103002BDB
:1044800000F0E98053480DF0D4FD0346032B4BD8D0
:1044900001A252F823F000BFA9440000C744000065
:1044A000E944000007450000FB7B002B37D14A4B55
:1044B0005B68C3F34213DBB21946FB7B1A464548DF
:1044C000FDF7EEFF2BE0FB7B03F00203002B28D16E
:1044D000414B5B68C3F34213DBB21946FB7B1A46C0
:1044E0003C48FDF7DDFF1CE0FB7B002B1BD13A4B6A
:1044F0005B68C3F34213DBB21946FB7B1A463548AF
:10450000FDF7CEFF0FE0344B5B68C3F34213DBB221
:104510001946FB7B1A462F48FDF7C2FF04E000BF97
:1045200002E000BF00E000BFFB7B032B00F29380A2
:1045300001A252F823F000BF494500006F4500007A
:10454000B745000009460000002122480EF0CAFAD3
:10455000034603F00F03D9B21D4A137861F3030336
:1045600013701B4A937843F00103937073E019486A
:104570000DF05FFD034603F00103012B03D07B68C0
:10458000DB7B002B01D0012300E00023002B5DD05A
:10459000012110480EF0A6FA034603F00F03D9B22A
:1045A0000B4A137861F307131370094A937843F0A9
:1045B000020393704AE007480DF03BFD0346032BCE
:1045C00003D07B68DB7B002B08D0012307E000BF12
:1045D000E4010020A81E0020F40100200023002B8D
:1045E00036D00221B5480EF07DFA034603F00F03E2
:1045F000D9B2B34A537861F303035370B04A937846
:1046000043F00403937023E0AC480DF012FD034621
:10461000032B03D07B68DB7B002B01D0012300E060
:104620000023002B16D00321A4480EF05BFA0346AA
:1046300003F00F03D9B2A24A537861F30713537002
:104640009F4A937843F00803937003E000BF02E0B1
:1046500000BF00E000BFFB7B0133FB7300E77B681A
:104660009B7B83F00103DBB2002B02D0954B002231
:10467000DA810023BB73BB7B032B00F22D817B68A7
:104680009B7B83F00103DBB2002B08D08E4B1B69B0
:10469000C3F34333DBB20A2B01D0012300E0002334
:1046A000002B13D0BB7B194684480EF01BFA03463F
:1046B0001A46012303FA02F1824BDB899BB21AB23C
:1046C0000BB213431BB29AB27E4BDA81BB7B013330
:1046D000BB73D0E77B68DB881A467B685B7A42FA5B
:1046E00003F303F00103002B00F0F88073480DF092
:1046F000A0FC0346002B08D1744B5B68C3F3421344
:10470000DBB2052B01D1012300E00023002B40F098
:10471000F5806E4B5B68C3F34213DBB21946674802
:10472000FEF71CF8002165480EF0DCF9034603F0A3
:104730000F03DAB23B7A62F303033B723B7A43F036
:1047400010033B72B9686248FFF774FA7B689B7B81
:1047500083F00103DBB2002B00F0C080002157483A
:104760000EF0C0F903461A46012303FA02F1554B35
:10477000DB899BB21AB20BB213431BB29AB2514BF4
:10478000DA81ABE07B68DB881A467B685B7A42FAA9
:1047900003F303F00103002B00F0A28047480DF063
:1047A00048FC0346002B08D1484B5B68C3F3421317
:1047B000DBB2052B01D1012300E00023002B40F0E8
:1047C0009F80424B5B68C3F34213DBB219463B4800
:1047D000FDF7C4FF002139480EF084F9034603F0C9
:1047E0000F03D9B2364A537861F3071353707B68CD
:1047F0009B7B83F00103DBB2002B08D0334B5B685B
:10480000C3F30013DBB2012B01D1012300E000232D
:10481000002B0AD0002129480EF064F903461A46FD
:10482000012393409AB2274BDA81254A937843F0CB
:104830000803937054E07B68DB881A467B685B7AD8
:1048400042FA03F303F00103002B4BD0214B93F802
:104850007831812B04D11F4B93F87931012B09D08A
:104860001C4B93F87831832B3CD11A4B93F87A3157
:10487000012B37D111480DF0DCFB0346002B0CBF98
:1048800001230023DBB2002B3CD105210B48FDF7AF
:1048900065FF002109480EF025F9034603F00F03D8
:1048A000DAB23B7A62F303033B723B7A43F01003C4
:1048B0003B72B9680648FFF7BDF913E0A81E002057
:1048C000E4010020C01D002000F00F40F401002092
:1048D000141F00202C20002000BF04E000BF02E0D5
:1048E00000BF00E000BF7B689B7B002B02D0786894
:1048F00000F02EF978680EF06EFE04E000BF02E0D2
:1049000000BF00E000BF1437BD4690BD80B584B045
:1049100000AF78600023FB60654B1B78DBB2093B7E
:10492000042B00F2BA8001A252F823F06B49000078
:10493000414900009B4A0000F74900003F4A00003F
:104940005C4A93786FF3000393705A4A93786FF33D
:1049500041039370574A93786FF382039370554ADB
:1049600093786FF3C303937097E0002152480EF0E1
:10497000B9F8034603F00F03DAB23B7B62F303039B
:104980003B733B7B6FF304133B73F9684B48FFF7B2
:1049900051F97B689B7B83F00103DBB2002B0AD0CB
:1049A000002145480EF09EF803461A460123934025
:1049B0009AB2434BDA813F4B9B7803F00103DBB2A1
:1049C000002B14D13B4B9B7803F00203DBB2002B8E
:1049D0000DD1384B9B7803F00403DBB2002B06D1DA
:1049E000344B9B7803F00803DBB2002B50D03348E4
:1049F000FEF7CEFE4CE02F4A93786FF3C30393701B
:104A00007B689B7B83F00103DBB2002B08D0284B33
:104A10005B68C3F30013DBB2012B01D1012300E07B
:104A20000023002B36D0002123480EF05BF803460C
:104A30001A46012393409AB2214BDA812AE0214B96
:104A400093F87831812B04D11E4B93F87931012BE7
:104A500009D01C4B93F87831832B1DD1194B93F857
:104A60007A31012B18D1002113480EF03BF8034690
:104A700003F00F03DAB23B7B62F303033B733B7B30
:104A80006FF304133B73F9680C48FFF7D3F803E0A6
:104A900000BF02E000BF00E000BF7B689B7B002BF3
:104AA00002D0786800F054F800BF1037BD4680BDD2
:104AB000F4010020E4010020A81E0020141F0020A3
:104AC000C01D00202C20002080B582B000AF78608F
:104AD0000C48FFF745FA0C480EF04EFA0B4B1B8AB8
:104AE0009AB27B681A80094BDB899AB27B685A803C
:104AF000064B9B8A9AB27B689A8000BF0837BD46F6
:104B000080BD00BF141F0020A81E0020C01D002073
:104B100080B582B000AF78600A48FFF70FFA0A4804
:104B20000EF01CFA7B681A88084B1A827B685A8838
:104B3000064BDA817B689A88044B9A8200BF08375B
:104B4000BD4680BD141F0020A81E0020C01D0020EF
:104B500080B483B000AF78607B68DA88034B9A82B8
:104B600000BF0C37BD465DF8047B7047C01D0020B8
:104B700080B582B000AF78607868FFF7A5FF094B79
:104B800001229A76074B0022DA81064B00229A8294
:104B90007868FFF7DDFF7B6801229A7300BF083752
:104BA000BD4680BDC01D002080B483B000AF7860DA
:104BB0000B46FB707B68DB881AB2FB78012101FA97
:104BC00003F31BB253401BB29AB27B68DA807B6856
:104BD000DA88044B9A8200BF0C37BD465DF8047B2F
:104BE000704700BFC01D002080B582B000AF786064
:104BF0007B68DA88134BA3F8DA227B681B7C1846A3
:104C00000EF027FD034603F00103D9B20D4A92F8D6
:104C1000DC3261F3000382F8DC327B68DB7B184610
:104C20000EF017FD034603F00103D9B2054A92F8CE
:104C3000DC3261F3410382F8DC3200BF0837BD4645
:104C400080BD00BFF401002080B582B000AF786065
:104C500078680EF08CFC134BB3F8DA329AB27B68AA
:104C6000DA80104BD3F8DC32C3F30003DBB25BB263
:104C700018460EF0FFFC03461A467B681A74094B6F
:104C8000D3F8DC32C3F34003DBB25BB218460EF05C
:104C9000F1FC03461A467B68DA7300BF0837BD464D
:104CA00080BD00BFF401002080B483B000AF786005
:104CB0007B684FF000021A607B684FF07E525A60AA
:104CC0007B68134A9A607B689A687B68DA607B68C5
:104CD0004FF000025A617B684FF07C52DA617B68CA
:104CE0005A697B689A617B684FF07E521A627B68D2
:104CF00000225A627B6804229A627B684FF07C52E1
:104D00001A617B6818460C37BD465DF8047B704716
:104D10000AD7233C80B52DED028B84B000AF7860BC
:104D200087ED000A7B68D3ED037A97ED007A77EE82
:104D3000677AC7ED037AD7ED037AF5EEC07AF1EE24
:104D400010FA27D57B6893ED027A7B68D3ED007A61
:104D500037EE677AD7ED037A27EE278A7B6893EDE3
:104D6000037A7B68D3ED007A77EE677ADFED330A5A
:104D7000B0EE670A78680EF0D9FEF0EE407A88EE61
:104D8000277A7B68D3ED027A77EE277A7B68C3EDCA
:104D9000027A2DE0D7ED037AF5EEC07AF1EE10FA43
:104DA00026DD7B6893ED017A7B68D3ED027A37EEDE
:104DB000677AD7ED037A27EE278A7B6893ED017A2D
:104DC0007B68D3ED037A77EE677ADFED1C0AB0EEED
:104DD000670A78680EF0AAFEF0EE407A88EE277A2D
:104DE0007B68D3ED027A77EE277A7B68C3ED027A8F
:104DF0007B68D3ED027A7B6893ED007A7B68D3ED14
:104E0000016AB0EE661AF0EE470AB0EE670A7868FB
:104E10000EF0A9FEF0EE407A7B68C3ED027A7B6863
:104E20003A68DA607B689B6807EE903AB0EE670AF2
:104E30001037BD46BDEC028B80BD00BFBD37863547
:104E400080B483B000AF1A4B1B6CC3F38023DBB27A
:104E5000174983F00103DAB2B1F8403062F38A23D4
:104E6000A1F840301249B1F8403062F3CB23A1F8E9
:104E700040300023FB80FB884FF6FF729342E2D064
:104E800000233B603B680F2B0EDC094A3B6803F0B4
:104E90000F03D9B2D2F8803061F34813C2F88030E2
:104EA0003B6801333B60EDE7FB880133FB80E2E7C1
:104EB00000F00F4080B582B000AF00237B607B68BC
:104EC000DBB21A46002115480EF0F5FB7B68DBB219
:104ED0001A46032111480EF0EEFB7B68DBB21A463E
:104EE00005210F480EF0E7FB7B68DBB21A46012173
:104EF0000C480EF0E0FB00233B603B68C72B05DC51
:104F00000EF0A2FE3B6801333B60F6E77B68002BA6
:104F10000CBF01230023DBB27B60D0E740F00F40E1
:104F2000C0F00F4080F00F4080B584B000AF7860D3
:104F30000B46FB70FB78284A32F813301A467B6820
:104F4000934201DA002343E0FB78234A103332F81E
:104F500013301A467B68934202DD4FF6FF7337E049
:104F6000FB781D4A32F813301A467B689B1A07EE0D
:104F7000903AF8EEE76AFB78174A103332F81330AC
:104F80001946FB78144A32F81330CB1A07EE903AE0
:104F9000B8EEE77AC6EE877AC7ED037AFB780E4A59
:104FA00010339B001344D3ED007AF0EE670A97EDBF
:104FB000030A0BF061FE87ED030AD7ED037A9FED3C
:104FC000077A67EE877AFCEEE77A17EE903A9BB2A3
:104FD00018461037BD4680BDC01B002000FF7F472C
:104FE00080B59EB000AF002387F8773001233B6780
:104FF000AC4BD3F81031C3F38063DBB2002B00D08D
:10500000F6E7A94B01221A70A84B1B78002B00F081
:10501000B982002387F8773097F877300F2BF3D8D1
:1050200001220A21A2480EF046FB01220B21A048D2
:105030000EF041FB9F4B4FF4F0729A6097F8773077
:105040005A019C4B5A609C4B1B7897F877209A42E8
:1050500004D100220B2196480EF02DFB97F87730F3
:10506000042B02D13B6F002B19D197F87730052B19
:1050700002D13B6F002B12D08A4B1B69C3F3433321
:10508000DBB2012B03D197F87730002B07D097F8CC
:1050900077208A4B93F8803008339A4201D101235C
:1050A00000E00023002B04D000220A2180480EF0EB
:1050B00002FB814B1B781A46814B33F812301B13CD
:1050C0007D4A127810467F4A9B0013441A687B4938
:1050D00000F110039B000B441A60774B1B781846B5
:1050E000754B1B781946764A00F1100332F81320ED
:1050F0004B0007F178010B4423F8482C6E4B1B78CA
:105100005B0007F17802134433F8483C18466B4BB8
:1051100093F880301A466C4B53F82230664A127866
:10512000114698428CBF01230023DAB207F17803BD
:105130000B4403F8782C604B1B7818465E4B1B78A9
:105140001946624A00F1100332F813204B0007F1B0
:1051500078010B4423F8282C574B1B785B0007F190
:105160007802134433F8283C1A13534B1B7892B23D
:105170005B0007F178010B4423F8682C4E4B1B7839
:1051800007F17802134413F8783C002B10D097F8FD
:105190007720494B1B785B0007F178010B4433F80B
:1051A000683C9A4204DA00220A2141480EF083FA50
:1051B000414B1B7807F17802134413F8783C002B1D
:1051C00014D0012200213A480EF075FA0122032181
:1051D00037480EF070FA012205213D480EF06BFAB7
:1051E0000122012133480EF066FA13E0002200216B
:1051F0002F480EF060FA002203212D480EF05BFAD2
:105200000022052132480EF056FA002201212948D9
:105210000EF051FA234BD3F81031C3F38063DBB2A5
:10522000002B17D001233B67244B93F880301A469C
:10523000284B53F82210204B1B781A4689B21F4B7B
:1052400023F812101C4B1B781C4A10334FF6FF71C9
:1052500022F81310134B1B69C3F34333DBB2012B4A
:105260000CBF01230023DBB2002B46D0124B1B786E
:1052700007F17802134413F8783C002B3DD03B6FC4
:10528000002B29D00C4B1B7819460B4B1B781A4668
:105290004B0007F178010B4433F8481C074B23F807
:1052A00012102AE000F00F407F2C00208E2C0020EE
:1052B00040F00F4080F00F408D2C0020C01B0020DC
:1052C000A0010020B4550100A0550100381B0020AA
:1052D000C0F00F408C550100A64B1B781A46A54B19
:1052E0001B781846530007F17802134433F8481C22
:1052F000A14A00F1100322F81310A04B1B69C3F35D
:105300004333DBB2052B0CBF01230023DBB2002BA0
:1053100001D001233B67994B1B69C3F34333DBB2D5
:10532000062B0CBF01230023DBB2002B01D000238E
:105330003B67924B1B69C3F34333DBB2082B0CBFB3
:1053400001230023DBB2002B58D08C4B1B69C3F325
:105350004333DBB2082B0CBF01230023DBB2002B4D
:1053600000D0F2E7834B1B781A46834B33F81220A8
:10537000804B1B788049103331F813309A422DD975
:105380007C4B1B781A467B4B1B7819467A4B33F8BB
:1053900012204B0007F178010B4423F8682C754B61
:1053A0001B781846734B1B781946734A00F110039B
:1053B00032F81320704B23F811206E4B1B781A46DD
:1053C0006C4B1B781846530007F17802134433F8EE
:1053D000681C694A00F1100322F81310654B1B7812
:1053E0000E2B08D801233B67624B1B780133DAB2DE
:1053F000604B1A7002E0624B00221A705F4B1B690F
:10540000C3F34333DBB2072B0CBF01230023DBB212
:10541000002B58D0594B1B69C3F34333DBB2072B26
:105420000CBF01230023DBB2002B00D0F2E7514B6D
:105430001B781A46504B33F812204E4B1B784E49BE
:10544000103331F813309A422DD94A4B1B781A4643
:10545000484B1B781946484B33F812204B0007F194
:1054600078010B4423F8682C424B1B781846414BBB
:105470001B781946404A00F1100332F813203E4BC6
:1054800023F811203B4B1B781A463A4B1B781846E1
:10549000530007F17802134433F8681C364A00F1D0
:1054A000100322F81310334B1B78002B08D0012374
:1054B0003B67304B1B78013BDAB22E4B1A7002E08F
:1054C0002F4B00221A702D4B1B69C3F34333DBB201
:1054D000092B0CBF01230023DBB2002B03D0264B8A
:1054E000002283F88020254B1B69C3F34333DBB2D2
:1054F0000A2B0CBF01230023DBB2002B03D01E4B71
:10550000012283F880201D4B1B69C3F34333DBB2B8
:105510000B2B0CBF01230023DBB2002B03D0164B57
:10552000022283F88020154B1B69C3F34333DBB29F
:105530000C2B0CBF01230023DBB2002B03D00E4B3E
:10554000032283F880200D4B1B69C3F34333DBB286
:105550000D2B0CBF01230023DBB2002B03D0064B25
:10556000042283F8802097F87730013387F877306A
:1055700052E500BF8D2C0020C01B002000F00F4022
:105580008E2C00200B4B00221A700B4B1868012345
:105590000A4A0B4905F04AFD0346002B14BF0123BC
:1055A0000023DBB2002B01D0FFF74AFC00BF7837A5
:1055B000BD4680BD7F2C002000010020BFC3C90173
:1055C000C01B002080B483B000AF0346FB71FB79A1
:1055D000052B0BD10B4B1B78DBB2092B06D0094BEB
:1055E0001B78DBB20C2B01D0012300E00023002B41
:1055F00001D0042300E0FB7918460C37BD465DF866
:10560000047B7047F401002098B500AF954B5B68B0
:10561000C3F30013DBB21AB2924B1B78DBB2013B2F
:10562000012101FA03F31BB213431CB28E48FCF7AD
:10563000B5F90346C3F30103DBB20133012202FAD9
:1056400003F31BB223431BB29AB2884B1A82874BD7
:105650001B7BDBB2002B0AD0844B1B8A9BB223F04E
:105660000E039AB2814B1A82804B00221A737D4B33
:105670001B78DBB20A2B0CBF01230023DBB2002B0B
:1056800007D07A4B1B8A9BB223F00E039AB2774B5A
:105690001A82744B5B68C3F34213DBB2002B14BF56
:1056A00001230023DBB2002B59D06E4B1B78DBB2F9
:1056B000092B09D06B4B1B78DBB20A2B04D0694B4A
:1056C0001B78DBB20C2B01D1012300E00023002B5F
:1056D0000FD0644B5B68C3F34213DBB21846FFF78D
:1056E00071FF03460433DBB2012219465F480CF018
:1056F000F1FD5C4B1B78DBB20E2B0CBF01230023AA
:10570000DBB2002B2BD0574B93F89933DBB2002B35
:105710000CBF01230023DBB21A460F2153480CF0C3
:10572000D9FD534B93F8D130052B12D0052B16DC45
:10573000032B02D0042B06D011E0012208214B4894
:105740000CF0C8FD0BE00122072148480CF0C2FD17
:1057500005E00122012145480CF0BCFD00BF454B8E
:105760009B7B002B08D0414B5B8A9BB243F4804368
:105770009AB23E4B5A8207E03C4B5B8A9BB223F4C1
:1057800080439AB2394B5A82364B1B78DBB20D2BD1
:105790000BD1394B93F87831812B06D1364B93F8E6
:1057A0007931FF2B01D0012300E00023002B18D01A
:1057B000314B93F87931002B0AD0012B11D12B4BAF
:1057C0001B8A9BB243F480739AB2284B1A8208E07A
:1057D000264B1B8A9BB243F480639AB2234B1A82F6
:1057E00000BF204B1B78DBB20A2B0CBF0123002328
:1057F000DBB2002B20D01F4B1B7C002B07D01B4B98
:105800001B8A9BB243F004039AB2184B1A82194BBD
:10581000DB7B002B08D0154B1B8A9BB243F008039F
:105820009AB2124B1A8207E0104B1B8A9BB243F0CC
:1058300002039AB20D4B1A82104B1B78002B07D033
:105840000F4B1B781A46102108480CF043FD06E068
:105850000C4B1B781A46102104480CF03BFD00BF8E
:1058600098BD00BFF40100206C1E0020C01D002068
:10587000441F0020182000202C200020802C002015
:10588000832C0020822C002090B583B000AFA74964
:1058900009787971797901390E2901F2668001A0C0
:1058A00050F821F0E1580000495A00000F5B000059
:1058B000D35B0000B35C0000D95C0000FF5C00001B
:1058C000015E0000E75E0000A56000005B62000072
:1058D00071630000F9640000D1660000D767000022
:1058E000934B1B78DBB20C2B1ED0914B1B78DBB299
:1058F0000E2B19D08E4B5B68C3F38103DBB2032BF5
:1059000012D08B4B1B78DBB20F2B0DD0884B1B7842
:10591000DBB20D2B08D0874B9B7B83F00103DBB2FE
:10592000002B01D0012300E00023002B37D0804B57
:105930005B68C3F30013DBB283F00103D9B27C4A86
:10594000137961F304131371794B1B78DBB20B2BC2
:105950000CBF01230023DBB2002B08D0744B5B6823
:10596000C3F30013DBB2194673480DF087FD704B8B
:105970001B78DBB2092B04D06D4B1B78DBB20A2BF2
:1059800001D1012300E00023002B08D0684B5B68A5
:10599000C3F30013DBB2194668480DF024FA644BD8
:1059A0001B78DBB20D2B0BD1654B93F87831832B31
:1059B00004D0634B93F87831032B01D1012300E02D
:1059C0000023002B19D05A4B5B68C3F30013DBB2E2
:1059D00083F00103D9B2564A137961F304131371AA
:1059E00057480DF0E2FC0346002B0CBF01230023B7
:1059F000DBB2194652480DF0C4FC4D4B1B78DBB2AC
:105A00000E2B0CBF01230023DBB2002B00F07E879E
:105A10004C4B93F8D130052B08D0052B00F376873B
:105A2000032B07D0042B09D000F070BF45480DF0C0
:105A300065FD07E04348FEF717FB03E04148FEF72A
:105A400013FB00BF00F062BF3A4B9B7B83F0010366
:105A5000DBB2002B06D0364B1B78DBB20A2B01D011
:105A6000012300E00023002B41D0314B1B78DBB237
:105A70000D2B14BF01230023DBB2002B1FD02C4BB6
:105A80005B68C3F30103DBB2002B14BF01230023C7
:105A9000DBB2002B2BD02C4B0022DA81244A137965
:105AA0006FF301031371294B1B78DBB203F003037F
:105AB000D9B21F4A137961F38303137117E0204BA6
:105AC00093F87831812B12D11D4B93F87931012B4A
:105AD0000DD16FF30102022363F383026FF304120B
:105AE000052363F34712114615480DF0FEFB104BDA
:105AF0001B78DBB20A2B0CBF01230023DBB2002B87
:105B000000F006870B4B0022DA7300F001BF094B4F
:105B10009B7B83F00103DBB2002B19D0044B1B7875
:105B2000DBB20A2B14D0012313E000BF792C002034
:105B3000F401002018200020141F0020A81E0020BF
:105B40002C200020441F0020C01D0020F405002050
:105B50000023002B29D0A34B1B78DBB20D2B14BFE5
:105B600001230023DBB2002B1FD09E4B5B68C3F3E5
:105B70000103DBB2012B14BF01230023DBB2002B96
:105B800013D0994B0022DA81964A1379012161F3EF
:105B900001031371954B5B78DBB203F00303D9B2B9
:105BA000904A137961F3830313718E4B1B78DBB238
:105BB0000A2B0CBF01230023DBB2002B00F0BC86B4
:105BC0008B4B1B7C83F00103DAB2894B1A7400F013
:105BD000B3BE874A927B82F00102D2B2002A06D07D
:105BE000804A1278D2B20A2A01D0012200E00022B3
:105BF000002A4ED07B4A1278D2B20D2A14BF01225D
:105C00000022D2B2002A2CD0764B5B68C3F301038A
:105C1000DBB2022B14BF01230023DBB2002B38D0F0
:105C2000704A1379022161F3010313716F4B9B7862
:105C3000DBB203F00303D9B26A4A137961F3830339
:105C40001371684B5B68C3F38103DBB2032B0CBF9A
:105C500001230023DBB2002B1BD0634B0722DA8128
:105C600017E0644A92F87821812A12D1614A92F8A9
:105C70007921012A0DD1022262F301036FF383031C
:105C80006FF30413052262F34713194659480DF0C8
:105C90002CFB544B1B78DBB20A2B0CBF01230023D7
:105CA000DBB2002B00F04A86514B0122DA7300F080
:105CB00045BE4F4B9B7B83F00103DBB2002B00F012
:105CC0003F86484A1379012161F347131371464B0C
:105CD00001229A7600F034BE454B9B7B83F0010392
:105CE000DBB2002B00F02E863E4A1379022161F3CD
:105CF000471313713C4B01229A7600F023BE3C4BB4
:105D00009B7B83F00103DBB2002B00F01D86354B3B
:105D10001B78DBB20E2B0CBF01230023DBB2002B60
:105D20001DD0354B93F8D130042B15D0324B93F85E
:105D3000D130022B04D0304B93F8D130032B0ED14D
:105D40002D4B93F8D130022B02D12B48FEF7A0F94E
:105D50002948FEF781FA02E02748FEF7C5F9214BF2
:105D60001B78DBB20D2B0CBF01230023DBB2002B11
:105D70002DD0204B93F87831812B40F0E5851F48DA
:105D8000FDF706FD1B480DF0D4F91A4B93F8793155
:105D9000002B13D1012119480DF070FB15480DF0AF
:105DA0006AFA03461C4613480DF0C4FA0346012262
:105DB00021461248FEF76EF800F0C6BD00210F48DC
:105DC0000DF05CFB0B48FDF71BF900F0BDBD054A6B
:105DD0001379032161F347131371034B01229A7660
:105DE00000F0B2BDF4010020C01D0020F405002029
:105DF000182000202C200020441F0020141F002009
:105E0000B24B9B7B83F00103DBB2002B00F09E853D
:105E1000AF4B1B78DBB20E2B0CBF01230023DBB290
:105E2000002B1DD0AB4B93F8D130032B15D0A94BD1
:105E300093F8D130022B04D0A64B93F8D130042B29
:105E40000ED1A44B93F8D130022B02D1A148FEF71A
:105E50001FF9A048FEF7E8F902E09E48FEF744F972
:105E60009B4B1B78DBB20D2B0CBF01230023DBB255
:105E7000002B2DD0984B93F87831812B40F066851C
:105E80009648FDF785FC94480DF03BF9924B93F84A
:105E90007931002B13D1012190480DF0EFFA8E4893
:105EA0000DF0E9F903461C468B480DF043FA034612
:105EB000012221468948FDF7EDFF00F047BD002192
:105EC00086480DF0DBFA8448FDF79AF800F03EBDF5
:105ED0007F4A1379042161F347131371804B012228
:105EE0009A7600F033BD794B9B7B83F00103DBB2E4
:105EF000002B00F02D85764B5B68C3F34213DBB2B9
:105F0000002B0CBF01230023DBB2002B05D0704A0D
:105F10001379052161F3471313716D4B1B78DBB2C5
:105F20000E2B0CBF01230023DBB2002B02D06948EB
:105F3000FEF7AEF8664B1B78DBB20B2B0CBF0123D0
:105F40000023DBB2002B25D064480DF051FA604BE2
:105F50005B68C3F30103DBB2022B08D15C4B5B68C7
:105F6000C3F38103DBB2032B01D1012300E0002343
:105F7000002B0FD0564A13796FF383031371544BE0
:105F80005B68C3F38103DBB21A46564B9A70544BDD
:105F90000022DA814E4B1B78DBB2092B0CBF0123A8
:105FA0000023DBB2002B07D0494A1379052161F3A6
:105FB0004713137100F0CCBC454B1B78DBB20A2BA6
:105FC0000CBF01230023DBB2002B08D046480CF0A5
:105FD00091FF4548FCF706FD4348FCF7CBFD3C4BE1
:105FE0001B78DBB20D2B06D13B4B93F87831812B1C
:105FF00001D0012300E00023002B02D03648FDF73A
:106000005FFB334B1B78DBB20D2B06D1324B93F881
:106010007831812B01D1012300E00023002B0BD02C
:106020002D480DF09EF82D48FDF7B2FB00212B48BE
:106030000DF024FA00F08CBC00212B480CF0B7FEC8
:10604000234A13796FF3041313712448FDF7A0FB5F
:1060500026480CF0FCFB24480CF060FF0346012BA3
:106060000CBF01230023DBB2002B08D0184A1379A0
:1060700043F0100313711C48FCF7B4FC0AE0144A07
:1060800013796FF3041313711748FCF7ABFC164830
:10609000FCF770FD0E4B09221A70114B01229A7603
:1060A00000F056BC094B9B7B83F00103DBB2002B55
:1060B00000F05084064B1B78DBB20D2B18D1064B39
:1060C00093F87831812B13D1012312E0182000209E
:1060D000F4010020441F00202C200020141F002069
:1060E000C01D0020F4050020A81E00206C1E00200A
:1060F0000023002B40F08884A74B1B78DBB20D2BCC
:1061000006D1A64B93F87831812B01D0012300E012
:106110000023002B02D0A148FDF7D2FA9E4B1B783A
:10612000DBB20B2B0CBF01230023DBB2002B25D0ED
:106130009B480DF05DF9984B5B68C3F30103DBB23C
:10614000022B08D1944B5B68C3F38103DBB2032BB2
:1061500001D1012300E00023002B0FD08E4A1379D8
:106160006FF3830313718C4B5B68C3F38103DBB262
:106170001A468C4B9A708C4B0022DA81864B1B7826
:10618000DBB20E2B0CBF01230023DBB2002B02D0AD
:106190008648FDF77DFF804B1B78DBB2092B09D0C9
:1061A0007D4B1B78DBB20C2B04D07B4B1B78DBB216
:1061B0000D2B01D1012300E00023002B12D0764BE0
:1061C0001B78DBB2092B0CBF01230023DBB2002BB1
:1061D00002D077480CF08EFE7548FCF703FC74483B
:1061E000FCF7C8FC6C4B1B78DBB20A2B14BF0123F5
:1061F0000023DBB2002B00F0AD8301216C480CF0D2
:10620000D6FD6748FDF7C4FA6A480CF020FB6848E1
:106210000CF084FE0346012B0CBF01230023DBB2EC
:10622000002B08D05C4A137943F0100313716048C7
:10623000FCF7D8FB0AE0584A13796FF30413137183
:106240005B48FCF7CFFB5A48FCF794FC524B0A2200
:106250001A70554B01229A767CE3574B9B7B83F057
:106260000103DBB2002B00F077834B4B1B78DBB2D2
:106270000E2B0CBF01230023DBB2002B02D04B48B6
:10628000FDF706FF444B1B78DBB2092B09D0424BCC
:106290001B78DBB20A2B04D03F4B1B78DBB20C2BF4
:1062A00001D1012300E00023002B1AD03A4B1B78C8
:1062B000DBB2092B02D00A2B04D007E03C480CF0DB
:1062C00019FE03E03A480CF015FE00BF3848FCF711
:1062D00089FB3748FCF74EFC2F4A13796FF3041300
:1062E00013712D4B1B78DBB20D2B06D12B4B93F882
:1062F0007831812B01D0012300E00023002B07D04F
:106300002648FDF7DDF9244A13796FF3041313715E
:10631000214B1B78DBB20D2B06D1204B93F8783143
:10632000812B01D1012300E00023002B07D01B4863
:106330000CF044FF01211A480DF0A0F80CE31848B6
:10634000FDF726FA144B5B68C3F30013DBB2194662
:1063500013480DF093F817480CF079FA0E4B0B2206
:106360001A700F480DF067F80F4B00229A76F3E28F
:10637000114B9B7B83F00103DBB2002B00F0EE821C
:10638000054B1B78DBB20D2B18D1044B93F87831F9
:10639000812B13D1012312E0F40100202C200020D6
:1063A000141F0020F4050020C01D0020441F002001
:1063B000A81E00206C1E0020182000200023002BA7
:1063C00040F024839C4B1B78DBB20D2B06D19B4BFA
:1063D00093F87831812B01D0012300E00023002BBA
:1063E00002D09648FDF76CF9934B1B78DBB20B2B70
:1063F0000CBF01230023DBB2002B25D090480CF00A
:10640000F7FF8D4B5B68C3F30103DBB2022B08D1AE
:10641000894B5B68C3F38103DBB2032B01D10123FA
:1064200000E00023002B0FD0834A13796FF383031E
:106430001371814B5B68C3F38103DBB21A46814B56
:106440009A70814B0022DA817B4B1B78DBB20E2BDA
:106450000CBF01230023DBB2002B02D07B48FDF7E9
:1064600017FE754B1B78DBB2092B0CBF01230023F1
:10647000DBB2002B02D07648FCF7B4FA6E4B1B78E7
:10648000DBB20A2B04D06C4B1B78DBB20D2B01D195
:10649000012300E00023002B05D06D48FCF7A2FA91
:1064A0006B48FCF767FB002169480CF080FC624BED
:1064B0001B78DBB20C2B14BF01230023DBB2002BB3
:1064C0000ED06348FCF78EFA5D48FDF761F961482C
:1064D0000CF0B0F9584B0C221A705B4B01229A76E3
:1064E000554A13796FF304131371574B00229A82A4
:1064F000554B0022DA8131E2574B9B7B83F001033D
:10650000DBB2002B00F02C824B4B1B78DBB20B2B49
:106510000CBF01230023DBB2002B25D048480CF030
:1065200067FF454B5B68C3F30103DBB2022B08D165
:10653000414B5B68C3F38103DBB2032B01D1012321
:1065400000E00023002B0FD03B4A13796FF3830345
:106550001371394B5B68C3F38103DBB21A46394BC5
:106560009A70394B0022DA81334B1B78DBB20E2B49
:106570000CBF01230023DBB2002B02D03348FDF710
:1065800087FD2F48FDF704F92B4B1B78DBB20D2B51
:1065900014BF01230023DBB2002B5FD0264B1B78F6
:1065A000DBB2092B09D0244B1B78DBB20C2B04D0B7
:1065B000214B1B78DBB20A2B01D1012300E0002321
:1065C000002B05D02248FCF70DFA2148FCF7D2FA3F
:1065D000194B0D221A7002211D480CF0E8FB1D48D2
:1065E0000CF035F915480CF069FD0023FB71002310
:1065F000BB71BB790F2B12D8BB7919460F480CF031
:10660000A6FE0346012B0CBF01230023DBB2002BA7
:1066100001D00123FB71BB790133BB71E9E7074B63
:1066200093F87831812B47D1FB79002B44D0034874
:10663000FCF79EFC40E000BFF40100202C2000206D
:10664000141F0020F4050020C01D0020441F00205E
:10665000A81E00206C1E002018200020AD48FCF76A
:1066600087FCAC480CF0A1FE0346002B14BF0123AD
:106670000023DBB2002B03D00021A6480CF081FEE2
:10668000A44B93F87831812B16D1A24B93F8793132
:10669000002B11D10121A0480CF0F0FE9D480CF018
:1066A000EAFD03461C469B480CF044FE03460122CB
:1066B00021469948FDF7EEFB984BDB899BB27B8026
:1066C0007B889AB2954BDA81944B01229A7647E106
:1066D000934B9B7B83F00103DBB2002B00F04281E4
:1066E000904B1B78DBB20B2B0CBF01230023DBB2DA
:1066F000002B25D088480CF07BFE8A4B5B68C3F3E7
:106700000103DBB2022B08D1864B5B68C3F3810324
:10671000DBB2032B01D1012300E00023002B0FD0BB
:10672000804A13796FF3830313717E4B5B68C3F365
:106730008103DBB21A467C4B9A70784B0022DA81D7
:10674000784B1B78DBB20D2B06D1724B93F8783166
:10675000812B01D1012300E00023002B40F0588160
:10676000704B1B78DBB20D2B06D16A4B93F8783156
:10677000812B01D0012300E00023002B02D06548CB
:10678000FCF79EFF674B1B78DBB20E2B0CBF01237F
:106790000023DBB2002B05D0624A13796FF3041398
:1067A0001371DFE05F4A13796FF3041313715F48CD
:1067B000FCF7E0F900215D480CF0F9FA594B0E2284
:1067C0001A705548FCF7E4FF59480CF040F8594856
:1067D000FDF7DCFCC6E0534B1B78DBB20E2B06D07A
:1067E000504B1B78DBB20B2B01D0012300E00023C0
:1067F000002B5FD04A4B9B7B83F00103DBB2002B65
:1068000025D0484B1B78DBB2092B04D0454B1B78B5
:10681000DBB20A2B01D1012300E00023002B12D0B0
:1068200042480CF067FB4148FCF7DCF83D4B5B68E5
:10683000C3F30013DBB283F00103DBB2002B02D001
:106840003A48FCF797F93648FEF792F98CE034485D
:106850000CF0B3FE334B1B78DBB20C2B14BF0123BF
:106860000023DBB2002B7FD030480BF0E2FB034665
:10687000002B05D12D480CF051FB0346002B01D015
:10688000012300E00023002B08D0264A137943F0AF
:10689000100313712548FCF7A5F865E0214A137928
:1068A0006FF3041313712148FCF79CF81F48FCF7A1
:1068B00061F959E018480CF0F5FD034683F0010337
:1068C000DBB2002B05D0174A13796FF30413137151
:1068D00004E0144A137943F010031371114B1B7831
:1068E000DBB20E2B0CBF01230023DBB2002B3BD00D
:1068F0000C4B93F89933DBB2002B0CBF0123002320
:10690000DBB21A46074B83F899232DE000BF2CE039
:1069100000BF2AE02C200020141F0020C01D0020F2
:1069200018200020F4010020F4050020A81E0020FB
:106930006C1E0020441F002000BF16E000BF14E0C2
:1069400000BF12E000BF10E000BF0EE000BF0CE08F
:1069500000BF0AE000BF08E000BF06E000BF04E09F
:1069600000BF02E000BF00E000BF2B4B1B78DBB292
:106970000D2B06D1294B93F87831812B01D10123BE
:1069800000E00023002B1ED024480CF0D3FC03466B
:10699000194622480CF0BDFC0346C3F30103DBB2E9
:1069A0001C461E480CF0C6FC034619461B480CF05A
:1069B000B0FC0346C3F38103DBB21A4621461848F4
:1069C000FAF736FC1DE0144B1B78DBB20D2B06D119
:1069D000124B93F87831832B01D1012300E000237F
:1069E000002B0ED10C4B5B68C3F30103DBB21946DD
:1069F000094B5B68C3F38103DBB21A460848FAF718
:106A000017FCFEF701FE04E000BF02E000BF00E05B
:106A100000BF0C37BD4690BDF40100202C200020A3
:106A20006C1E002080B500AF404B00221A70404B16
:106A300000221A813F4B93F87831812B02D13D48D7
:106A4000FCF796FA3C480BF0D4FB3C480BF0D2F92B
:106A50003B480BF0B5FC3B480BF0E9FC3A480BF027
:106A600044FA3A480BF046FF39480CF0ABFC384882
:106A7000FCF78EFE2F480CF0A5FA314B2F4A9A6096
:106A80004FF4806200212A480EF07DFA284B012243
:106A900083F8E022264B0B221A702E4B0B221A7021
:106AA000FEF7F2FE224A13796FF301031371204AB5
:106AB00013796FF3830313711D4B5B68C3F30103F9
:106AC000DBB219461A4B5B68C3F38103DBB21A468B
:106AD0001C48FAF7ADFB164A1379042161F34713FA
:106AE0001371134A13796FF3041313711A4B0022B5
:106AF0001A70194B00225A70174B00229A701148D5
:106B00000BF0A5FE11480CF046F9144B00221A7048
:106B1000134B00221A70134B00221A700B480CF012
:106B20001DFA0B48FDF70AFA00BF80BD782C002043
:106B3000F40100202C200020C01D0020DC1D0020BE
:106B4000601E00206C1E0020941E0020A81E002045
:106B5000141F0020792C0020F40500207A2C00203E
:106B60007B2C00207C2C002080B584B000AF034635
:106B7000FB715448FCF776F85348FCF74DFB53483B
:106B8000FEF732F85248FCF71DFE524B00221A70F5
:106B9000514B93F8D130022B02D14F48FDF778FAD0
:106BA0004E4B1B78DBB20D2B0BD1474B93F8783152
:106BB000812B04D0444B93F87831012B01D1012370
:106BC00000E00023002B02D03F48FCF7D1F9434BF3
:106BD0001B78DBB20E2B0BD13F4B93F8D130012B3E
:106BE00004D03D4B93F8D130002B01D1012300E0BC
:106BF0000023002B07D03A480BF0FBFA394B0B224D
:106C00001A70FEF741FE344B93F8C630002B1CD0AF
:106C1000354BDB68FB60314BD3F89C33324AD36091
:106C20002E4AFB68C2F89C33304B186801230022BF
:106C30002D4904F0FBF90346002B14BF0123002368
:106C4000DBB2002B01D0FEF7FBF84222284929488D
:106C50000EF08BF9254B1868FB795B0001331A465F
:106C600002231E4904F0E2F90346002B14BF01235E
:106C70000023DBB2002B01D0FEF7E2F84FF4806274
:106C800016491D480EF071F9144B93F89833DBB296
:106C9000002B14BF01230023DAB20F4B83F8C52069
:106CA0000D4B002283F8C6200A4B01221A70134BA9
:106CB00001221A70124B00221A7000BF1037BD4615
:106CC00080BD00BFA81E00202C200020182000201E
:106CD000141F00207F2C0020441F0020F4010020FE
:106CE000C01D0020792C0020502800200001002029
:106CF0007C1B0020D6040020F41600208C2C0020E1
:106D0000822C002080B5ADF5836D00AF0246FB1DDF
:106D10001A70A94B00221A70A84B01221A70A84BB6
:106D20001868FB1D1B785B0001331A4607F10C0144
:106D3000022304F0C3F80346002B14BF01230023F1
:106D4000DBB2002B01D0FEF77BF807F10C0393F8C0
:106D5000E032012B08D19B4B1B69C3F34333DBB2F9
:106D6000022B01D0012300E00023002B00F0F5806E
:106D7000FFF758FE07F10C031B78C7F8143407F12E
:106D80000C031B79C3F30013DBB2C7F8103407F10F
:106D90000C0213796FF30413137107F10C034FF412
:106DA0008062194688480EF0E0F88848FCF73AF807
:106DB0008748FCF701FB8748FDF746FF8648FCF74C
:106DC00067FDD7F814340B2B07D0D7F81434DAB298
:106DD000824B1A70FEF758FD09E0804B09221A70A9
:106DE000FEF752FD7D4B0B221A70FEF74DFDD7F8D2
:106DF00014340E2B09D1794B0B221A70FEF744FD87
:106E0000764B0E221A70FEF73FFDD7F814340D2B87
:106E100009D1724B0B221A70FEF736FD6F4B0D2213
:106E20001A70FEF731FDD7F81034002B08D0664BEE
:106E30005B68C3F30013DBB2002B01D1012300E038
:106E40000023002B04D0654B01221A70FEF71CFDB5
:106E5000D7F81434092B43D107F10C031B79C3F382
:106E60004213DBB2A7F80E34B7F80E34042B05D06A
:106E70005A4B08221A70FEF707FD04E0574B072211
:106E80001A70FEF701FDB7F80E34052B26D801A2C3
:106E900052F823F0AD6E0000B56E0000BD6E00002C
:106EA000C56E0000CD6E0000D56E00004B4B002279
:106EB0001A7013E0494B05221A700FE0474B062267
:106EC0001A700BE0454B07221A7007E0434B08226B
:106ED0001A7003E0414B09221A7000BFFEF7D4FC80
:106EE000D7F814340C2B13D13C4B09221A70FEF73F
:106EF000CBFC3A4B01221A70FEF7C6FC374B01223D
:106F00001A70FEF7C1FC354B0C221A70FEF7BCFC60
:106F1000D7F814340A2B03D0D7F81434092B0DD129
:106F2000D7F81034002B09D02C4B01221A70FEF731
:106F3000ABFC2A4B01221A70FEF7A6FCFEF764FB9D
:106F40004FF48062204926480EF00FF8254B0122AD
:106F50001A701A4B00221A7011E0FFF763FD224BE2
:106F600001221A70FEF750FBFB1D1B781846FFF735
:106F7000FBFD1C4B01221A70104B00221A70124BA1
:106F800093F89833DBB2002B14BF01230023DAB24D
:106F9000164B83F8C520154B002283F8C620144AEF
:106FA000FB1D1B781370044B01221A7000BF07F5FC
:106FB0008367BD4680BD00BF7F2C0020822C00204F
:106FC0000001002000F00F40F4010020A81E002066
:106FD0002C20002018200020141F0020792C0020D5
:106FE000F41600208C2C0020832C0020441F00204D
:106FF000842C002080B483B000AF0346FB71044AA8
:10700000FB79D37000BF0C37BD465DF8047B704739
:107010000070064080B483B000AF0346FB71074B9D
:107020009B79DAB20549FB791343DBB28B7100BF60
:107030000C37BD465DF8047B704700BF007006400A
:1070400080B400AF064B9B79DBB2054A43F02003C6
:10705000DBB2937100BFBD465DF8047B704700BF93
:107060000070064080B400AF064B9B79DBB2054A46
:1070700023F02003DBB2937100BFBD465DF8047BB3
:10708000704700BF0070064080B500AF0A4B1B7808
:10709000022B0BD1094B01221A70074B01221A70E7
:1070A0000022002106480DF034FA02E0054B0022D0
:1070B0001A7000BF80BD00BF882C0020872C0020E4
:1070C00000700640822C002080B500AF03480DF010
:1070D00051FA034B00221A7000BF80BD00700640B9
:1070E000872C002080B584B000AF504B1A78504BED
:1070F0001B789A4200F096804D4B1B785A1CD1B2F7
:107100004B4A117019464B4A0B469B000B445B00DF
:107110001A443B1D1068516803C312891A807B7999
:10712000042B7FD13B7A013B162B76D801A252F873
:1071300023F000BF91710000B17100001B720000CC
:107140001B7200001B7200001B7200001B7200000B
:107150001B7200001B7200001B7200001B720000FB
:107160001B7200001B7200001B7200001B720000EB
:107170001B7200001B7200001B7200001B720000DB
:10718000077200001B720000D17100000F72000036
:10719000294B1B78002B42D0284B1B78002B3ED06C
:1071A0007B7A1E2B3BD87B7A1846FFF7ABFD36E087
:1071B000214B1B78002B34D0204B1B78002B30D078
:1071C0007B7A1E2B2DD87B7A1846FFF7CDFC28E062
:1071D000194B01221A701A4B1B78002B0DD042223A
:1071E000184919480DF0C1FE4FF48062174918483C
:1071F0000DF0BBFE124B00221A70104B01221A70C8
:10720000FEF702FA0EE00D4B01221A700AE00A4B5B
:1072100000221A70FEF7F8F904E000BF02E000BF98
:1072200000E000BF00BF1037BD4680BD8A2C0020A3
:107230008B2C0020F40C0020832C0020802C0020BC
:10724000822C00207C1B0020D6040020F4010020AA
:10725000F416002080B582B000AFAC4B4FF4004272
:107260001A82AB4AD2F8803043F4F073C2F880300F
:10727000A74AB2F840306FF38A23A2F84030A44AFC
:10728000B2F8403043F40063A2F84030FFF7CAFB85
:10729000A04B00221A70A04B01221A709F4B0022B3
:1072A0001A709F4B1868012300229E4903F006FEC6
:1072B0000346002B14BF01230023DBB2002B01D0B7
:1072C000FDF7BEFD974B1B68974A934206D1954B3D
:1072D0009B68B3F5087F01D0FDF7ECFD8C4B1B6973
:1072E000C3F34333DBB2012B09D1894BD3F81031FF
:1072F000C3F38063DBB2002B01D0012300E0002345
:10730000002B17D0824B1B69C3F34333DBB2012B35
:1073100007D07F4BD3F81031C3F38063DBB2002B6F
:1073200001D0012300E00023002B03D07D4B00227D
:107330001A60E7E77B4B1B687B4A934200F0898029
:10734000784B794A1A60774B4FF408729A60754B04
:1073500000225A60734B754ADA607548FBF782FC6D
:107360007448FBF759FF7448FDF73EFC7348FCF77F
:1073700029FA00237B607B681E2B20DC7B68704A27
:1073800002FB03F33F331A466E4BC3F89C23644B56
:1073900018687B685B0001331A460223694903F0D1
:1073A00045FE0346002B14BF01230023DBB2002B54
:1073B00001D0FDF745FD7B6801337B60DBE7624B65
:1073C000022283F8802000233B603B680F2B1EDCE9
:1073D0005D4B93F880301A465C4B53F8223099B2DB
:1073E000594A3B6822F81310574A3B6810334FF64E
:1073F000FF7122F81310544A3B6810339B0013446A
:107400004FF07E521A603B6801333B60DDE7444B2E
:1074100018680123454A4C4903F008FE0346002B37
:1074200014BF01230023DBB2002B01D0FDF708FDC0
:107430003B4B1868012300223A4903F0F7FD03464D
:10744000002B14BF01230023DBB2002B01D0FDF77A
:10745000F7FC334B18680123344A3B4903F02EFDF7
:107460000346002B14BF01230023DBB2002B01D005
:10747000FDF7E6FC344B93F88030042B03D9324BF4
:10748000022283F88020224B1B69C3F34333DBB213
:107490000F2B09D11E4BD3F81031C3F38063DBB23D
:1074A000002B01D0012300E00023002B17D0184B44
:1074B0001B69C3F34333DBB20F2B07D0144BD3F854
:1074C0001031C3F38063DBB2002B01D0012300E055
:1074D0000023002B03D01E4B01221A70E7E71C4B40
:1074E0001B78002B3AD01B480CF002F9FDF778FD11
:1074F0001E20FFF707FCFEF787F80448F9F724FB86
:10750000002115480CF019F937E000BFC01D00201C
:1075100000F00F40832C00208C2C0020822C0020B7
:1075200000010020502800204B45454EBFC3C90133
:10753000A81E00202C20002018200020141F00204E
:107540001C4E0E00F4010020C01B00208C550100D1
:107550008E2C002000600340007003401E20FFF7C7
:10756000D1FBFEF751F80848F9F7EEFA0021074879
:107570000CF0E3F806480CF0BBF8064B01221A7039
:1075800000BF0837BD4680BDC01D0020007003400D
:10759000006003407F2C002080B500AF574B0022D5
:1075A0009A72574B1B69C3F34333DBB2002B0CBFFA
:1075B00001230023DBB2002B2AD0524B1B78002B77
:1075C00020D0514B1B78002B0CBF01230023DBB2D2
:1075D0001A464D4B1A704C4B1B78002B15D04B4B59
:1075E0001B78002B11D0422249494A480DF0BDFCBE
:1075F0004FF48062484949480DF0B7FC434B0022E4
:107600001A7002E01E20FFF7AFFAFDF7FDFF73E0EE
:10761000414B1B78DBB2093B052B64D801A252F821
:1076200023F000BF3D76000049760000557600004B
:10763000917600009D760000B776000038480BF088
:107640007FFCFDF7E1FF4EE035480BF079FCFDF7DC
:10765000DBFF48E02A4B1B69C3F34333DBB20B2B40
:107660000CBF01230023DBB2002B39D02D480BF0D7
:10767000A9FE2C48FCF78CF8274B5B68C3F300137A
:10768000DBB2194627480BF0F9FEFDF7BDFF27E0F6
:1076900023480BF055FCFDF7B7FF24E022480BF020
:1076A00091FC21480BF00AFD1F48FBF7A9FC1E487E
:1076B000FBF75EFC17E0124B1B69C3F34333DBB2ED
:1076C0000E2B0CBF01230023DBB2002B0AD017487E
:1076D000FCF788FC1548FCF759FDFDF795FF01E024
:1076E00000BF00E000BF124B9B7B002B04D0104872
:1076F0000BF0D3FFFDF788FF00BF80BDC01D002049
:1077000000F00F40802C0020832C0020822C0020D1
:107710007C1B0020D6040020F4010020F416002079
:10772000A81E0020141F00202C200020441F002031
:107730001820002090B583B000AF9A4B022283F846
:1077400080200DF0FAFB0DF0CCFA0DF09CFB964B6F
:1077500000221A70944B00229A70934B9B78DBB2F4
:10776000914A63F03F03DBB29370FFF77BFC8F4BD2
:1077700002221A7000218E480CF017F88D4B186801
:1077800000230522002101F0A3FE0CF05DFA0CF0AD
:107790005BFA0CF059FA874B1B68184603F006FE9B
:1077A0000346002B14BF01230023DBB2002B01D0C2
:1077B000FDF746FB7F4B1B68184603F047FD034669
:1077C000002B14BF01230023DBB2002B01D0FDF7F7
:1077D00037FB784B1B68184603F0E8FD0346002B87
:1077E00014BF01230023DBB2002B01D0FDF728FBDF
:1077F0000DF043FB6F4B1B68D3F888326E4A9342FF
:107800000ED96C4B1B68D3F88C32B3F5007F07D1CF
:10781000684B1B68184603F025FB0346002B01D07C
:10782000012300E00023002B01D0FDF709FBFFF747
:1078300011FD624B1B78002B5AD0614B1B78002B3B
:107840001DD140F2E1225F495F480DF080FB034605
:10785000002B14BF01230023DBB2002B0FD0584BA9
:1078600001221A70594B1B78002B06D0584B1B78FD
:10787000002B02D0FFF708FC01E0FDF7C5FE002356
:10788000FB71FB790F2B30D84D4B1B78002B28D187
:10789000FB79504A32F813301946FB794A4A03F50E
:1078A000B8735B0013445B889BB2CB1A18460DF08B
:1078B0004AFB0346282BCCBF01230023DBB2002B5D
:1078C0000FD03F4B01221A70404B1B78002B06D083
:1078D0003F4B1B78002B02D0FFF7D6FB01E0FDF7F2
:1078E00093FEFB790133FB71CBE7344B00221A7016
:1078F000FFF7F8FB384B9B7ADBB2012B0CBF01235F
:107900000023DBB2002B01D0FFF746FE334B1B698F
:10791000C3F34333DBB2052B14D12B4B1B78DBB203
:107920000E2B0FD02E4B9B7B83F00103DBB2002B81
:1079300008D0254B5B68C3F38103DBB2032B01D076
:10794000012300E00023002B50D01F4B1B78DBB23B
:107950000B2B14BF01230023DBB2002B0CD0214BD7
:107960001B7883F00103DBB2002B05D01C48FDF728
:10797000ABF81C4B01221A70134B1B899BB2DB43E3
:107980009BB20022194614480AF06BFC0E4B1B896F
:107990009BB20122194610480AF063FC124B0122E7
:1079A0001A703DE0C01B002000700640882C0020AB
:1079B00000D0004000010020BEC3C901812C00207E
:1079C000822C0020F4160020F4010020802C0020DE
:1079D000832C0020381B0020C01D002000F00F4029
:1079E000182000207E2C00207D2C00209C4B1B7832
:1079F000002B15D09B4B1B899BB21846FAF71AF83F
:107A000099480AF0F6FB994B1B78002B05D0984853
:107A1000FDF77EF8954B00221A70914B00221A70E8
:107A200094480AF043FA0346002B3FF402AF914812
:107A30000AF01DFA0346904A13608D4B9B7B002B86
:107A400011D08D4B1B7803F01003DBB2002B3FF4F9
:107A5000F0AE894B1B78C3F30303DBB219468448AD
:107A6000FDF7A2F8E5E6854B1B69C3F34333DBB2B0
:107A7000052B0DD17B4B1B78DBB20E2B08D07C4B3A
:107A80009B7B83F00103DBB2002B01D0012300E0DC
:107A90000023002B19D0734B1B899BB21AB2764B73
:107AA0001B78C3F30013DBB21946734B1B78C3F387
:107AB0000303DBB201FA03F31BB253401BB29AB2C9
:107AC000684B1A81664B01221A706B4B1B7803F0CE
:107AD0001003DBB2002B0CD069480AF090FC03467F
:107AE000002B06D0674B93F8D130012B01D1012335
:107AF00000E00023002B02D06248FCF76FFB594BDB
:107B00001B78DBB20B2B04D0564B1B78DBB20E2B51
:107B100001D1012300E00023002B4ED0514B1B78F4
:107B2000DBB20E2B13D1574B93F8D130052B0ED16E
:107B300053480AF064FC0346002B08D14F4B1B69E5
:107B4000C3F34333DBB2002B01D1012300E0002358
:107B5000002B04D04B480BF0D1FCFDF755FD414BF9
:107B60001B78DBB20E2B18D1464B93F8D130032B88
:107B700004D0444B93F8D130042B0ED140480AF086
:107B80003EFC0346002B08D03C4B1B69C3F3433338
:107B9000DBB2002B01D1012300E00023002B07D032
:107BA0003848FCF761FA3848FBF7F2FDFDF72CFD89
:107BB000314B19683448FCF73DF82A4B1B78DBB28F
:107BC0000D2B0CBF01230023DBB2002B00F0AA8198
:107BD0002E4B93F87831812B2ED12C4B93F87931A1
:107BE000002B02D0012B06D09CE1234B19682648BC
:107BF000FCF720F896E1204B1B7803F01003DBB272
:107C0000002B0CD01C4B1B78C3F30303DBB21946CB
:107C10001F48FAF721F91D48FBF7A0FA82E1164B3D
:107C20001B78C3F30303DBB2194619480AF006FFB9
:107C30001648FBF793FA75E1144B93F87831832BD0
:107C400028D10D4B1B78C3F30303DBB219460F4851
:107C50000BF07DFB0346002B1CD001231BE000BF73
:107C60007D2C0020F4010020C01D00207E2C00206F
:107C700018200020DC1D0020F805002000F00F4037
:107C8000601E0020441F0020141F00202C20002014
:107C9000A81E00200023002B00F04481AE4B1B786F
:107CA00003F01003DBB2002B00F08F80AB4B93F896
:107CB0008E31002B23D1A84B1B78C3F30303DBB217
:107CC0007B71A54B1B78C3F30303DBB21946A448B1
:107CD0000AF031F9A2480AF0ACF90346012B8CBF37
:107CE00001230023DBB2002B06D001219C480AF0BF
:107CF000BCF90346BB7195E0FF23BB7192E0002104
:107D000098480AF0B2F903461A46934B1B78C3F31E
:107D10000303DBB29A420CBF01230023DBB2002B2A
:107D200004D0FF237B71FF23BB717BE08A4B1B7860
:107D3000C3F30303DBB27B71874B1B78C3F30303ED
:107D4000DBB2194687480AF0F6F8002185480AF0A8
:107D50008CF903461A46012303FA02F1824BDB8AAF
:107D60009BB21AB20BB213431BB29AB27E4BDA82A9
:107D70007C480AF05EF90346012B8CBF01230023E7
:107D8000DBB2002B1ED0012176480AF06EF90346C3
:107D9000BB71012173480AF068F903461A460123B2
:107DA0009340D943704BDB8A9BB21AB20BB213409B
:107DB0001BB29AB26C4BDA82BB79194669480AF059
:107DC000EFF82FE0FF23BB712CE0644B93F88E316A
:107DD000002B23D1604B1B78C3F30303DBB2BB71D1
:107DE0005D4B1B78C3F30303DBB219465C480AF012
:107DF000D7F85B480AF01DF90346002B14BF012396
:107E00000023DBB2002B06D0002155480AF02DF9E3
:107E100003467B7106E0FF237B7103E0FF237B7148
:107E2000FF23BB71BB79FF2B24D04C4BFF2283F87F
:107E30007A214E48FAF79EFE4C480AF0BDFD4C48A8
:107E4000FBF7A6FC484B1B8A9BB223F480739AB2C3
:107E5000454B1A82444B1B8A9BB223F480639AB22F
:107E6000414B1A82404B1B8A9BB223F00E039AB2FD
:107E70003D4B1A827B79FF2B54D07B7919463748CA
:107E80000BF01CFA0346002B02D0012B1BD049E05B
:107E9000324B002283F87A217B7919462F480BF068
:107EA000FCF9034619467B7901223148FBF7F2FFC2
:107EB000FDF7AAFB2C4B1B8A9BB243F480639AB25A
:107EC000294B1A822EE0254B012283F87A2127487C
:107ED000FAF788FD7B79194620480BF01AFA034619
:107EE000C3F30103DBB21C467B7919461B480BF038
:107EF00010FA0346C3F38103DBB21A4621461D483C
:107F0000F9F796F97B7919461448FBF76BF9FDF7F9
:107F10007BFB154B1B8A9BB243F480739AB2124BC6
:107F20001A8200BF144B1B78DBB20C2B0CBF012351
:107F30000023DBB2002B3BD00F4B5B68C3F3001375
:107F4000DBB283F00103DBB2002B17D0024B1968C0
:107F50000748FBF76FFE2BE0F80500202C200020DF
:107F6000A7210020BB210020C01D0020A81E00204A
:107F7000141F00206C1E0020F4010020244B1B78ED
:107F800003F01003DBB2002B09D0214B1B78C3F3A5
:107F90000303DBB219461F48F9F75EFF08E01C4BEC
:107FA0001B78C3F30303DBB219461A480AF046FDF7
:107FB000194B1B78DBB20A2B04D0174B1B78DBB2B2
:107FC000092B01D1012300E00023002B3FF431AC49
:107FD0000F4B1B7803F01003DBB2002B09D00C4BC6
:107FE0001B78C3F30303DBB219460A48F9F734FFE1
:107FF00008E0074B1B78C3F30303DBB219460548BF
:108000000AF01CFD044B1B78DBB20A2B11E400BF05
:10801000F8050020A81E0020F401002080B500AF64
:108020001C4B1B69C3F34333DBB2002B14BF01238A
:108030000023DBB2002B27D0164B1B69C3F343335D
:10804000DBB21A46144B1A70124B1B69C3F343334D
:10805000DBB20C2B0CBF01230023DBB2002B13D0AF
:108060000E4A137943F0100313710C4B1B78DBB2EB
:108070000C2B0CBF01230023DBB2002B02D00848DD
:10808000FAF7B0FCFDF7C0FA012106480BF055FBEA
:1080900000BF80BD00F00F40782C0020F4010020CC
:1080A000A81E00200070034080B582B000AF2748B2
:1080B00005F05AFA78607B6803F40033002B27D070
:1080C000224B1B69C3F34043DBB283F00103DBB2F5
:1080D000002B0BD01E4B1B78DBB283F00103DBB20D
:1080E000002B15D01B48FCF715F911E01A4B1B7833
:1080F000DBB283F00103DBB2002B09D01548FCF79B
:1081000005FC134B01221A70022114480BF015FBD9
:108110007B6803F4F033002B0CD0114B1B7883F0F9
:108120000103DBB2002B05D00E4B1B78002B01D0D6
:10813000FFF774FF7968054805F02EFABFF34F8FFB
:1081400000BF00BF0837BD4680BD00BF00F00F4034
:108150007A2C0020182000207B2C00200070034087
:108160008E2C00207F2C002080B500AF0122012141
:1081700016480BF0CDFA012114480BF0FAFA144B13
:108180001B69C3F34333DBB2002B14BF012300236D
:10819000DBB2002B15D00E4B1B69C3F34333DBB2AC
:1081A0001A460C4B1B78DBB29A420CBF012300230A
:1081B000DBB2002B07D0074B1B78DAB2064B1A70E4
:1081C00001E0FDF761FB00BF80BD00BF0070034010
:1081D00000F00F40782C0020792C002080B500AFF3
:1081E0000122022105480BF093FA022103480BF00B
:1081F000C0FA034B00221A7000BF80BD007003401C
:108200007A2C002080B582B000AF012200215E48A8
:108210000BF07EFA5D4B1B7883F00103DBB2002B81
:1082200000F0AD805A480AF0EAF80346BB80594B8B
:108230001B78DBB20E2B0BD1574B93F8D130022BAE
:1082400006D0554B93F8D130012B01D0012300E02B
:108250000023002B00F08D80BB88002B02D14F4BF8
:1082600000221A704E4B1B69C3F34333DBB20E2B53
:1082700009D14A4B1B78DBB283F00103DBB2002B40
:1082800001D0012300E00023002B5AD0454B0122EE
:108290009A76454B01221A703F4B93F9C430022B5A
:1082A0001ED0022B29DC002B0ED0012B25D1002261
:1082B0004FF6FF713B4809F0D4FF012248F201015B
:1082C000384809F0CEFF18E000224FF6FF7135481C
:1082D00009F0C7FF01220121324809F0C2FF0CE07A
:1082E00000224FF6FF712F4809F0BBFF01224FF427
:1082F00000412C4809F0B5FF00BF0023FB71FB795A
:108300000F2B39D8BA88FB7942FA03F303F0010343
:10831000002B12D0FB7919461F48FBF7B5FFFB79FC
:10832000002B0AD0FB790E2B07D8FB790133DBB287
:108330001A460E211B480AF020F8FB790133FB7125
:10834000DDE7174B1B69C3F343330123002B13D025
:10835000154B1B78002B08D0002248F20101114870
:1083600009F07FFF104B00221A700948F8F79EFCB5
:1083700002E00748F8F79AFC0A48F8F729F900BF25
:108380000837BD4680BD00BF007003408E2C002022
:10839000601E0020F4010020441F00207C2C0020DF
:1083A00000F00F40C01D0020852C002084B090B448
:1083B00000AF07F1080484E80F00474B1B7883F0F7
:1083C0000103DBB2002B64D0444B1B78C3F30303DF
:1083D000DBB207F1080232F813301A11404B1A6170
:1083E0003E4B1B78C3F30303DBB2103307F10802E3
:1083F00032F813301A113B4B1A63384B1B78C3F316
:108400000313DBB207F1080232F813301A11364BAE
:108410001A61324B1B78C3F30313DBB2103307F13D
:10842000080232F813301A112D4B1A622B4B5B786D
:10843000C3F30303DBB207F1080232F813301A1159
:10844000274B9A61254B5B78C3F30303DBB21033F0
:1084500007F1080232F813301A11214B9A621F4BB0
:108460005B78C3F30313DBB207F1080232F8133071
:108470001A111C4B9A64194B5B78C3F30313DBB2DC
:10848000103307F1080232F813301A11154B1A6233
:108490001DE0164B1B781A46154B33F812301B1192
:1084A000104A93640E4A93610F4A13610C4A136198
:1084B0000E4B1B780F4A103332F813301B11094A48
:1084C0001362074A9362064A1362064A136300BFA7
:1084D000BD4690BC04B070478E2C0020E401002003
:1084E00000900B4000800340009003408D2C002042
:1084F000A00100207C1B002080B500AF764B1B78CC
:10850000DBB20D2B75D00D2B00F3BA800A2B02DCE9
:10851000092B03DAB4E00C2B3DD0B1E06F4BDB7AD2
:10852000002B05D0012200216D480BF0C4F804E0B7
:10853000002200216A480BF0BEF8684B1B7B002B21
:1085400005D00122032166480BF0B5F804E00022B3
:10855000032163480BF0AFF8604B5B7B002B05D029
:10856000012205215F480BF0A6F804E00022052156
:108570005C480BF0A0F8594B9B7B002B05D00122E7
:10858000012159480BF097F8A3E000220121564839
:108590000BF091F89DE0514B9B78C3F30003DBB2E5
:1085A0001A4600214E480BF086F84C4B9B78C3F3DB
:1085B0004003DBB21A46032149480BF07CF8474BD5
:1085C0009B78C3F38003DBB21A46052145480BF0C4
:1085D00072F8424B9B7B002B05D0012201214248BF
:1085E0000BF069F875E0002201213F480BF063F8B9
:1085F0006FE03E4B93F87831832B41D13B4B93F89E
:108600007A31002B3CD0354BDB7A002B05D0012290
:10861000002133480BF04FF804E0002200213048DD
:108620000BF049F82D4B1B7B002B05D001220321B9
:108630002B480BF040F804E00022032128480BF0FF
:108640003AF8264B5B7B002B05D0012205212548FB
:108650000BF031F804E00022052122480BF02BF842
:108660001E4B9B7B002B05D0012201211E480BF0E5
:1086700022F82EE0002201211B480BF01CF828E014
:10868000164B9B78C3F30003DBB21A460021144853
:108690000BF011F8114B9B78C3F34003DBB21A4681
:1086A00003210F480BF007F80C4B9B78C3F38003B2
:1086B000DBB21A4605210B480AF0FDFF074B9B78F9
:1086C000C3F3C003DBB21A46012107480AF0F3FFE7
:1086D00000BF00BF80BD00BFF4010020E401002006
:1086E00040F00F40C0F00F4080F00F402C200020E1
:1086F00080B500AF8A4B93F903301A46884B1B783C
:10870000C3F30303DBB29A420BD1854B93F90730D5
:10871000002B16D1824B9B7803F00103DBB2002BB8
:108720000FD0012201217F480AF0C5FF7C4B1B7846
:10873000C3F30303DBB25AB2794BDA70784B0122F0
:10874000DA72774BDB7A012B07D9002201217548B9
:108750000AF0B1FF724B0022DA72714BDB7A002B08
:1087600005D06F4BDB7A0133DAB26D4BDA726C4BAA
:108770009B78C3F30003DBB25AB2694BDA71684BE2
:1087800093F904301A46664B1B78C3F30313DBB22C
:108790009A420BD1624B93F90830002B16D1604BF3
:1087A0009B7803F00203DBB2002B0FD001220221E1
:1087B0005C480AF080FF5A4B1B78C3F30313DBB20B
:1087C0005AB2574B1A71564B01221A73544B1B7BEA
:1087D000012B07D90022022152480AF06CFF504BAE
:1087E00000221A734E4B1B7B002B05D04C4B1B7B7E
:1087F0000133DAB24A4B1A73494B9B78C3F34003F7
:10880000DBB25AB2464B1A72454B93F905301A4601
:10881000434B5B78C3F30303DBB29A420BD1404B6B
:1088200093F90930002B16D13D4B9B7803F00403DC
:10883000DBB2002B0FD0012206213B480AF03BFFA0
:10884000374B5B78C3F30303DBB25AB2344B5A7134
:10885000334B01225A73324B5B7B012B07D9002229
:10886000062131480AF027FF2D4B00225A732C4B6A
:108870005B7B002B05D02A4B5B7B0133DAB2284BA4
:108880005A73274B9B78C3F38003DBB25AB2244B55
:108890005A72234B93F906301A46214B5B78C3F387
:1088A0000313DBB29A420BD11D4B93F90A30002B14
:1088B00016D11B4B9B7803F00803DBB2002B0FD0C3
:1088C0000122022119480AF0F6FE154B5B78C3F32A
:1088D0000313DBB25AB2124B9A71114B01229A73F5
:1088E0000F4B9B7B012B07D9002202210F480AF076
:1088F000E2FE0B4B00229A73094B9B7B002B05D0A9
:10890000074B9B7B0133DAB2054B9A73044B9B7880
:10891000C3F3C003DBB25AB2014B9A7200BF80BDF1
:10892000E401002040F00F40C0F00F4080F00F4005
:10893000F0B595B00EAF0023FB750023FB75FB7DF2
:108940000F2B15D8FA7DFB7DA74931F81210A74AE5
:1089500022F81310FA7DFB7DA349103231F8121072
:10896000A24A103322F81310FB7D0133FB75E6E7B2
:108970009F4BB3F840209D4BA3F840209D4B1B78A4
:10898000DBB20E2B10D19C4B93F8D130032B09D0C6
:10899000994B93F8D130042B04D0974B93F8D130F6
:1089A000052B01D1012300E00023002B00F0C3813F
:1089B000914B93F8C630002B02D0904B1B6802E01D
:1089C0008C4BD3F89C33FB608B4B93F8D130032B4B
:1089D00060D189480AF0AAFDB0EE407A864BD3ED0B
:1089E000337A77EE277A844BC3ED337A824BD3ED1B
:1089F000337AB1EE0C7AF4EEC77AF1EE10FA0DDBB1
:108A00007D4BD3ED337AB1EE0C7A77EEC77A7A4BA1
:108A1000C3ED337A784B012283F8D020764BD3ED27
:108A2000337AFCEEE77AC7ED017A3B79DAB2724B22
:108A300083F8C820704B93F8D030002B2AD0704BAD
:108A400018686C4BD3F8A4335A1C6A49C1F8A423A4
:108A5000FA681A4401236B4902F030FA0346002BEE
:108A600014BF01230023DBB2002B01D0FCF7E8F98F
:108A7000604BD3F8A0235F4BD3F8A433B3FBF2F1E0
:108A800002FB01F29B1A5B4AC2F8A4335A4B002244
:108A900083F8D020584B93F8D130042B77D1564827
:108AA0000AF044FDB0EE407A534BD3ED337A77EEC3
:108AB000C77A514BC3ED337A4F4BD3ED337AF5EE92
:108AC000C07AF1EE10FA0DD54B4BD3ED337AB1EEFF
:108AD0000C7A77EE877A484BC3ED337A464B012206
:108AE00083F8D020444BD3ED337AFCEEE77AC7ED20
:108AF000017A3B79DAB2404B83F8C8203E4B93F8B9
:108B0000D030002B43D03B4BD3F8A433002B14BF01
:108B100001230023DBB2002B19D0394B1868354BE9
:108B2000D3F8A4335A1E3349C1F8A423FA681A446F
:108B30000123344902F0C2F90346002B14BF01237C
:108B40000023DBB2002B1ED0FCF77AF91BE02C4B84
:108B50001868284BD3F8A423FB681A440123294939
:108B600002F0ACF90346002B14BF01230023DBB253
:108B7000002B01D0FCF764F91E4BD3F8A033013B66
:108B80001C4AC2F8A4331C4B002283F8D0201A4B95
:108B900093F8C83019461C481A4A0B465B010B442F
:108BA0005B001344194642231A460CF0DEF9114BC0
:108BB00093F89933DBB2002B14BF01230023DBB2FF
:108BC000002B23D00023FB75FB7D0F2B1ED8FA7DD5
:108BD000FB7D074931F812100B4A22F81310FB7D78
:108BE0000133FB75F0E700BF381B00207C1B002021
:108BF000A0010020F4010020441F00205C28002078
:108C00000001002040080020FC050020AA4E6D460F
:108C100006F110040FCC0FC50FCC0FC50FCC0FC53C
:108C200023682B8096E80F00FFF7C0FBA34809F0EC
:108C3000E6FB0346BB820023FB75FB7D0F2B34D87C
:108C4000FB7D9F4A103332F813301A469D4B93F840
:108C5000803019469C4B53F821309A4208D9FB7D4D
:108C6000012202FA03F39AB2BB8A1343BB8218E0D3
:108C7000FB7D934A103332F813301A46914B93F828
:108C800080301946914B53F821309A4209D2FB7D2E
:108C9000012202FA03F39BB2DB439AB2BB8A134070
:108CA000BB82FB7D0133FB75C7E7BB8A194683484E
:108CB00009F096FB864B93F8D130052B2FD1BB8A58
:108CC000002B25D00023FB75FB7D0F2B0BD8FA7DE5
:108CD000FB7D7B4931F812107E4A22F81310FB7D90
:108CE0000133FB75F0E77B4E6D4606F110040FCCA7
:108CF0000FC50FCC0FC50FCC0FC523682B8096E88E
:108D00000F00FFF753FB6E4ABB8AA2F84030CEE05B
:108D1000694BB3F840206A4BA3F84020C7E0BB8AF8
:108D2000002B03D1644BB3F8403000E0BB8A644AA7
:108D3000A2F84030BBE00023FB75FB7D0F2B3ED833
:108D4000FB7D5F4A103332F813301A465D4B93F8BF
:108D5000803019465C4B53F821309A420DD9584B5C
:108D6000B3F84020FB7D012101FA03F39BB21343CA
:108D70009AB2534BA3F840201DE0FB7D504A1033BC
:108D800032F813301A464F4B93F8803019464F4B48
:108D900053F821309A420ED2494BB3F84020FB7D64
:108DA000012101FA03F39BB2DB439BB213409AB259
:108DB000434BA3F84020FB7D0133FB75BDE7404BDF
:108DC000B3F8403019463D4809F00AFB424B1B7886
:108DD000DBB20E2B06D13E4B93F8D130022B01D1E2
:108DE000012300E00023002B51D0394B93F8C5300C
:108DF000002B02D0394B1B6802E0374BD3F89C3371
:108E00003B61334B93F8C7305A1CD1B2304A82F8D9
:108E1000C7101946324A0B465B010B445B001344F2
:108E20002C4A1846114642231A460CF09EF8284B4D
:108E300093F8C7202B4BA3FB0213D11A49080B440C
:108E400099080B46DB005B1AD31ADAB2204B83F881
:108E5000C7201F4B93F8C730002B18D1224B18683E
:108E60001D4BD3F8A0335A1C1B49C1F8A0233A6903
:108E70001A4401231A4902F0D9F80346002B14BF03
:108E800001230023DBB2002B01D0FBF7D9FF114EE9
:108E90006D4606F110040FCC0FC50FCC0FC50FCCDB
:108EA0000FC523682B8096E80F00FFF77FFA00BFFD
:108EB0001C37BD46F0BD00BFFC050020601E002031
:108EC000A0010020C01B00208C550100A05501000E
:108ED000441F00207C1B0020F40100205C2800209F
:108EE00040060020254992240001002090B583B05F
:108EF00000AF0221B44803F0ADFC38603A680221AB
:108F0000B14803F0E9FCB14B1B78002B00F0B980AD
:108F10000023FB71FB790F2B00F2B080FB792C2230
:108F200002FB03F3AA4A1A44FB79AA4931F8133029
:108F300007EE903AF8EE677A0A21DFEDA72AB0EE45
:108F4000672ADFEDA61A9FEDA61ADFEDA60A9FEDB0
:108F5000A60A10460AF07FFCFB792C2202FB03F3E1
:108F6000A24A1A44FB799B49103331F8133007EEBB
:108F7000903AF8EE677A0A21DFED972AB0EE672A79
:108F8000DFED9B1A9FED9B1ADFED960A9FED960A87
:108F900010460AF060FCFB792C2202FB03F38C4A9A
:108FA0001A44FB798B4931F8133007EE903AF8EE0A
:108FB000677AB0EE670A10460AF0E8FCF0EE407AF5
:108FC000FB79FCEEE77A17EE902A91B28A4A22F8F2
:108FD0001310FB792C2202FB03F3844A9C18FB79C3
:108FE0007C4A103332F813301A46FB791946104682
:108FF000FBF79AFF034607EE903AF8EE677AB0EE79
:10900000670A20460AF0C2FCF0EE407AFB79FCEEDB
:10901000E77A17EE902A91B2774A103322F81310AC
:10902000FB791B01754A1A44FB79734931F81330F7
:1090300007EE903AF8EE677AB0EE671ADFED690A4C
:109040009FED690A10460AF0D3FDFB791B016B4ABC
:109050001A44FB796A4903F5B8735B000B445B88DB
:109060009BB207EE903AF8EE677AB0EE670A1046C8
:109070000AF0DBFDFB790133FB714BE7534B002218
:109080001A700023BB71BB790F2B70D8BB792C22CF
:1090900002FB03F34E4A1A44BB794E4931F81330B0
:1090A00007EE903AF8EE677AB0EE670A10460AF0DB
:1090B0006DFCF0EE407ABB79FCEEE77A17EE902A71
:1090C00091B24D4A22F81310BB791B014B4A1A4446
:1090D000BB79494931F8133007EE903AF8EE677AD8
:1090E000B0EE670A1046FBF715FEF0EE407ABB794A
:1090F000FCEEE77A17EE902A91B2424A22F813105A
:10910000BB792C2202FB03F3384A9C18BB79314A05
:10911000103332F813301A46BB7919461046FBF764
:1091200003FF034607EE903AF8EE677AB0EE670A5F
:1091300020460AF02BFCF0EE407ABB79FCEEE77A91
:1091400017EE902A90B22C4903F1100221F8120078
:10915000BA792949103331F813002A4902F1100372
:10916000024621F81320BB790133BB718BE7264BF4
:109170001B78002B20D0FFF7DBFBFFF7B9FAFFF7D6
:10918000BBF9224BD3F89830204B4FF0FF32C3F895
:1091900098201F4BD3F898301D4B4FF0FF32C3F887
:1091A00098201C4BD3F898301A4B4FF0FF32C3F87D
:1091B0009820194B01221A70BFF34F8F00BF00BFD8
:1091C0000C37BD4690BD00BF008000408C2C0020B5
:1091D000D0210020A00100200AD7A33D9A99993EF2
:1091E00066D6A34300FF7F470000000090240020C4
:1091F000CDCCCC3D99C1F544F41A00205027002075
:10920000F4010020381B00207F2C00200080034048
:109210000090034000900B40812C002080B582B06C
:1092200000AF584B1B78002B2CD0574B0222DA7022
:10923000564B1B78DBB2062B0CBF01230023DBB29D
:10924000002B07D0FDF740FF514B02221A704F4B05
:1092500000221A704D4B1B78DBB2052B94BF012303
:109260000023DBB2002B00F08680484B1B78DBB27A
:109270005A1CD1B2454A11701946434B454A525CBB
:109280001A7178E0404BDB78DBB23B603B6803F05F
:109290001003002B0ED01020FDF7ACFE3B6803F04E
:1092A0004003002B06D15020FDF7B4FE0220FDF74D
:1092B000A1FE63E0344B9B79FB713B6803F04003F4
:1092C000002B1BD0344B00221A70FDF7B9FE2E4B39
:1092D000C0229A702C4B304A1278D2B21B79D9B284
:1092E0002E4B99542A4B03221A705020FDF792FE00
:1092F0004220FDF77FFE244B9B79FB71FB7903F045
:109300005003002B25D05020FDF784FEFDF7AAFE68
:109310001D4BC8229A700220FDF76CFE204B1B7873
:109320005A1CD1B21E4A11701A4613469B001344B0
:109330005B001C4A13440A22184918460BF015FE1C
:109340002022002115480BF01EFE114B02221A703C
:1093500014E00D4A104B1B78DBB2591CC8B20E4901
:10936000087019461379DAB20C4B5A5445F20201CF
:1093700005480AF063FABFF34F8F00BF0837BD46B8
:1093800080BD00BF872C002000700640862C002086
:10939000882C002084550100892C0020D40C00204A
:1093A0008A2C0020F40C0020B0B582B000AF7860A9
:1093B00039607B68012B43D13B684FF6FF729342C3
:1093C0003ED1214808F009FF204808F007FD204859
:1093D00008F0EAFF1F4809F01EF81F4808F079FD61
:1093E0001E4809F06BFA1E48FAF7B4F91D48FAF75F
:1093F000C9FD1D480AF0AFF81C4809F0CBFD1C4B15
:109400000F241D46002C05DB2846FBF74DFC2C35B0
:10941000013CF7E7174B0F241D46002C05DB2846BF
:10942000FBF742FC2C35013CF7E7134B0F241D469C
:10943000002C05DB28460AF0C0FB1035013CF7E79D
:1094400000BF0837BD46B0BDC01D0020DC1D002098
:10945000601E00206C1E0020941E0020A81E00200C
:10946000141F0020441F0020182000202C20002062
:10947000D0210020902400205027002080B483B009
:1094800000AF03463960FB7197F90730002B0ADB08
:109490003B68DAB20C4997F907301201D2B20B449B
:1094A00083F800230AE03B68DAB20849FB7903F04D
:1094B0000F03043B1201D2B20B441A7600BF0C37E3
:1094C000BD465DF8047B704700E100E000ED00E080
:1094D00090B585B000AFF860B9607A603B60FB681A
:1094E000002B05D1144B154A4A21154806F090FC73
:1094F000144B154ADA62134B20221A63FB68114A97
:109500001A60FB681B68114A1A60FB681C6800201F
:1095100002F086FB03466360FB681B680C4A9A6591
:10952000FB680C4A1A6179685120FFF7A7FF00BF5A
:109530001437BD4690BD00BFF45501000C56010024
:10954000FC550100E42A0020502A002000100B40A6
:10955000482B0020D02A002080B582B000AF786070
:1095600039607B68002B06D1084B094A4FF4A4717F
:10957000084806F04DFC7B681B683968184601F006
:10958000A1FF034618460837BD4680BDF4550100CB
:10959000505701001C56010080B582B000AF7860C2
:1095A0007B68002B06D1084B084A40F24F1108484F
:1095B00006F02EFC7B681B6818460AF0C3FB0346C6
:1095C00018460837BD4680BDF4550100EC5801002F
:1095D0001C56010080B582B000AF786039607B68AE
:1095E000002B06D1084B094A4FF4AB71084806F02E
:1095F0000FFC7B681B683968184601F0A1FF034621
:1096000018460837BD4680BDF455010004590100D5
:109610001C56010080B58EB000AF78607B68002BCF
:1096200006D11C4B1C4A4FF4D8711C4806F0F0FBC5
:1096300007F12C0300221A605A6007F10C03202264
:10964000002118460BF09FFC00237B630C23FB607A
:1096500000233B6103233B7502237B75104BBB62E8
:1096600007F10C033B630023FB627B681B6807F177
:109670002C02114618460AF0FEFB78637B6B002B28
:1096800002D040F2097300E0002318463837BD4687
:1096900080BD00BFF4550100FC5601001C560100BE
:1096A0000800F9FF80B586B000AFF860B9607A6055
:1096B000BB68002B06D1154B154A4FF4E5711548D0
:1096C00006F0A6FBFB681B68B96818460AF0D3FBD6
:1096D00078617B69002B10D0BB681B68002B02D01F
:1096E000F868FFF797FF7B68002B08D07B68013B89
:1096F0007B607B69002BE5D102E000BF00E000BF8A
:109700007B6918461837BD4680BD00BF285601004A
:10971000105701001C56010080B58EB000AF786074
:109720007B68002B06D1204B204A40F20B212048B9
:1097300006F06EFB07F12C0300221A605A6007F155
:109740000C032022002118460BF01DFC00237B6334
:109750000D23FB607B685B6A1B043B6101237B7507
:1097600007F10C033B630023FB6207F12C03032288
:1097700019467868FFF796FF78637B6B002B0BD157
:10978000BB6903F48073002BEAD0BB695B0A03F06A
:109790000F03072B02D1E3E700BF00E000BF7B6BA4
:1097A00018463837BD4680BDF45501001C570100EE
:1097B0001C56010080B594B000AF786039607B68BA
:1097C000002B06D1334B344A4FF40B71334806F06B
:1097D0001FFB07F13C0300221A605A6007F11C03CB
:1097E0002022002118460BF0CEFB07F108030022CF
:1097F0001A605A609A60DA601A610023FB647B6821
:109800003033BB6404220021B86C0BF0BCFB7868D9
:10981000FFF782FF0346002B02D04FF4E36335E0ED
:109820007B685B6A19467868FFF796FE0346002B53
:1098300002D040F2157329E01623FB61012387F85B
:1098400025300423FB6001233B61BB6C7B6107F186
:109850001C033B6407F10803FB637B681B6807F18B
:109860003C02114618460AF006FBF864FB6C002B1C
:109870000BD1BA6A0A4B1340002B06D1BB6C1B6894
:109880007B647B6C1ABA3B681A60FB6C18465037D5
:10989000BD4680BDF4550100345701001C5601003F
:1098A0000800F9FF80B58EB000AF78607B68002BB0
:1098B00006D11A4B1A4A40F259211A4806F0A8FA62
:1098C00007F12C0300221A605A6007F10C032022D2
:1098D000002118460BF057FB00237B630323FB603A
:1098E00000233B6108237B7507F10C033B630023D6
:1098F000FB627B681B6807F12C02114618460AF0D0
:10990000BAFA78637B6B002B03D1BB691A0C7B68B6
:109910005A627B6B18463837BD4680BDF45501004E
:10992000685701001C56010080B594B000AFF86084
:10993000B9607A603B60FB68002B06D12E4B2F4A42
:1099400040F275212E4806F063FABB6D002B06D15C
:109950002C4B2A4A40F27621294806F059FA07F1A1
:10996000440300221A605A6007F1240320220021D8
:1099700018460BF008FB07F1100300221A605A602A
:109980009A60DA601A610023FB6406237B62BB687D
:10999000DB0763F07F43BB62BA6A7B689B000F21E1
:1099A00001FA03F3DB431340BB62BA6A7B689B0096
:1099B000396801FA03F31343BB62012387F82D30A2
:1099C00040237B610123BB61BB6DFB6107F1240375
:1099D000BB6407F110037B64FB681B6807F144025A
:1099E000114618460AF047FAF864FB6C002BFB6C32
:1099F00018465037BD4680BDF4550100745701002C
:109A00001C5601003056010080B584B000AF78606C
:109A100039607B68002B06D15C4B5D4A4FF42571A1
:109A20005C4806F0F5F93B68002B06D15A4B584AC2
:109A300040F29521574806F0EBF97B6803F51A735D
:109A4000FB603B681B681B0FDAB2FB681A703B684F
:109A50001B681B0EDBB203F00F03DAB2FB685A700F
:109A60003B681B68DB0DDBB203F00103DBB2002BAC
:109A700006D0FB685B8843F001039AB2FB685A800A
:109A80003B681B681B0DDBB203F00703DAB2FB680F
:109A90001A713B681B681B0CDBB203F00F03DAB2D0
:109AA000FB685A713B681B68DB0BDBB203F00103F8
:109AB000DBB2002B06D0FB685B8843F002039AB24E
:109AC000FB685A803B681B689B0ADBB203F01E03ED
:109AD000DAB2FB689A713B681B68DBB203F00303E0
:109AE000DAB2FB68DA713B685A68FB689A60FB6817
:109AF0005B78022B0ED0022B1ADC002B02D0012B3C
:109B000004D015E07B6801229A6214E07B6802228F
:109B10009A6210E07B6804229A627B68B3F86A322A
:109B200003F00203002B05D07B6808229A6201E053
:109B300000BF00E000BF7B6893F86D3203F00403C0
:109B4000002B05D07B68DB6A43F004027B68DA6295
:109B50007B6893F86F3203F00103002B05D07B681C
:109B6000DB6A43F080027B68DA627B6893F86F32CD
:109B700003F00203002B05D07B68DB6A43F0400250
:109B80007B68DA6200BF1037BD4680BDF455010026
:109B9000885701001C5601003856010080B59AB064
:109BA00000AF78607B68002B06D14A4B4A4A40F2EE
:109BB000CE214A4806F02CF907F1400300221A6032
:109BC0005A6007F120032022002118460BF0DBF930
:109BD00007F10C0300221A605A609A60DA601A6179
:109BE0007B6830337B6600233B6608220021786E59
:109BF0000BF0C9F97B685B6A19467868FFF7ACFC23
:109C00000346002B02D040F215735EE033233B6223
:109C1000012387F8293000237B6208233B6101235D
:109C20007B617B6EBB6107F10C033B6407F1200392
:109C30007B647B681B6807F14002114618460AF0F6
:109C40001AF938663B6E002B3ED1FA6A244B13405A
:109C5000002B39D17B681B685B7A022B06D0022B64
:109C60002ADC002B2BD0012B11D025E07B6E1B684A
:109C7000BB65BB6D1ABA7B6E1A607B6E04331A68C3
:109C80007B6E0433FA65FA6D12BA1A6018E07B6EC7
:109C90001B68FB64FB6C5BBABB64BA6C7B6E1A60BE
:109CA0007B6E04331A687B6E04337A657A6D52BA20
:109CB0003A653A6D1A6003E04FF4E16305E000BFD6
:109CC000796E7868FFF7A0FE3B6E18466837BD4690
:109CD00080BD00BFF4550100985701001C560100DB
:109CE0000800F9FF80B5A0B002AFF860B9607A60F3
:109CF000FB68002B06D1994B994A4FF44371994860
:109D000006F086F8FB6830337B6707F1100300220A
:109D10001A605A609A6000233B6740220021786FE6
:109D20000BF031F9FB689B6A012B06D9FB68B3F88D
:109D3000503203F48063002B02D14FF4E1632DE134
:109D40007B6F00937B68BA680021F868FFF7ECFD31
:109D50000346002B02D040F209731FE1FB681B6829
:109D60005B7A022B06D0022B66DC002B67D0012B1E
:109D70002CD061E07B6F1B68FB65FB6D1ABA7B6FB3
:109D80001A607B6F04331A687B6F04333A663A6E4D
:109D900012BA1A607B6F08331A687B6F08337A66D1
:109DA0007A6E12BA1A607B6F0C331A687B6F0C33B1
:109DB000BA66BA6E12BA1A607B6F10331A687B6F7C
:109DC0001033FA66FA6E12BA1A6039E07B6F1B68BC
:109DD000BB63BB6B5BBA7B637A6B7B6F1A607B6F19
:109DE00004331A687B6F04333A643A6C52BAFA63EC
:109DF000FA6B1A607B6F08331A687B6F0833BA649A
:109E0000BA6C52BA7A647A6C1A607B6F0C331A6837
:109E10007B6F0C333A653A6D52BAFA64FA6C1A6089
:109E20007B6F10331A687B6F1033BA65BA6D52BA04
:109E30007A657A6D1A6003E04FF4E163AEE000BF2B
:109E40007B6F1B689BB27B837B6F04331B681B0C8F
:109E50009BB23B837B6F04331B689BB2FB827B6F9F
:109E600008331B681B0C9BB2BB827B6F08331B68DB
:109E70009BB27B827B6F0C331B681B0C9BB23B82BB
:109E80007B6F0C331B681B029AB27B6F10331B680D
:109E90001B0E13433B67BB685B0007F1780213445A
:109EA00033F8683C1A467B6842FA03F303F0010377
:109EB000002B09D0BB689B003A6F22FA03F303F032
:109EC0000F037A689A4202D04FF4E16366E07B6F39
:109ED00000937B68BA680121F868FFF725FD034607
:109EE000002B02D040F2097358E0FB681B685B7AD4
:109EF000022B06D0022B2EDC002B35D0012B13D0E9
:109F000029E07B6F0C331A687B6F0C33FA62FA6AB4
:109F100012BA1A607B6F10331A687B6F10333A6382
:109F20003A6B12BA1A6020E07B6F0C331A687B6FB1
:109F30000C333A623A6A52BAFA61FA691A607B6F74
:109F400010331A687B6F1033BA62BA6A52BA7A62F7
:109F50007A6A1A6009E04FF4E1631FE0F4550100EA
:109F6000A45701001C56010000BF7B6F0C331B6817
:109F70001B029AB27B6F10331B681B0E13433B67A7
:109F8000BB689B003A6F22FA03F303F00F037A6871
:109F90009A4202D040F2167300E000231846783748
:109FA000BD4680BD80B58EB000AF786039607B68FB
:109FB000002B06D1244B254A40F27D31244805F080
:109FC00027FF07F12C0300221A605A6007F10C03E7
:109FD0002022002118460AF0D6FF00237B637B680D
:109FE0005B6A19467868FFF7B7FA0346002B02D080
:109FF00040F2157323E00623FB6001237B753B6869
:10A00000002B03D03B68012B03D005E000233B610C
:10A0100004E002233B6101E0042310E007F10C039C
:10A020003B630023FB627B681B6807F12C0211462F
:10A03000184609F020FF78637B6B002B7B6B18467A
:10A040003837BD4680BD00BFF4550100B857010048
:10A050001C56010080B584B000AF786039607B6821
:10A06000002B06D1914B924A40F2A331914805F062
:10A07000CFFE3B68002B06D18F4B8D4A4FF46971A0
:10A080008C4805F0C5FE7B6803F51373FB603B68E5
:10A090000C331B689B0FDAB2FB681A703B680C33F9
:10A0A0001B681B0CDAB2FB685A703B680C331B68E8
:10A0B0001B0ADAB2FB689A703B680C331B68DAB291
:10A0C000FB68DA703B6808331B681B0D9AB2FB68AB
:10A0D0009A803B6808331B681B0CDBB203F00F034C
:10A0E000DAB2FB689A713B6808331B6803F40043DB
:10A0F000002B06D0FB681B8943F001039AB2FB6872
:10A100001A813B6808331B6803F48043002B06D098
:10A11000FB681B8943F001039AB2FB681A813B6814
:10A1200008331B6803F40053002B06D0FB681B891F
:10A1300043F004039AB2FB681A813B6808331B683A
:10A1400003F48053002B06D0FB681B8943F00803FF
:10A150009AB2FB681A81FB681B78002B02D0012B96
:10A1600079D0ACE03B6808331B689A0040F6FC737A
:10A170001340FA68D360FB68DA683B6804331B68F5
:10A180009B0F1A43FB68DA603B6804331B68DB0EE5
:10A19000DBB203F00703DAB2FB681A743B680433DE
:10A1A0001B681B0EDBB203F00703DAB2FB685A74BC
:10A1B0003B6804331B681B0DDBB203F00E03DAB2FD
:10A1C000FB689A743B6804331B689B0CDBB203F09A
:10A1D0000703DAB2FB68DA743B6804331B68DB0BF5
:10A1E000DBB203F00703DAB2FB681A75FB68DB68C1
:10A1F0005A1CFB681B7D02339A407B68C3F8882297
:10A20000FB689B791A46012303FA02F27B68C3F8C4
:10A210008C227B68D3F88C32B3F5007F4ED07B68FC
:10A22000D3F888327A68D2F88C2202FB03F27B687A
:10A23000C3F888227B684FF40072C3F88C227B68D5
:10A24000D3F888227B68D3F88C32B2FBF3F27B68B8
:10A25000C3F8882232E07B684FF40072C3F88C2286
:10A260003B6808331B681B0403F47C12FB68DA604C
:10A27000FB68DA683B6804331B681B0C1A43FB68F5
:10A28000DA60FB68DB684FF6FE72934205D97B68A3
:10A29000DB6A43F010027B68DA62FB68DB6801333B
:10A2A0009A027B68C3F8882209E000BFF4550100D8
:10A2B000CC5701001C5601004056010000BF3B680E
:10A2C00004331B689B0BDBB203F00103DBB2002BF2
:10A2D00006D0FB681B8943F010039AB2FB681A8111
:10A2E0003B6804331B68DB09DBB203F07F03DAB29F
:10A2F000FB685A753B6804331B68DBB203F07F03CD
:10A30000DAB2FB689A753B681B689B0EDBB203F000
:10A310000703DAB2FB68DA753B681B689B0DDBB29A
:10A3200003F00F03DAB2FB681A763B681B685B0D1B
:10A33000DBB203F00103DBB2002B06D0FB681B8904
:10A3400043F040039AB2FB681A813B681B68DB0B41
:10A35000DBB203F00103DBB2002B06D0FB681B89E4
:10A3600043F080039AB2FB681A813B681B689B0B21
:10A37000DBB203F00103DBB2002B06D0FB681B89C4
:10A3800043F480739AB2FB681A813B681B685B0BCD
:10A39000DBB203F00103DBB2002B06D0FB681B89A4
:10A3A00043F400739AB2FB681A813B681B681B0B6D
:10A3B000DBB203F00103DBB2002B06D0FB681B8984
:10A3C00043F480639AB2FB681A813B681B689B0A5E
:10A3D000DBB203F00303DAB2FB685A7600BF103732
:10A3E000BD4680BD80B58EB000AF78607B68002B25
:10A3F00006D1234B234A4FF48161234805F008FD21
:10A4000007F12C0300221A605A6007F10C03202286
:10A41000002118460AF0B7FD00237B630923FB6087
:10A420007B685B6A1B043B6103237B7507F10C03AC
:10A430003B630023FB627B681B6807F12C0211461B
:10A44000184609F018FD78637B6B002B10D17B68F0
:10A4500003F1300007F10C030C33102219460AF007
:10A4600084FD7B68303319467868FFF7F3FD02E01E
:10A4700040F209737B637B6B18463837BD4680BD5D
:10A48000F4550100DC5701001C56010080B584B072
:10A4900000AF786039607B68002B06D1324B334ABD
:10A4A00040F22641324805F0B3FC3B68002B06D150
:10A4B000304B2E4A40F227412D4805F0A9FC7B681D
:10A4C00003F50E73FB603B680C331B681B0EDAB29E
:10A4D000FB681A703B680C331B681B0A9AB2FB6856
:10A4E0005A803B680C331B68DAB2FB681A713B6810
:10A4F00008331B681B0EDAB2FB685A713B680833DD
:10A500001B681B0CDAB2FB689A713B6808331B6846
:10A510001B0ADAB2FB68DA713B6808331B68DAB2EF
:10A52000FB681A723B6804331B681B0EDAB2FB68C7
:10A530005A723B6804331B681A02FB68DA60FB68D6
:10A54000DA683B681B681B0E1A43FB68DA603B68DD
:10A550001B681B0A9BB2C3F30B039AB2FB681A82F7
:10A5600000BF1037BD4680BDF4550100E85701001B
:10A570001C5601004856010080B58CB000AF7860D1
:10A580007B68002B06D1204B204A40F23F412048F7
:10A5900005F03EFC07F1280300221A605A6007F11B
:10A5A00008032022002118460AF0EDFC0223BB60BC
:10A5B0000023FB6003237B7407F10803FB62002385
:10A5C000BB627B681B6807F128021146184609F038
:10A5D00052FC0346002B11D17B6803F1300007F1D8
:10A5E00008030C33102219460AF0BFFC7B68303395
:10A5F00019467868FFF74AFF002301E040F209732B
:10A6000018463037BD4680BDF4550100F8570100AB
:10A610001C56010080B58EB000AF786039607B6851
:10A62000002B06D1334B344A40F25741334805F0F2
:10A63000EFFB07F1280300221A605A6007F10803B4
:10A640002022002118460AF09EFC01237B634FF470
:10A650007A733B632923BB603B68FB6004237B74F4
:10A660003DE000217868FEF777FF0346002B00D01D
:10A6700035E007F10803FB620023BB627B681B68BF
:10A6800007F128021146184609F0F5FB78637B6B49
:10A69000002B02D040F2097327E07B69002B1BDA04
:10A6A0007B6903F08043002B05D07B68DB6A43F0B5
:10A6B00002027B68DA627B6903F08073002B05D0AD
:10A6C0007B68DB6A43F020027B68DA627A697B6828
:10A6D000C3F83422002308E00A2000F065FF3B6B3A
:10A6E0005A1E3A63002BBCD17B6B18463837BD46E7
:10A6F00080BD00BFF4550100085801001C56010040
:10A7000080B58EB000AF78607B68002B06D1234BFC
:10A71000234A40F28E41234805F07AFB07F12803D3
:10A7200000221A605A6007F108032022002118460F
:10A730000AF029FC0A237B6300233B630823BB60E8
:10A740004FF4D573FB6009237B7407F10803FB62A8
:10A750000023BB627B681B6807F12802114618467C
:10A7600009F089FB38633B6B002B09D17B69DBB2B5
:10A77000AA2B03D040F20C733B6301E000233B6340
:10A780007B6B013B7B637B6B002B02D03B6B002B15
:10A79000E0D13B6B18463837BD4680BDF45501000B
:10A7A000305801001C56010080B584B000AF7860BD
:10A7B0007B68002B06D1344B344A40F2B541344813
:10A7C00005F026FB40F21B73FB607B6893F8933225
:10A7D000032B28D0012200217868FFF783FAF86064
:10A7E000FB68002B19D17B68012283F890227B68DB
:10A7F0001A687B685B69002B06D07B685B6925491A
:10A800008B4228BF0B4600E0224B1946104609F048
:10A8100071FA02467B681A6230E0FB68B3F5E16FBB
:10A820002CD100232BE07B6893F89032012B22D8A7
:10A83000012200217868FFF755FAF860FB68002BC9
:10A840001BD17B68012283F890227B681A687B68A1
:10A850005B69002B06D07B685B690E498B4228BF81
:10A860000B4600E00B4B1946104609F043FA02462E
:10A870007B681A6201E000BF00E000BFFB68184679
:10A880001037BD4680BD00BFF45501004C58010093
:10A890001C56010080F0FA0280B582B000AF7860EB
:10A8A00039607B68002B06D1424B434A40F2265167
:10A8B000424805F0ADFA3B68002B06D1404B3E4ABA
:10A8C00040F227513D4805F0A3FA3B681B689B0FF7
:10A8D000DAB27B6883F874223B681B685B0FDBB2DB
:10A8E00003F00103DAB27B6883F875223B681B68CA
:10A8F0009AB27B68A3F876223B685A687B68C3F8F3
:10A9000078223B6808331B681B0EDAB27B6883F839
:10A910007C223B6808331B681B0CDAB27B6883F827
:10A920007D223B6808331B681B0BDBB203F00F036F
:10A93000DAB27B6883F87E223B6808331B689BB2DF
:10A940001B029AB23B680C331B681B0E9BB213436D
:10A950009AB27B68A3F880223B680C331B681B0CFF
:10A96000DBB29B08DAB27B6883F882223B680C3347
:10A970001B681B0CDBB203F00303DAB27B6883F8BD
:10A9800083223B680C331B681B0ADBB21B09DAB25B
:10A990007B6883F884223B680C331B681B0ADBB29C
:10A9A00003F00F03DAB27B6883F8852200BF083713
:10A9B000BD4680BDF4550100605801001C560100E1
:10A9C0005056010080B598B000AF78607B68002BCE
:10A9D00006D1554B554A40F23951554805F018FA01
:10A9E0000023FB6507F1400300221A605A6007F15B
:10A9F00020032022002118460AF0C5FA07F10C03B3
:10AA000000221A605A609A60DA601A610023BB65FE
:10AA10007B6830337B6540220021786D0AF0B3FA01
:10AA20007868FEF779FE0346002B02D04FF4E3630B
:10AA300075E07B685B6A19467868FEF78DFD034612
:10AA4000002B02D040F2157369E00D233B62012315
:10AA500087F8293040233B6101237B617B6DBB611B
:10AA600007F120037B6407F10C033B647B681B68E0
:10AA700007F140021146184609F0FDF9B865BB6DB3
:10AA8000002B04D1FA6A2B4B1340002B02D040F26A
:10AA9000097344E07B681B685B7A022B06D0022BAB
:10AAA00034DC002B35D0012B17D02FE00023FB65C1
:10AAB0000FE0FB6D9B007A6D13441A68FB6D9B00E1
:10AAC000796D0B443A653A6D12BA1A60FB6D013329
:10AAD000FB65FB6D0F2BECD91CE00023FB6511E03F
:10AAE000FB6D9B007A6D13441A68FB6D9B00796DBA
:10AAF0000B44FA64FA6C52BABA64BA6C1A60FB6D11
:10AB00000133FB65FB6D0F2BEAD903E04FF4E163E2
:10AB100005E000BF796D7868FFF7BEFE0023184698
:10AB20006037BD4680BD00BFF4550100705801007C
:10AB30001C5601000800F9FF80B582B000AF7860B4
:10AB40000B46FB707B68002B06D10A4B0A4A40F289
:10AB50007E510A4805F05CF97B6818687B685B6A7F
:10AB6000FA78194600F06EFC034618460837BD46D1
:10AB700080BD00BFF4550100805801001C56010043
:10AB800080B594B000AFF860B9607A603B60FB6854
:10AB9000002B06D1484B494A40F29D51484805F0E8
:10ABA00037F9BB68002B06D1464B444A40F29E5110
:10ABB000434805F02DF9BB6D002B06D1424B3F4AAF
:10ABC00040F29F513E4805F023F93B68B3F5007F02
:10ABD00006D03E4B394A4FF4B461394805F018F9B4
:10ABE00007F1480300221A605A6007F12803202267
:10ABF000002118460AF0C7F907F1140300221A6071
:10AC00005A609A60DA601A61FB68DB6A03F002033B
:10AC1000002B03D03B68B3F5007F0ED1FB68D3F85F
:10AC20008C323A689A4208D83B68B3F5805F04D802
:10AC30003B6803F00303002B02D040F20C7337E0B3
:10AC4000F868FEF769FD0346002B02D04FF4E3637A
:10AC50002EE03B68BB61BB6DFB61BB683B620123BF
:10AC60003B75BB6D012B01D1112300E01223BB62A8
:10AC70007B68FB62FB68DB6A03F00203002B04D1F4
:10AC8000FB6ABA6902FB03F3FB62012387F83130E8
:10AC90000F4B7B6407F12803FB6407F11403BB64CB
:10ACA00007F1480303221946F868FEF7FBFC034648
:10ACB00018465037BD4680BDF4550100905801003C
:10ACC0001C560100545601005C56010068560100F4
:10ACD0000800F9FF80B594B000AFF860B9607A6001
:10ACE0003B60FB68002B06D1574B584A40F2CE51CF
:10ACF000574805F08DF8BB68002B06D1554B534AD9
:10AD000040F2CF51524805F083F8BB6D002B06D1BD
:10AD1000514B4E4A4FF4BA614D4805F079F83B6803
:10AD2000B3F5007F06D04D4B484A40F2D151484818
:10AD300005F06EF807F1440300221A605A6007F12B
:10AD400024032022002118460AF01DF907F1100300
:10AD500000221A605A609A60DA601A61FB68DB6A46
:10AD600003F00203002B03D03B68B3F5007F0ED144
:10AD7000FB68D3F88C323A689A4208D83B68B3F53E
:10AD8000805F04D83B6803F00303002B02D040F23D
:10AD90000C7354E0F868FEF7BFFC0346002B02D0AA
:10ADA0004FF4E3634BE000BFFB681B68184608F0F4
:10ADB000B3FF0346002BF7D101233B743B687B6153
:10ADC000012387F82D30264B3B64BB6D012B01D14D
:10ADD000182300E019237B627B68BB62FB68DB6A97
:10ADE00003F00203002B04D1BB6A7A6902FB03F370
:10ADF000BB62FB6DBA6D1A60BB6DBB61BB683B6229
:10AE000007F12403BB6407F110037B6407F14403DB
:10AE100003221946F868FEF745FCF864FB6C002B2A
:10AE20000CD0F96DF868FEF7C5FC0346002B05D180
:10AE3000FB6D1B68002B01D00023FB64FB6C1846E4
:10AE40005037BD4680BD00BFF45501009858010041
:10AE50001C560100545601005C5601006856010062
:10AE60000800F9FF80B582B000AF78607B68002BE6
:10AE700006D10F4B0F4A40F25E610F4804F0C8FF45
:10AE80007B68B3F8543203F40073002B06D17B685F
:10AE9000B3F8543203F48063002B01D0012300E0A7
:10AEA000002303F00103DBB218460837BD4680BD1E
:10AEB000F4550100A45801001C56010080B58CB067
:10AEC00002AFF860B9607A603B60FB68002B06D186
:10AED000504B514A40F26661504804F099FFBB68FC
:10AEE000002B06D14E4B4C4A40F267614B4804F0B0
:10AEF0008FFF3B68002B06D14A4B474A4FF4CD6188
:10AF0000464804F085FF3A687B681A44FB68D3F82A
:10AF100088329A4206D9444B3F4A40F269613F4821
:10AF200004F076FF0023FB61BB687B610123FB76A5
:10AF3000FB68303323F0030304333B613B683B621F
:10AF40005FE0FB695B02BA6813447B61FB685B7F6F
:10AF500083F00103DBB2002B15D0FB7E83F00103ED
:10AF6000DBB2002B04D17B6903F00303002B0AD072
:10AF700001237B624FF40072002138690AF003F864
:10AF80000023FB7610E03B6AB3F5803F08D33B6AB1
:10AF9000A3F57F43FF3B3B624FF6FF737B6203E009
:10AFA0003B6A7B6200233B62FB7E002B01D0796908
:10AFB00000E039697A68FB691A447B6A00934FF4B0
:10AFC0000073F868FFF7DCFD0346002B02D040F267
:10AFD00009731AE0FA697B6A1344FB61FB685B7FC3
:10AFE00083F00103DBB2002B0BD0FB7E83F0010367
:10AFF000DBB2002B05D04FF400723969786909F093
:10B00000B4FF3B6A002B9CD1002318462837BD466D
:10B0100080BD00BFF4550100B85801001C56010066
:10B02000545601005C5601009456010080B58CB066
:10B0300002AFF860B9607A603B60FB68002B06D114
:10B04000514B524A40F29E61514804F0E1FEBB6808
:10B05000002B06D14F4B4D4A40F29F614C4804F003
:10B06000D7FE3B68002B06D14B4B484A4FF4D461C6
:10B07000474804F0CDFE3A687B681A44FB68D3F871
:10B0800088329A4206D9454B404A40F2A161404875
:10B0900004F0BEFE00237B6200233B6100233B6281
:10B0A0000123FB77FB68303323F003030433BB61D8
:10B0B0003B683B625FE03A683B6AD31A5B02BA685E
:10B0C00013447B61FB685B7F83F00103DBB2002BE1
:10B0D00015D0FB7F83F00103DBB2002B04D17B6929
:10B0E00003F00303002B0AD001237B624FF40072AC
:10B0F0007969B86909F039FF0023FB7709E03B6AF9
:10B10000B3F5803F03D34FF6FF737B6201E03B6AE8
:10B110007B62FB7F002B01D0796900E0B9697A6816
:10B120003B681A443B6AD21A07F1100301937B6A09
:10B1300000934FF40073F868FFF7CCFD0346002B33
:10B1400002D040F209731AE03B693A6AD31A3B62B3
:10B15000FB685B7F83F00103DBB2002B0BD0FB7F2E
:10B1600083F00103DBB2002B05D04FF40072002105
:10B17000B86909F008FF3B6A002B9CD100231846F0
:10B180002837BD4680BD00BFF4550100C8580100F6
:10B190001C560100545601005C56010094560100F3
:10B1A00080B584B000AF78607B68002B06D1244B5B
:10B1B000244A4FF4E261244804F02AFE0023FB6095
:10B1C0000023BB60FB6843F44813FB607B680122EB
:10B1D00083F893227868FEF7DFF90346002B03D04B
:10B1E00040F21373BB6026E07868FFF789FA0346E4
:10B1F000002B0AD1FB6843F08043FB607B68DB6A6D
:10B2000043F008027B68DA6209E07868FEF7C4F967
:10B210000346002B03D040F21373BB600BE0F968C8
:10B220007868FFF7F7F90346002B03D040F2147358
:10B23000BB6000E000BFBB6818461037BD4680BD4C
:10B24000F4550100D85801001C56010080B582B0A9
:10B2500000AF78607B68002B06D14E4B4E4A40F21F
:10B2600086714E4804F0D4FD7B681B7F012B06D00D
:10B270004B4B494A40F28771484804F0C9FD7B684E
:10B280000022DA627B681B680021184608F03CFE49
:10B290007B681B684349184608F02CFD02467B6812
:10B2A0001A627B681B68184608F016FD7868FFF77D
:10B2B00077FF034640F22A72934202D140F22A738A
:10B2C00064E07868FFF758F90346002B02D040F29B
:10B2D0000D735BE07868FEF7E5FA0346002B02D0B9
:10B2E00040F20E7352E07868FFF77CF80346002BBB
:10B2F00002D040F20F7349E001217868FFF71CFC8F
:10B300000346002B02D04FF4E2633FE07B681B68EA
:10B310002549184608F0EEFC02467B681A627868F8
:10B32000FEF73CFC0346002B02D040F211732DE0E7
:10B330007B68DB6A03F00403002B0FD001217868DF
:10B34000FEF730FE0346002B02D040F212731DE0E0
:10B350007B681B680121184608F0D6FD4FF4007188
:10B360007868FEF737F90346002B02D040F20A73E3
:10B370000CE07868FFF718FA0346002B02D040F281
:10B380001B7303E07868FFF71DFB0023184608379E
:10B39000BD4680BDF4550100F85801001C5601005F
:10B3A000C4560100801A060040787D0180B582B045
:10B3B00000AF78607B68002B06D11E4B1E4A40F21E
:10B3C000D6711E4804F024FD7B681B69002B06D152
:10B3D0001B4B194A40F2D771184804F019FD7B68DD
:10B3E0001B7F83F00103DBB2002B09D07B681B6855
:10B3F000184600F0EDF80346002B01D0012315E0BC
:10B400007B681B691B78012B04D07B681B691B7848
:10B41000022B07D17B681A687B681B6919461046A6
:10B4200008F008FD7B6801221A77002318460837C8
:10B43000BD4680BDF4550100145901001C560100A1
:10B44000E056010080B58EB000AFF860B9601346D9
:10B45000FB7107F1300300221A605A6007F11003F4
:10B4600020220021184609F08EFD07233B61FB795D
:10B47000002B05D0BB681B047B6101237B7603E0B6
:10B4800000237B6100237B7607F110037B6300239D
:10B490003B6307F130031946F86808F0ECFC0346FB
:10B4A000002B04D1FA69064B1340002B02D040F266
:10B4B000097300E0002318463837BD4680BD00BF41
:10B4C0000800F9FF80B58CB000AF7860396007F1F3
:10B4D000280300221A605A6007F108032022002185
:10B4E000184609F050FD3723BB603B681B04FB6026
:10B4F00001237B7407F10803FB620023BB6207F1A1
:10B5000028031946786808F0B6FC0346002B04D1DE
:10B510007A690A4B1340002B02D040F2097308E00D
:10B520007B6903F02003002B02D140F20C7300E092
:10B53000002318463037BD4680BD00BF0800F9FF24
:10B5400080B58CB000AF7860396007F12803002225
:10B550001A605A6007F1080320220021184609F0FA
:10B5600012FD1023BB603B68FB6001237B7407F175
:10B570000803FB620023BB6207F1280319467868C1
:10B5800008F079FC0346002B04D17A69054B13407F
:10B59000002B02D040F2097300E000231846303738
:10B5A000BD4680BD0800F9FF80B582B000AF78606D
:10B5B0007B684FF47A7202FB03F30449184600F0EB
:10B5C000A5FE00BF0837BD4680BD00BF000E27079F
:10B5D00080B584B000AF78607B68002B05D1154B37
:10B5E000154AB021154804F013FC7B689B6D002BB5
:10B5F00005D1134B104AB121104804F009FC7B68B7
:10B60000FB60FB6802225A72FB6802229A72FB6896
:10B610008022DA60FB6880221A61FB681A68FB6886
:10B6200008331946104602F053FC00231846103721
:10B63000BD4680BD205901007059010030590100FC
:10B640005859010080B584B000AF78600023FB60DA
:10B6500009E00E4AFB6852F823307A689A4206D015
:10B66000FB680133FB60FB68012BF2D900E000BFEF
:10B67000FB68012B05D9064B064A3521064804F024
:10B68000C7FBFB6818461037BD4680BD80590100D6
:10B6900090590100F4590100B459010080B584B0FB
:10B6A00000AF786039603B68002B05D13E4B3F4AC4
:10B6B00042213F4804F0ACFB7868FFF7C3FF034624
:10B6C0003C4A52F82330184608F038FC3B685B7857
:10B6D00003F003023B681B799B0003F00C03134348
:10B6E000FB603B685B79042B03D0FB6843F01003DD
:10B6F000FB603B68DB785B0103F06003FA6813438F
:10B70000FB603B68DB79002B03D0FB6843F08003D0
:10B71000FB607B68FA689A607B68DB6823F00F0344
:10B72000FB603B685B79042B06D03B685B7903F0D8
:10B730000303FA681343FB603B689B79002B03D03B
:10B74000FB6843F00403FB603B689B78002B03D04D
:10B75000FB6843F00803FB607B68FA68DA607B688B
:10B760001B6A23F00303FB603B681B7803F00303B1
:10B77000FA681343FB607B68FA681A623B681B7ABD
:10B78000002B06D07B685B6A43F008027B685A6234
:10B7900005E07B685B6A23F008027B685A6200BFA1
:10B7A0001037BD4680BD00BFC4590100085A0100D2
:10B7B000B45901008859010080B586B000AFF86027
:10B7C000B9607A60BB68012B06D9174B174A40F263
:10B7D000C711174804F01CFB7B68002B06D1154BE2
:10B7E000124A4FF4E471124804F012FB7B681B68A4
:10B7F00003F01F037B617B685B79002B03D07B69BF
:10B8000043F020037B617B681B79002B03D07B69AD
:10B8100043F040037B61FB68BA68796943F8221002
:10B8200000BF1837BD4680BDD4590100145A01002D
:10B83000B4590100C459010080B584B000AF7860EC
:10B8400039603B68012B06D90C4B0D4A40F2E511DB
:10B850000C4804F0DDFA0023FB607B683A6853F87B
:10B86000223003F08003002B03D0FB6843F08003F9
:10B87000FB60FB6818461037BD4680BDD4590100F7
:10B880002C5A0100B459010080B483B000AF786035
:10B89000084B1B6823F440227B689B0403F440237D
:10B8A000044913430B6000BF0C37BD465DF8047BB1
:10B8B000704700BF0070044080B483B000AF786070
:10B8C0000B4B03F5805304331B6823F440327B6831
:10B8D0001B0403F4403306491A4301F58053043333
:10B8E0001A6000BF0C37BD465DF8047B704700BF8F
:10B8F0000070044080B582B000AF1A4B1B7BDBB2F6
:10B9000003F00303022B22D0022B23D8002B02D0FA
:10B91000012B0ED01EE0144B1B68002B05D1134BDE
:10B92000134ADA21134804F073FA0F4B1B687B604B
:10B9300013E0114B1B68002B05D1104B0C4ADF2183
:10B940000C4804F065FA0C4B1B687B6005E00C4B5F
:10B950007B6002E000237B6000BF7B6818460837ED
:10B96000BD4680BD00400640582B0020485A0100CB
:10B97000A85A01005C5A01005C2B00206C5A01009F
:10B98000006CDC0280B582B000AFFFF7B3FF7860D7
:10B99000254B1B78DBB2DB08DBB203F00703FB703F
:10B9A000FB787A6822FA03F37B601F4B5B78DBB28B
:10B9B0001B09DBB203F00303BB701B4B1B7BDBB229
:10B9C00003F003037B70BB78002B02D07B78002B45
:10B9D00002D07B78022B21D1FB78072B14D0072BC8
:10B9E00019DC052B02DC002B03DA14E0062B04D053
:10B9F00011E07B685B097B6011E07B680B4AA2FB6E
:10BA000003231B097B600AE07B68094AA2FB03232E
:10BA1000DB087B6003E000237B6000E000BF7B6805
:10BA200018460837BD4680BD00400640CDCCCCCC82
:10BA3000ABAAAAAA80B483B000AF0E4B9B79DBB24D
:10BA400003F00103002B03D10B4B1B687B600AE062
:10BA50000A4B1A68074B1B7ADBB25B0803F007033B
:10BA600022FA03F37B607B6818460C37BD465DF80D
:10BA7000047B7047004006400401002008010020BC
:10BA800080B582B000AF094B9B79DBB203F01003A5
:10BA9000002B03D1FFF776FF786002E0044B1B68B0
:10BAA0007B607B6818460837BD4680BD0040064075
:10BAB0000401002080B485B000AF78607B6849F64F
:10BAC0009702934202D80023FB7308E07B68074A81
:10BAD000934202D80123FB7301E00223FB73FB7B3B
:10BAE00018461437BD465DF8047B704700127A0093
:10BAF00080B582B000AF0E4B1B78DBB25BB2002B7F
:10BB00000EDA0C4B1B68002B06D10B4B0B4A40F294
:10BB100067110B4804F07CF9064B1B687B6001E061
:10BB200000237B607B6818460837BD4680BD00BF98
:10BB300000500640582B0020805A0100C05A0100D6
:10BB40005C5A010080B582B000AF1A4B1B689B0C99
:10BB500003F00303032B21D0032B23D8002B02D0A7
:10BB6000022B0CD01EE0FFF7C3FF0346B3F5004FD6
:10BB700002D14FF4004300E000237B6015E00E4B40
:10BB80001B68002B06D10D4B0D4A4FF4C1710D48B7
:10BB900004F03EF9084B1B687B6006E04FF47A73B3
:10BBA0007B6002E000237B6000BF7B68184608379B
:10BBB000BD4680BD007004405C2B00208C5A010003
:10BBC000D85A01005C5A010080B582B000AF124B18
:10BBD00003F5805304331B681B0C03F00303032B92
:10BBE0000ED0032B0FD8002B02D0012B04D00AE07B
:10BBF00000F090F9786009E000F0E6F9786005E07F
:10BC0000064B7B6002E000237B6000BF7B68184628
:10BC10000837BD4680BD00BF00700440006CDC02E8
:10BC200080B584B000AF0346FB71FB79132B00F2A3
:10BC30008E8001A252F823F089BC000089BC00006C
:10BC4000A9BC0000C9BC0000E9BC00004FBD000059
:10BC500009BD000011BD000019BD00004FBD00006E
:10BC60004FBD000021BD000029BD000031BD000016
:10BC700039BD00004FBD00004FBD00004FBD0000AA
:10BC800041BD000047BD000000F012F90246344BF0
:10BC900003F5825304331B681B0F03F00F030133BA
:10BCA000B2FBF3F3FB6055E000F002F902462C4BC7
:10BCB00003F5825304331B681B0E03F00F0301339B
:10BCC000B2FBF3F3FB6045E000F0F2F80246244BD0
:10BCD00003F5825304331B681B0D03F00F0301337C
:10BCE000B2FBF3F3FB6035E000F0E2F802461C4BD8
:10BCF00003F5825304331B681B0C03F00F0301335D
:10BD0000B2FBF3F3FB6025E0FFF75EFFF86021E094
:10BD1000FFF718FFF8601DE0FFF7EAFEF86019E092
:10BD200008F08BFAF86015E000F036F9F86011E0E1
:10BD300000F0F0F8F8600DE000F046F9F86009E076
:10BD4000084BFB6006E04FF47A73FB6002E00023CF
:10BD5000FB6000BFFB6818461037BD4680BD00BFC2
:10BD600000700440006CDC0280B582B000AF7860E7
:10BD70000A497B685A6801F5825304331A607B686C
:10BD80001B781846FFF798FD7B685B781846FFF72D
:10BD90007BFD00BF0837BD4680BD00BF007004407A
:10BDA00080B584B000AF786039600123FB733948F7
:10BDB00008F0ECF97B68002B0CD1374B03F580536E
:10BDC00004331B68344923F4802201F58053043383
:10BDD0001A6045E03B68314A934214D03B682F4AD1
:10BDE00093422CD83B682E4A934213D03B682C4A8E
:10BDF000934224D83B682B4A934219D03B682A4A85
:10BE000093420ED01BE0244B03F5825308330922E2
:10BE10001A6017E0204B03F58253083302221A60A0
:10BE200010E01D4B03F58253083305221A6009E028
:10BE3000194B03F58253083300221A6002E00023F5
:10BE4000FB7300BF144B03F5805304331B6823F4CA
:10BE5000E02211497B681A4301F5805304331A60CC
:10BE60000C4808F079F97B68B3F5E02F0DD10F4B42
:10BE7000032283F844210D4B93F84031DBB20B4A87
:10BE800063F07F03DBB282F84031FB7B184610374A
:10BE9000BD4680BD1200341000700440000E27071C
:10BEA00000D8B805006CDC0200A24A04002007405C
:10BEB00080B582B000AF164B9B79DBB29B0803F0D4
:10BEC00003033B603B68032B1AD801A252F823F00E
:10BED000E9BE0000F1BE0000F9BE0000E1BE0000B6
:10BEE00000F072F878600EE000F014F878600AE074
:10BEF000FFF7A0FD786006E0FFF7FCFC786002E049
:10BF000000237B6000BF7B6818460837BD4680BDB4
:10BF10000040064080B584B000AF1D4B5B78DBB2BB
:10BF200003F00203002B06D1194B9B79DBB203F01F
:10BF30002003002B02D00023FB6024E0FFF7A0FDCC
:10BF4000B860BB68002B02D1BB68FB601BE0104BE4
:10BF5000DB78DBB25B09DBB203F00303FB710C4B54
:10BF6000DB78DBB2DB09DBB203F00103BB71FA79EA
:10BF7000BB7908495200134431F813301A46BB68A4
:10BF800002FB03F3FB60FB6818461037BD4680BD1B
:10BF900000400640F05A010080B582B000AF094B66
:10BFA0001B78DBB203F00203002B02D100237B607D
:10BFB00002E0FFF73FFD78607B6818460837BD4612
:10BFC00080BD00BF0040064080B584B000AF1C4B70
:10BFD0009B79DBB203F04003002B02D10023FB600E
:10BFE00028E008F023F9B860BB68002B06D1154B98
:10BFF000154A40F2F921154803F00AFF104B1B794E
:10C00000DBB203F01F03DBB20133FB71FB79BA68CB
:10C01000B2FBF3F3BB600A4B5B79DBB203F01F03A7
:10C02000DBB21833BB71BA79BB6802FB03F3BB60A8
:10C03000BB68FB60FB6818461037BD4680BD00BF7B
:10C04000004006409C5A0100005B01005C5A010060
:10C0500080B485B000AF0346FB71174B1B7BDBB28E
:10C0600003F00302FB799A4202D00123FB7301E043
:10C070000023FB73104B1B7BDBB223F00303DAB20C
:10C08000FB7903F00303DBB20B491343DBB20B7301
:10C09000FB7B002B09D040F2DC53BB6000E000BF0B
:10C0A000BB685A1EBA60002BF9D10023184614371A
:10C0B000BD465DF8047B70470040064080B584B003
:10C0C00000AF78607B68002B06D11E4B1E4A40F201
:10C0D000F9311E4803F09CFE0023FB737B685B78FC
:10C0E00003F01F03DAB2FB7B1343FB73184AFB7B9D
:10C0F0001371174B5B79DBB223F01F03DAB27B6855
:10C100009B7803F01F03DBB211491343DBB24B7181
:10C110000F4B1B79DAB27B681B781343DBB20C4AF6
:10C1200043F04003DBB2137100BF094B9B79DBB2D4
:10C1300003F04003002BF8D000BF00BF1037BD460E
:10C1400080BD00BFCC590100145B01005C5A0100A6
:10C150000040064080B584B000AF78607B681B6803
:10C160001846FFF7A7FC0346FB737B681B7919464B
:10C17000194808F041F8194B5B78DBB223F03C0317
:10C18000DAB2FB7B1B01DBB203F03003DBB21343FB
:10C19000DAB27B685B7911491343DBB24B707B6881
:10C1A000063319460C4808F00DF87B685B79002BC4
:10C1B0000DD0094B1B78DBB25BB2002B07DA00BF56
:10C1C000064B9B79DBB203F00203002BF8D000BFD3
:10C1D0001037BD4680BD00BF0050064000400640FD
:10C1E00080B582B000AF03463960FB713B68002B1D
:10C1F00006D1254B254A40F26971254803F008FE17
:10C20000244B5B78DBB2234A23F00203DBB253708A
:10C21000204B1B78DBB203F03B03DBB21D4A63F01B
:10C220007F03DBB2137000BF1A4B9B79DBB203F0C4
:10C230001C03082BF8D1174B5B79DBB2154A23F0AE
:10C240004003DBB2537100BF124B9B79DBB203F0AA
:10C250002003002BF8D13868FFF730FF0D4B5B79D6
:10C26000DBB20C4A43F04003DBB2537100BF094B11
:10C270009B79DBB203F02003002BF8D00023184693
:10C280000837BD4680BD00BFCC590100285B0100C6
:10C290005C5A01000040064080B582B000AF034602
:10C2A0003A60FB710B46BB713B68002B06D1134B08
:10C2B000134A40F68201134803F0AAFDFB791846A1
:10C2C000FFF7C6FEBB7939681846FFF789FF0E4BAA
:10C2D0001B78DBB20C4A03F03F03DBB2137000BFE4
:10C2E000094B9B79DBB29B0803F00303032BF7D1C7
:10C2F000002318460837BD4680BD00BFCC59010059
:10C300003C5B01005C5A010000400640B0B584B0BF
:10C3100000AF786039607B68002B05D11F4B204A45
:10C32000F321204803F074FD7B6818464FF00001AC
:10C330003B681A464FF0000302FB01F500FB03F4D3
:10C340002C44A0FB020163181946174A4FF0000362
:10C3500003F0E2FB02460B46C7E90223D7E90223BA
:10C36000012B08BF002A05D3104B0D4AF5210D48BB
:10C3700003F04EFDD7E902014FF000024FF0000339
:10C38000820842EA81728B08C7E90223BB6818461B
:10C3900007F06DFF00BF1037BD46B0BD505B010018
:10C3A000845B0100605B010040420F00705B010094
:10C3B00080B584B000AF78600023FB6006E00D4AD2
:10C3C0007B68934206D0FB680133FB60FB68002B5F
:10C3D000F5D000E000BFFB68002B05D0064B074AF4
:10C3E0003B21074803F014FDFB6818461037BD4693
:10C3F00080BD00BF00100240985B0100D05B0100CF
:10C40000C05B010080B582B000AF78607868FFF74C
:10C41000CFFF044B184607F03AFF00BF0837BD4670
:10C4200080BD00BF01003C1080B582B000AF7860D5
:10C430003960786807F045FF0346002B05D0094BAB
:10C440001B6839687868984704E0074B1B683968AF
:10C4500078689847BFF34F8F00BF00BF0837BD46CD
:10C4600080BD00BF6C2B0020702B002080B500AF7A
:10C47000094B1B68002B06D1084B094A40F6930173
:10C48000084803F0C5FC044B1B6819460648FFF733
:10C49000CBFF00BF80BD00BF602B0020145C0100FB
:10C4A0005C5C0100085C010000C0024080B500AF88
:10C4B000094B5B68002B06D1084B094A40F69B01EB
:10C4C000084803F0A5FC044B5B6819460648FFF7D3
:10C4D000ABFF00BF80BD00BF602B00202C5C0100C3
:10C4E000745C0100085C010000D0024080B500AF20
:10C4F000094B9B68002B06D1084B094A40F6A30163
:10C50000084803F085FC044B9B6819460648FFF772
:10C510008BFF00BF80BD00BF602B0020445C01008A
:10C520008C5C0100085C010000C00A4080B584B04A
:10C5300000AF78600023FB6006E00D4A7B68934201
:10C5400006D0FB680133FB60FB68002BF5D000E0F0
:10C5500000BFFB68002B05D0064B074A4A2107485D
:10C5600003F056FCFB6818461037BD4680BD00BF7F
:10C5700000800040A45C0100545D0100C85C010023
:10C5800080B584B000AFF860B9607A60BB680F2BEB
:10C5900005D94E4B4E4A58214E4803F039FC7B6872
:10C5A000002B05D14C4B4A4A59214A4803F030FC34
:10C5B0007B6803F01F03002B05D0484B444A5A21E7
:10C5C000444803F025FC7B681A68F968BB6880332F
:10C5D0005B010B441A607B689B8899B2FA68BB6860
:10C5E00080335B01134404330A461A807B68DB887E
:10C5F00099B2FA68BB6880335B01134406330A467C
:10C600001A807B689A68F968BB685B010B4403F584
:10C61000805308331A607B68DA68F968BB685B018D
:10C620000B4403F580530C331A607B681A69F96870
:10C63000BB685B010B4403F5805310331A607B68C1
:10C640009B8A99B2FA68BB685B01134403F5805377
:10C6500014330A461A807B68DB8A99B2FA68BB6891
:10C660005B01134403F5805316330A461A807B6836
:10C670009A69F968BB685B010B4403F58053183372
:10C680001A60FA68BB685B01134403F580531C33DE
:10C6900000221A807B689B8B99B2FA68BB685B01A9
:10C6A000134403F580531C330A461A807B68DB8BE6
:10C6B00099B2FA68BB685B01134403F580531E33DB
:10C6C0000A461A8000BF1037BD4680BDD45C010009
:10C6D000685D0100C85C0100085D0100145D010097
:10C6E00080B584B000AF786039603B68002B05D11D
:10C6F000204B214A7821214803F08AFB7868FFF714
:10C7000015FF1F4B184607F0EFFD7B680022DA602B
:10C710007B684FF0FF325A627B684FF0FF32DA627B
:10C720007B681B68FB60FB6823F05603FB603B687B
:10C730009B789B0003F004023B685B781B0103F0CD
:10C7400010031A433B681B789B0103F040031A4314
:10C750003B68DB785B0003F002031A43FB6813437A
:10C7600043F08003FB607B68FA681A6000BF1037F3
:10C77000BD4680BD345D0100785D0100C85C0100EC
:10C780000100401080B582B000AF786039603B682E
:10C790000F2B05D9084B094AC421094803F038FB7F
:10C7A0003B6880335B017A681344184600F00AF84E
:10C7B00000BF0837BD4680BDD45C0100845D010028
:10C7C000C85C010080B582B000AF78607B68002B48
:10C7D00006D11C4B1C4A40F2A7111C4803F018FB61
:10C7E0007B6803F01F03002B06D0194B164A4FF449
:10C7F000D471164803F00CFB7B6800221A607B683A
:10C8000000229A807B680022DA807B6800229A608E
:10C810007B680022DA607B6800221A617B68002254
:10C820009A827B680022DA827B6800229A617B68A8
:10C8300008229A837B680022DA8300BF0837BD464E
:10C8400080BD00BF085D0100985D0100C85C01006B
:10C85000145D010080B584B000AF786039603B683A
:10C860000F2B06D9194B1A4A40F2CD21194803F073
:10C87000CFFA0023FB607A683B685B01134403F541
:10C8800080531C331B889BB2DB0903F00103FA6859
:10C890001343FB607B68DA6A3B6822FA03F35B00B0
:10C8A00003F00203FA681343FB607B685A6A3B6833
:10C8B00022FA03F39B0003F00403FA681343FB60BE
:10C8C000FB6818461037BD4680BD00BFD45C010030
:10C8D000A85D0100C85C010080B584B000AFF860BD
:10C8E000B9607A60BB680F2B06D9134B134A40F22C
:10C8F000E521134803F08CFA7B6803F00103002B59
:10C9000003D0BB68DAB2FB681A777B6803F00203D6
:10C91000002B03D0BB68DAB2FB689A777B6803F020
:10C920000403002B03D0BB68DAB2FB68DA7700BFE0
:10C930001037BD4680BD00BFD45C0100C45D01005E
:10C94000C85C010090B589B000AF78607B68002BAF
:10C9500006D1554B554A40F22351554803F058FA39
:10C960007B689B687A68127CDA777B689A687B6858
:10C970001B7C5B01134403F580531C331B889BB263
:10C9800003F08003002B14BF01230023BB767B68D8
:10C99000DB68002B0CD17B681B68002B7FD07B6889
:10C9A0001C687B685968BA7E00237868A04776E0E7
:10C9B0007B689A687B681B7C5B01134403F580539A
:10C9C00018331B687B617B68DB681A467B699B1A9E
:10C9D0007B617B695B093B61BB7E002B02D03B69BD
:10C9E000FB760EE03B69002B04D03B69DBB2013BD8
:10C9F000DBB205E07B681B7D5BB2DBB2013BDBB2E7
:10CA0000FB767B685B7C5AB297F91B309A4213D154
:10CA10007B68DB7CFB737B681B7DBB7397F90F2006
:10CA200097F90E309A4204D17B68DB7C5BB2FB61E4
:10CA300012E00023FB610FE0FB7E7A68527C52B269
:10CA40009B1AFB61FB69002B06DA7B681B7D5BB2DE
:10CA50001A46FB691344FB6197F91B207B685A74E3
:10CA60007B68DB7C5BB2DAB2FB69DBB2D31ADBB288
:10CA70005AB27B68DA747B681B68002B07D07B682E
:10CA80001C687B685968FB69BA7E7868A047BB7EE2
:10CA9000002B04D07B689B687A68127C1A7700BFF1
:10CAA0002437BD4690BD00BF445D0100E45D010038
:10CAB000C85C010080B500AF044B1B681846FFF747
:10CAC00041FFBFF34F8F00BF00BF80BD742B00201C
:10CAD00080B500AF044B5B681846FFF733FFBFF328
:10CAE0004F8F00BF00BF80BD742B002080B500AF0A
:10CAF000044BDB681846FFF725FFBFF34F8F00BFDD
:10CB000000BF80BD742B002080B500AF044B1B69B3
:10CB10001846FFF717FFBFF34F8F00BF00BF80BD60
:10CB2000742B002080B500AF044B5B691846FFF7FB
:10CB300009FFBFF34F8F00BF00BF80BD742B0020E3
:10CB400080B500AF044B9B691846FFF7FBFEBFF3AF
:10CB50004F8F00BF00BF80BD742B002080B500AF99
:10CB6000044BDB691846FFF7EDFEBFF34F8F00BFA4
:10CB700000BF80BD742B002080B500AF044B1B6A42
:10CB80001846FFF7DFFEBFF34F8F00BF00BF80BD29
:10CB9000742B002080B500AF044B5B6A1846FFF78A
:10CBA000D1FEBFF34F8F00BF00BF80BD742B0020AC
:10CBB00080B500AF044B9B6A1846FFF7C3FEBFF376
:10CBC0004F8F00BF00BF80BD742B002080B500AF29
:10CBD000044BDB6A1846FFF7B5FEBFF34F8F00BF6B
:10CBE00000BF80BD742B002080B500AF044B1B6BD1
:10CBF0001846FFF7A7FEBFF34F8F00BF00BF80BDF1
:10CC0000742B002080B500AF044B5B6B1846FFF718
:10CC100099FEBFF34F8F00BF00BF80BD742B002073
:10CC200080B500AF044B9B6B1846FFF78BFEBFF33C
:10CC30004F8F00BF00BF80BD742B002080B500AFB8
:10CC4000044BDB6B1846FFF77DFEBFF34F8F00BF31
:10CC500000BF80BD742B002080B500AF054B1B6862
:10CC6000054A1268114605489847BFF34F8F00BF29
:10CC700000BF80BDB82B0020B42B002000000C406A
:10CC800080B500AF054B1B68054A12681146054880
:10CC90009847BFF34F8F00BF00BF80BDBC2B002063
:10CCA000B42B002000000C4080B500AF054B1B6882
:10CCB000054A1268114605489847BFF34F8F00BFD9
:10CCC00000BF80BDC02B0020B42B002000000C4012
:10CCD00080B500AF054B1B68054A12681146054830
:10CCE0009847BFF34F8F00BF00BF80BDC42B00200B
:10CCF000B42B002000000C4080B500AF0B4B1B682C
:10CD0000002B06D10A4B0B4A40F683510A4803F028
:10CD10007FF80A4B1B68054A126811460848984775
:10CD2000BFF34F8F00BF00BF80BD00BFC82B0020E6
:10CD30002C5E0100485E01001C5E0100CC2B00202F
:10CD40000040024080B584B000AF78600423BB602F
:10CD50000023FB6009E00F4AFB6852F823307A6831
:10CD60009A4207D0FB680133FB60FA68BB689A42BD
:10CD7000F1D300E000BFFA68BB689A4205D3064BC6
:10CD8000064A5021064803F043F8FB68184610375E
:10CD9000BD4680BD605E0100805E0100345F010021
:10CDA0009C5E010080B586B000AF786039600023DA
:10CDB000FB7500233B610023FB607B68464A93427E
:10CDC00011D07B68454A93420DD07B68444A934218
:10CDD00009D07B68434A934205D0434B434A5B21C9
:10CDE000434803F015F87B689B6DFB60FB6843F0DC
:10CDF0000803FB607B685B6E3B610023FB750BE007
:10CE0000FB7DDB000533012202FA03F33A69134389
:10CE10003B61FB7D0133FB75FA7D7B682E498B42BC
:10CE200013D07B682D498B420DD07B682C498B42F7
:10CE300007D07B682B498B4201D1042306E07F2376
:10CE400004E0012302E0012300E004239342D7D849
:10CE50007B683A695A667B68D3F88C303B613B69E2
:10CE600043F0B4033B613B6803F08003002B03D025
:10CE70003B6943F4F8533B613B6803F07003002BBC
:10CE80001ED03B6943F4F8133B613B6803F0100389
:10CE9000002B03D0FB6843F01003FB603B6803F0FA
:10CEA0002003002B03D0FB6843F02003FB603B68AA
:10CEB00003F04003002B03D0FB6843F04003FB600A
:10CEC0007B68FA689A657B683A69C3F88C2000BF72
:10CED0001837BD4680BD00BF00800340009003406E
:10CEE00000A0034000900B40A85E0100445F0100D9
:10CEF0009C5E010080B586B000AF78603960002389
:10CF00007B6100233B617B68454A934214D07B6878
:10CF1000444A93420ED07B68434A934208D07B68D0
:10CF2000424A934201D1082307E04FF0FF3304E067
:10CF3000022302E0022300E00823FB7397F90F307D
:10CF4000B3F1FF3F05D13A4B3A4A98213A4802F0F3
:10CF50005FFF7B68D3F88C3043F004027B68C3F832
:10CF60008C207B685B6E3B6100237B610BE07B69FF
:10CF7000DB000533012202FA03F33A6913433B61F4
:10CF80007B6901337B6197F90F305B087A699A42BC
:10CF9000EDD37B683A695A667B68D3F898303B6179
:10CFA00097F90F30012202FA03F35B423A6913400A
:10CFB0003B6197F90F304FF0FF3202FA03F3DA4387
:10CFC0003B6813403A6913433B617B683A69C3F895
:10CFD00098207B689B6D3B613B6803F48073002B5A
:10CFE00004D03B6943F002033B6103E03B6923F05B
:10CFF00002033B613B6803F40073002B04D03B69E0
:10D0000043F001033B6103E03B6923F001033B6113
:10D010007B683A699A6500BF1837BD4680BD00BF7E
:10D02000008003400090034000A0034000900B40AC
:10D03000D45E0100545F01009C5E010080B584B0A5
:10D0400000AF786039603B68002B05D1374B384A18
:10D05000DF21384802F0DCFE3B685B6803F0F00338
:10D06000002B01D101235DE07868FFF76BFE0346DA
:10D07000314A52F82330184607F050F93B681B7BC1
:10D080005B0103F0600343F005027B685A653B686F
:10D090005B6819467868FFF785FE3B689B68194610
:10D0A0007868FFF727FF3B681B7803F007027B686F
:10D0B0001A603B685B789B01DAB23B689B7E5B023F
:10D0C00003F400731A437B68C3F884203B681B7E1B
:10D0D0001A467B68DA653B685B7E1A467B681A678E
:10D0E0003B685A697B68DA663B689B7B9B01DAB2D6
:10D0F0003B681B6903F03F031A437B689A667B68B1
:10D10000DB6FFB60FB6823F47063FB603B685B7B59
:10D110001B0203F47063FA681343FB607B68FA68D0
:10D12000DA67002318461037BD4680BDCC59010090
:10D13000685F01009C5E0100705E010080B58AB0EE
:10D1400000AFF860B96011461A460B46FB711346F2
:10D15000BB71BB68002B06D17C4B7D4A4FF4C1717B
:10D160007C4802F055FE7B6B002B06D17A4B784A47
:10D1700040F28311774802F04BFE3B6B002B06D147
:10D18000764B734A4FF4C271724802F041FEFB794C
:10D19000002B06D1724B6E4A40F285116D4802F0A9
:10D1A00037FEFB686F4A934212D0FB686E4A934287
:10D1B0000ED0FB686D4A93420AD0FB686C4A9342DA
:10D1C00006D06C4B624A40F28711624802F020FEA2
:10D1D000FB681B6803F007037A6B22FA03F37B6199
:10D1E000BB79012B0CD1FB681B6843F02002FB6864
:10D1F0001A603B6B5B007A69B2FBF3F37B620BE076
:10D20000FB681B6823F02002FB681A607A693B6B9D
:10D21000B2FBF3F3013B7B627B6AB3F5803F01D342
:10D22000012335E1FB687A6A9A600023FB7629E1E5
:10D23000BB689B78642B01D9012329E1BB79002BC2
:10D2400002D0BB79012B3FD1BB681B78FA68013350
:10D25000DB0013445B683B613B6923F03C033B61AB
:10D26000BB685B789B003A6913433B613B6943F0C1
:10D2700020033B61BB681B78FA680133DB00134471
:10D280003A695A60BB689B78002B02D100233B624D
:10D2900011E0BB689B781A467B6A03FB02F3364AAF
:10D2A000A2FB03235B093B623A6A7B6A9A4202D380
:10D2B0007B6A01333B62BB681B78FA680133DB0091
:10D2C00013443A6A9A60D7E0BB681B781946FB683A
:10D2D000244A934214D0FB68234A93420ED0FB6841
:10D2E000224A934208D0FB68214A934201D1042389
:10D2F00007E06FF0004304E0012302E0012300E0B7
:10D3000004238B4201D80123C2E0BB68DB78642B85
:10D3100001D90123BCE0BB68DB78002B02D10023DC
:10D32000FB610AE0BB68DB781A467B6A03FB02F309
:10D33000114AA2FB03235B09FB61BB689B78002BAE
:10D340001CD100233B620023FB6129E0E45E010065
:10D35000745F01009C5E0100F85E01000C5F01003B
:10D36000205F0100008003400090034000A00340C4
:10D3700000900B40A85E01001F85EB51BB689B78B5
:10D380001A467B6A03FB02F3434AA2FB03235B09B1
:10D390003B623A6A7B6A9A4202D37B6A01333B6200
:10D3A000BB681B785B00FA680133DB0013445B68E1
:10D3B0003B613B6923F03C033B61BB685B789B00AE
:10D3C0003A6913433B61BB681B785B00FA68013321
:10D3D000DB0013443A695A60BB681B785B00013379
:10D3E000FA680133DB0013445B683B613B6923F05F
:10D3F0003C033B61BB685B789B003A6913433B612C
:10D40000BB681B785B000133FA680133DB0013440F
:10D410003A695A60FB685A6EBB681B78DB000121D1
:10D4200001FA03F31A43FB685A66BB681B785B007A
:10D43000FA680133DB001344FA699A60BB681B7811
:10D440005B000133F9693A6A0A44F9680133DB0089
:10D450000B449A60BB79032B0ED1BB681B78012269
:10D460001946F86806F09DFFBB681978BB681B7900
:10D470001A46F86806F06CFFBB680533BB60FB7E9C
:10D480000133FB76FA7EFB799A42FFF4D1AE00239A
:10D4900018462837BD4680BD1F85EB5180B584B046
:10D4A00000AF78600023FB6009E00E4AFB6852F889
:10D4B00023307A689A4206D0FB680133FB60FB6830
:10D4C000042BF2D900E000BFFB68042B05D9064B02
:10D4D000064A4321064802F09BFCFB6818461037B9
:10D4E000BD4680BD985F0100AC5F0100DC5F0100BC
:10D4F000D05F010080B586B000AFF860B9607A6097
:10D500007B68002B05D1154B154A6421154802F0A4
:10D510007FFC01237B617B681B78002B0AD1FB68B1
:10D520005A697969BB6801FA03F3DB431A40FB6867
:10D530005A610FE07B685B781A46B968F86806F0B4
:10D5400059FFFB685A697969BB6801FA03F31A430A
:10D55000FB685A6100BF1837BD4680BDC459010041
:10D56000F05F0100D05F010080B584B000AF78604B
:10D570007868FFF793FF0346FB73FB7B054A52F87D
:10D580002330BB60BB68D3F8A03018461037BD46C7
:10D5900080BD00BF845F010080B584B000AF7860BB
:10D5A00039607868FFF77AFF0346FB73FB7B064A16
:10D5B00052F82330BB60BB683A68C3F8A02000BFB4
:10D5C0001037BD4680BD00BF845F010080B584B0C8
:10D5D00000AF78600023FB6009E00E4AFB6852F858
:10D5E00023307A689A4206D0FB680133FB60FB68FF
:10D5F000022BF2D900E000BFFB68022B05D9064BD5
:10D60000064A9F21064802F003FCFB6818461037C3
:10D61000BD4680BD8C60010098600100E0600100A3
:10D62000BC60010080B584B000AF786039607B6871
:10D63000DB78FB737B689B78BB73BB7B03F02003B9
:10D64000002B04D1FB7B03F01003002B05D0094B0A
:10D650001B6839687868984704E0074B1B6839688D
:10D6600078689847BFF34F8F00BF00BF1037BD46A3
:10D6700080BD00BFDC2B0020E02B002080B586B0F1
:10D6800000AFF860B9607A60BB68002B06D1354BFB
:10D69000354A40F23621354802F0BAFB7B68002B50
:10D6A00006D1334B304A40F23721304802F0B0FB0C
:10D6B000F868FFF78BFF03462E4A52F823301846CE
:10D6C00006F0B5FEFB6800221A70FB6800225A7053
:10D6D000FB6800229A70FB68FF22DA70FB68002268
:10D6E0005A71FB6850229A71FB680022DA71FB685C
:10D6F0009B78DBB203F07F03DAB2FB689A7045F2E5
:10D700001201F86806F0ADFEBB685B687A681946DE
:10D71000F86800F031F8FB689B79FB75FB7D03F03E
:10D720007F03FB75BB685B78DB01DAB2FB7D1343DB
:10D73000FB75FB7D23F00F03FB75BB681B7A03F0C1
:10D740000F03DAB2FB7D1343FB75FB68FA7D9A7118
:10D75000BB681B78DB01DAB2FB689A7000BF183730
:10D76000BD4680BDC8600100F0600100BC600100E2
:10D77000F85E01008060010080B48DB000AFF860F9
:10D78000B9607A604FF0FF33FB620023BB62002375
:10D790007B620123FB61002387F8233044E0FB6AAE
:10D7A000002B46D097F82330FA6902FA03F3BB61E5
:10D7B000002387F822302CE097F82230274A32F8ED
:10D7C00013301A46BB6903FB02F37A68B2FBF3F32A
:10D7D0007B61BA687B699A4203D9BA687B69D31ABC
:10D7E00002E07A69BB68D31A3B613A69FB6A9A42E4
:10D7F0000AD297F82330BB6297F822307B623B69EC
:10D80000FB623B69002B09D097F82230013387F87F
:10D81000223097F822303F2BCED900E000BF97F896
:10D820002330013387F8233097F82330022BB6D901
:10D8300000E000BFBB6ADBB29B01DAB27B6ADBB2FD
:10D8400003F03F03DBB21343DAB2FB685A7000BF48
:10D850003437BD465DF8047B704700BF00600100AF
:10D8600080B500AF034B1B6819460348FFF7DAFE8B
:10D8700000BF80BDD02B00200060064080B500AF07
:10D88000034B9B6819460348FFF7CCFE00BF80BDE1
:10D89000D02B002000600E4080B584B000AF7860CF
:10D8A0000023FB6006E00D4A7B68934206D0FB68CC
:10D8B0000133FB60FB68002BF5D000E000BFFB6884
:10D8C000002B05D0064B074A3421074802F0A0FA86
:10D8D000FB6818461037BD4680BD00BF006003409E
:10D8E00000610100306101002461010080B584B055
:10D8F00000AF786039603B68002B05D11F4B204A90
:10D900004621204802F084FA7868FFF7C5FF1E4BD5
:10D91000184606F071FE7B681A681C4B1340FB60CA
:10D920003B681B789B0403F440223B685B781B0335
:10D9300003F4E0431A433B68DB781B0203F4706393
:10D940001A433B689B789B0003F00C031343FA686F
:10D950001343FB603B681B79002B03D0FB6843F04B
:10D960000203FB607B68FA681A600121786806F0A0
:10D970005DFE00BF1037BD4680BD00BFC459010029
:10D98000406101002461010016003C10F180F3FFAA
:10D9900080B584B000AF78600023FB6006E00D4ADC
:10D9A0007B68934206D0FB680133FB60FB68002B69
:10D9B000F5D000E000BFFB68002B05D0064B074AFE
:10D9C0003721074802F024FAFB6818461037BD4695
:10D9D00080BD00BF007003404C6101007C6101000C
:10D9E0007061010080B584B000AF786039603B6839
:10D9F000002B05D1204B214A4621214802F008FA8C
:10DA00007868FFF7C5FF1F4B184606F02BFE7B68B2
:10DA10001B6823F002027B681A600023FB7312E08C
:10DA2000FB7B7A681B01134403F584731A68FB7B44
:10DA300022F0070279681B010B4403F584731A6016
:10DA4000FB7B0133FB73FB7B032BE9D93B681B7822
:10DA5000002B06D07B681B6823F001027B681A60EC
:10DA600005E07B681B6843F001027B681A6000BF19
:10DA70001037BD4680BD00BFC45901008C61010054
:10DA80007061010017003C1080B582B000AF786073
:10DA90000A4806F001FE094806F018FE074806F09D
:10DAA000FBFD7B6800221A607B681B6843F0010263
:10DAB0007B681A6000BF0837BD4680BD09003C1076
:10DAC00080B500AF0B4B1B68002B06D10A4B0B4AED
:10DAD00040F63D310A4802F09BF90A4B1B68054AA3
:10DAE0001268114608489847BFF34F8F00BF00BF28
:10DAF00080BD00BFE42B0020C0610100F86101007F
:10DB0000B4610100EC2B002000F0024080B500AFB2
:10DB10000B4B5B68002B06D10A4B0B4A40F6443195
:10DB20000A4802F075F90A4B1B68054A526811460B
:10DB300008489847BFF34F8F00BF00BF80BD00BFAC
:10DB4000E42B0020DC61010014620100B4610100DB
:10DB5000F02B002000F0024080B584B000AF786068
:10DB60000023FB7302E0FB7B0133FB73FB7B002B89
:10DB700003D1094A7B689342F5D1FB7B002B05D08A
:10DB8000064B074AE421074802F042F9FB7B18469E
:10DB90001037BD4680BD00BF00100B403062010051
:10DBA000546401005462010080B586B000AF786013
:10DBB00039603B68002B06D12C4B2D4A40F24B11AB
:10DBC0002C4802F025F97B681B697B617B685B69E7
:10DBD0003B617B689B69FB603B685B7A002B21D0D3
:10DBE0003B687A69DA603B685B7A032B1AD13B6841
:10DBF000DB681A023B68DA603B691A027B691B0E1C
:10DC00001A433B681A61FB681A023B691B0E1A43F0
:10DC10003B685A617B68DB691A02FB681B0E1A437A
:10DC20003B689A613B68DB69002B19D03B685B7AE3
:10DC3000012B0BD03B685B7A022B07D03B685B7AE9
:10DC4000082B03D03B685B7A062B09D13B68DA6965
:10DC50003B68DB681340002B02D040F2A66300E073
:10DC6000002318461837BD4680BD00BF6062010022
:10DC7000686401005462010080B586B000AF78602E
:10DC8000396000237B6100233B613B685B6803F0E4
:10DC90000303002B06D03B685B6823F003031A1DC7
:10DCA0003B685A603B689B683A68526802FB03F322
:10DCB0009B08FB6026E000BF786806F0ACFD0246DA
:10DCC000184B1340002BF7D0786806F0A4FD0346EC
:10DCD00003F0B873002B08D03B685B7883F0010336
:10DCE000DBB2002B01D001233B613B69002B05D146
:10DCF0007A693968786806F07AFE78610949786847
:10DD000006F095FD3B69002B03D17A69FB689A42C6
:10DD1000D1D30549786806F08AFD3B691846183763
:10DD2000BD4680BD200070010200700180B586B044
:10DD300000AF7860396000237B6100233B613B6862
:10DD40005B6803F00303002B06D03B685B6823F09D
:10DD500003031A1D3B685A603B689B683A68526827
:10DD600002FB03F39B08FB6026E000BF786806F027
:10DD700052FD0246254B1340002BF7D0786806F081
:10DD80004AFD034603F0B873002B08D03B685B786C
:10DD900083F00103DBB2002B01D001233B613B691F
:10DDA000002B05D17A693968786806F072FE7861CF
:10DDB0001649786806F03BFD3B69002B03D17A6970
:10DDC000FB689A42D1D300BF786806F024FD024672
:10DDD0000F4B1340002BF7D0786806F01CFD03466C
:10DDE00003F0B873002B08D03B685B7883F0010325
:10DDF000DBB2002B01D001233B610549786806F0B6
:10DE000016FD3B6918461837BD4680BD10007001ED
:10DE10000200700180B584B000AF786039600023E3
:10DE2000FB6000BF786806F0F6FC02460F4B13401B
:10DE3000002BF7D0786806F0EEFC034603F470235D
:10DE4000002B01D00123FB60FB68002B04D1396853
:10DE50007868FFF7A9FEF8600449786806F0E7FCE7
:10DE6000FB6818461037BD4680BD00BF01000F009B
:10DE700080B584B000AF786039600023FB6000BFDC
:10DE8000786806F0C8FC02460E4B1340002BF7D012
:10DE9000786806F0C0FC02460B4B1340002B08D0FC
:10DEA0003B685B7883F00103DBB2002B01D00123D8
:10DEB000FB600649786806F0BAFCFB681846103724
:10DEC000BD4680BD02007011000070110A00701183
:10DED00080B584B000AF786039603B68002B06D114
:10DEE000494B4A4A40F22A31494801F091FF3B68C8
:10DEF0009B78012B06D1474B444A4FF44B71444861
:10DF000001F086FF3B689B68002B03D03B689B6851
:10DF1000802B06D9404B3D4A40F22E313C4801F05F
:10DF200077FF3B685B68002B03D03B685B68802B06
:10DF300006D93A4B354A40F22F31354801F068FF97
:10DF40007868FFF709FE364B184606F04AFC7B68F6
:10DF5000DB6A43F0E0627B68DA627B689B6AFB60A5
:10DF60007B685B6CBB60FB6823F44E73FB603B68B3
:10DF70001B78002B03D0FB6843F00803FB603B6871
:10DF80005B781B0103F030023B689B781B0203F4B3
:10DF900040731343FA681343FB60BB6803F0FF232D
:10DFA000BB603B685B68DAB23B689B681B0403F4A8
:10DFB0007F031343BA681343BB607B68BA685A6433
:10DFC0007B68FA689A627B68DB6A43F007027B68C9
:10DFD000DA627B68134A5A637B6800229A637B6823
:10DFE000104A1A637B68DB6A43F000627B68DA627E
:10DFF00000BF7B68DB6A03F00063002BF9D100BF30
:10E0000000BF1037BD4680BD345D0100846401004F
:10E01000546201007062010098620100E862010030
:10E020001100301037017F1180B58AB000AFF86061
:10E03000B9607A60BB68002B06D15C4B5C4A40F249
:10E04000B3315C4801F0E4FE7B68002B03D07A68B2
:10E05000BB689A4206D9584B554A4FF46D715548E2
:10E0600001F0D6FE00237B6200233B620023FB61AC
:10E0700000237B610023BB61BA687B68B2FBF3F3CA
:10E080007B627B6AB3F5805F01D900238AE07B6AFB
:10E09000002B49D0BA687B6AB2FBF3F37A689A42E4
:10E0A00002D27B6A01337B627B6A102B32D97B6A96
:10E0B0001B09FB6102E0FB690133FB614FF48073D4
:10E0C000FA69B3FBF2F2F96901FB02F29B1A002B29
:10E0D000F1D1FB69012BEED07A6AFB69B2FBF3F355
:10E0E0003B6202E03B6A01333B623B6AFA6902FB36
:10E0F00003F37A6A9A42F5D83B6A002B01D03B6A57
:10E1000000E00123BA68B2FBF3F2FB69B2FBF3F360
:10E11000BB610FE07B6A3B620023FB61BA683B6A2C
:10E12000B2FBF3F3BB6105E000233B620023FB611C
:10E13000BB68BB613B6A002B02D03B6A013B3B6280
:10E14000FB69002B02D0FB695B08FB61FB68DB6AA3
:10E1500023F00802FB68DA62FB68DB6A7B617B699B
:10E1600023F47F2323F47F637B613B6A1B01DAB2D4
:10E17000FB691B029BB21A437B69134343F4602380
:10E180007B61FB687A69DA6200BFFB685B6A03F057
:10E190000803002BF9D0FB68DB6A43F00802FB6838
:10E1A000DA62BB6918462837BD4680BD3863010076
:10E1B00090640100546201004C63010080B582B09C
:10E1C00000AF786039603B68002B06D1204B214AB4
:10E1D00040F23F41204801F01BFE3B681B68B3F54D
:10E1E000005F06D31D4B1B4A4FF488611A4801F0AB
:10E1F0000FFE3B685B68B3F5803F06D3184B154AAA
:10E2000040F24141144801F003FE7B685B6803F46F
:10E2100060423B681B68C3F30C013B685B681B04EE
:10E220000B431A437B685A603B689A687B689A6024
:10E230003B68DB681B0603F07C523B681969094B9D
:10E240000B401A437B68DA6000BF0837BD4680BDCB
:10E25000345D0100A064010054620100806301008C
:10E26000D46301003700FB0080B48BB000AFF860CE
:10E270007A603B600B46FB7200237B623B6B3B6228
:10E280007B68002B02D03B68002B05D1FB7A012B69
:10E290000BD0FB7A022B08D03B6B002B05D07B6B9D
:10E2A000002B02D0FB7A012B02D104237B627FE09A
:10E2B000FB7A022B08D13B6A03F00303002B03D047
:10E2C0004FF4D5637B6273E0FB7A022B70D17B6BDA
:10E2D00003F00303002B04D07B6B23F00303043310
:10E2E0007B637B6B364AA2FB0323DB0B0133BB61F1
:10E2F0003B689B00DB08BA699A4202D903237B6220
:10E3000056E07B687B610023FB6147E03A6A3B6B28
:10E31000D31A9B007A6BD31AB3F5803F1ED2FB69E8
:10E32000DB007A6913443A6A5A603A6A3B6BD31A43
:10E330009B007A6BD21AFB69DB0079690B441204EB
:10E340001A60FB69DB007A6913441A68FB69DB0019
:10E3500079690B4442F023021A601CE0FB69DB0080
:10E360007A6913443A6A5A60FB69DB007A6913449C
:10E37000144A1A60FB69DB007A6913441A68FB6966
:10E38000DB0079690B4442F021021A603B6A03F515
:10E390007F43FC333B62FB690133FB61FA69BB6974
:10E3A0009A42B3D3FB6800221A607A68FB689A65C8
:10E3B0007B6A18462C37BD465DF8047B704700BF6A
:10E3C000018000800000FCFF80B58AB002AFF860D9
:10E3D000B9607A603B603B68002B06D13E4B3F4AF8
:10E3E00040F26E513E4801F013FD0023BB61FB6813
:10E3F0009B6A1B0A03F00303FB773B685B687B6146
:10E400003B681B683B617B69002B07D03B69002B95
:10E4100006D03B699B68B3F5803F01D3042356E0E7
:10E4200000BFF86806F011FA034603F00103002B61
:10E43000F7D13B69002B07D0F86806F006FA0346CF
:10E4400003F00203002BF4D13B69002B1FD0BB6803
:10E45000002B1CD03B69DB68002B02D03B69DB68DA
:10E4600001E03B691B693A6992683969496801FBB7
:10E4700002F2F97F019200937B68BA68F868FFF7AF
:10E48000F3FEB861BB69002B01D00023FB77FB7F53
:10E490003A697969F86806F0FEF97969F868FFF772
:10E4A000B9FCB861BB69002B01D0BB690FE03B69C7
:10E4B000002B0BD0FB7F3A69F968184606F060FB29
:10E4C000B861BB69002B01D0BB6900E0002318468E
:10E4D0002037BD4680BD00BF28640100B86401003C
:10E4E0005462010080B500AF0B4B1B68002B06D1B6
:10E4F0000A4B0B4A40F24B610A4801F089FC0A4B77
:10E500001B68054A1268114608489847BFF34F8FA9
:10E5100000BF00BF80BD00BFF42B00203C640100A1
:10E52000D064010054620100F82B002000100B4061
:10E5300080B500AF054B1B68054A126811460548B7
:10E540009847BFF34F8F00BF00BF80BD142C002041
:10E55000FC2B002000A0064080B500AF054B1B68D7
:10E56000054A5268114605489847BFF34F8F00BFD0
:10E5700000BF80BD142C0020FC2B002000B0064002
:10E5800080B500AF054B1B68054A926811460548E7
:10E590009847BFF34F8F00BF00BF80BD142C0020F1
:10E5A000FC2B002000C0064080B500AF054B1B6867
:10E5B000054AD268114605489847BFF34F8F00BF00
:10E5C00000BF80BD142C0020FC2B002000D0064092
:10E5D00080B500AF054B1B68054A12691146054816
:10E5E0009847BFF34F8F00BF00BF80BD142C0020A1
:10E5F000FC2B002000A00E4080B500AF054B1B682F
:10E60000054A5269114605489847BFF34F8F00BF2E
:10E6100000BF80BD142C0020FC2B002000B00E4059
:10E6200080B500AF0B4BD3F888300A4A43F470032F
:10E63000C2F88830084B4CF22052DA81064B4DF676
:10E640002812DA81044B4FF4E9721A8006F042FB7B
:10E6500000BF80BD00ED00E00020054080B483B025
:10E6600000AF78600B4B03F5805304331B6823F035
:10E6700040527B681B0703F0405306491A4301F5DB
:10E68000805304331A6000BF0C37BD465DF8047B2D
:10E69000704700BF0070044080B400AF054B03F525
:10E6A000825304334FF092721A6000BFBD465DF88A
:10E6B000047B70470070044080B483B000AF786082
:10E6C000044A7B68136000BF0C37BD465DF8047BCD
:10E6D000704700BF582B002080B483B000AF0346C2
:10E6E000FB710B4B1B78DBB223F03803DAB2FB79FA
:10E6F000DB00DBB203F03803DBB205491343DBB2C6
:10E700000B7000BF0C37BD465DF8047B704700BF3F
:10E710000040064080B500AFFFF7BEFF1048FDF790
:10E7200019FD104B1846FFF7C7FF00231846FFF7E7
:10E73000D3FF00230C4A00211846FDF7ADFD0B481E
:10E74000FDF712FB0A4B0B4A1A600B494FF4E0200D
:10E75000FDF726FB0120FFF781FF00BF80BD00BF52
:10E76000FC6401000024F400F0640100F464010082
:10E770000C010020000E2707006CDC0280B483B07F
:10E7800000AF0346FB7197F90730002B0BDBFB79D9
:10E7900003F01F02074997F907305B09012000FACF
:10E7A00002F241F8232000BF0C37BD465DF8047B20
:10E7B000704700BF00E100E080B483B000AF0346C3
:10E7C0003960FB7197F90730002B0ADB3B68DAB23E
:10E7D0000C4997F907301201D2B20B4483F8002399
:10E7E0000AE03B68DAB20849FB7903F00F03043B07
:10E7F0001201D2B20B441A7600BF0C37BD465DF849
:10E80000047B704700E100E000ED00E080B582B0DD
:10E8100000AF786039603B680F2B06D9084B094A76
:10E8200040F28621084801F0F3FA3B68DBB203F0BE
:10E830000F03DAB27B68DA7600BF0837BD4680BDC9
:10E8400004650100C06701003C65010080B582B02D
:10E8500000AF786039603B680F2B05D90B4B0C4A31
:10E860004D210C4801F0D4FA7A683B6813441B78B8
:10E87000DBB263F07F03D9B27A683B6813440A467F
:10E880001A7000BF0837BD4680BD00BF0465010097
:10E89000A86701009865010080B584B000AFF860FA
:10E8A000B9607A60BB680F2B05D90F4B0F4A6B21FB
:10E8B0000F4801F0ADFAFA68BB6813441B78DBB26D
:10E8C00023F03F03DAB27B68DBB203F03F03DBB235
:10E8D0001343D9B2FA68BB6813440A461A7000BFE2
:10E8E0001037BD4680BD00BF04650100946701007C
:10E8F0009865010080B584B000AFF8600B467A607F
:10E90000FB72FB7A012B06D9164B174A40F2D9113C
:10E91000164801F07DFA7B68002B06D1144B124A91
:10E920004FF4ED71114801F073FA7B689B681B048A
:10E9300003F47F027B685B681B029BB242EA03011F
:10E940007B681B68DBB2FA7A1943F86813469B00B0
:10E950001344DB0003441033196000BF1037BD4679
:10E9600080BD00BFF8650100DC670100346601006E
:10E97000C459010090B585B000AFF8607B600B46CC
:10E98000FB721346BB72FB7A012B06D9104B114A5E
:10E990004FF4F871104801F03BFABB7A012B06D90D
:10E9A0000E4B0C4A40F2F1110B4801F031FAFA7AA1
:10E9B000BC7A7B6898B2F96813469B0013445B00ED
:10E9C0002344063341F8230000BF1437BD4690BDF1
:10E9D000F8650100F86701003466010090660100E7
:10E9E00080B500AF4FF4807200212548FFF754FF37
:10E9F00000212348FFF72AFF00212248FDF7C2FE2D
:10EA0000214A00211F48FDF7BBFD4FF494720121FC
:10EA10001B48FFF741FF01211948FFF717FF0121AC
:10EA20001848FDF7AFFE194A01211648FDF7A8FD69
:10EA300040F2291202211248FFF72EFF022110484E
:10EA4000FFF704FF02210F48FDF79CFE0221022080
:10EA5000FFF7B2FE022006F04AF90D4A02210948EA
:10EA6000FDF78EFD00210748FFF7D0FE0121054884
:10EA7000FFF7CCFE02210348FFF7C8FE00BF80BDB0
:10EA80000010024000800040000000202000002014
:10EA90004000002080B500AF0F491048FCF7FEFD94
:10EAA00001210E4806F055F9032319460B4805F0DD
:10EAB00013FB00231946094805F0F2FA074805F050
:10EAC00057FA0121054806F028F9054A00210348B4
:10EAD000FCF772FE00BF80BDE466010000B0034099
:10EAE0001001002080B500AF0F491048FCF7D6FD9B
:10EAF00001210E4806F02DF9032319460B4805F0B5
:10EB0000EBFA00231946094805F0CAFA074805F050
:10EB10002FFA0121054806F000F9054A00210348B3
:10EB2000FCF74AFE00BF80BDF066010000B00B405C
:10EB30001801002080B582B002AF0C490C48FEF7E6
:10EB40007DFA0220FDF76CF80346019343F6381373
:10EB500000930023032207490548FEF7EFFA01213D
:10EB6000034806F012F900BFBD4680BDFC660100F7
:10EB7000008003401867010080B582B002AF0C49E5
:10EB80000C48FEF75BFA0220FDF74AF803460193B2
:10EB900043F6381300930023012207490548FEF786
:10EBA000CDFA0121034806F0F0F800BFBD4680BD54
:10EBB00028670100009003404467010080B582B0DF
:10EBC00002AF0C490C48FEF739FA0220FDF728F88D
:10EBD0000346019343F638130093002304220749A8
:10EBE0000548FEF7ABFA0121034806F0CEF800BF56
:10EBF000BD4680BD4C67010000900B406867010076
:10EC000080B500AF084A09490948FEF737FD4021A1
:10EC1000074805F053FC00211920FFF7CDFD19200E
:10EC200006F065F800BF80BD008793037C67010094
:10EC30000070064080B500AF11491248FEF756FE3D
:10EC400040F26C710F4806F0CDF80F4A00210D48D4
:10EC5000FFF750FE0123002200210A48FFF78AFE39
:10EC60000A4A01210748FFF745FE0123002201213E
:10EC70000448FFF77FFE034806F0A4F800BF80BDFC
:10EC80008867010000600340200100202C01002063
:10EC900080B500AF1C491D48FEF7A4FE41F26F721B
:10ECA00000211A4806F0CAF8194A0121174806F04F
:10ECB000C5F8184A0221154806F0C0F802220021C2
:10ECC000124806F09EF802220121104806F099F839
:10ECD000022202210D4806F094F801213020FFF7AE
:10ECE0006BFD02213120FFF767FD02213220FFF783
:10ECF00063FD302005F0FBFF312005F0F8FF3220E6
:10ED000005F0F5FF00BF80BD906701000070034073
:10ED1000BF270900DF93040080B500AF0248FEF76B
:10ED2000B3FE00BF80BD00BF0090024080B500AFC1
:10ED30000E48FDF767FB0E490E48FDF7D1FCFFF7C3
:10ED40004FFEFFF7A7FEFFF7CDFEFFF7F3FEFFF73D
:10ED500013FFFFF733FFFFF76DFFFFF799FFFFF793
:10ED6000DBFF06F07FF800BF80BD00BF001002404F
:10ED7000E06601000080004080B598B000AFDC483C
:10ED800006F087F8DB4806F084F8DB4806F081F8E7
:10ED9000DA4806F07EF8DA4806F07BF8002387F8B8
:10EDA0005C30002387F85D3007F15C031A460D21C3
:10EDB000D448FEF79FFB002387F85830002387F8DC
:10EDC000593007F158031A460E21CE48FEF792FB40
:10EDD000002387F85430002387F8553007F1540397
:10EDE0001A460F21C748FEF785FB002387F85030ED
:10EDF000002387F8513007F150031A461021C1480B
:10EE0000FEF778FB002387F84C30002387F84D305D
:10EE100007F14C031A461121BA48FEF76BFB012398
:10EE200087F84830002387F8493007F148031A462D
:10EE30000021B548FEF75EFB012387F8443000232C
:10EE400087F8453007F144031A460121AE48FEF722
:10EE500051FB012387F84030002387F8413007F148
:10EE600040031A460221A848FEF744FB012387F815
:10EE70003C30002387F83D3007F13C031A4603215C
:10EE8000A148FEF737FBA14B1B883B8707F13803EE
:10EE90001A460A219C48FEF72DFB9C4B1B88BB861B
:10EEA00007F134031A460B219748FEF723FB012391
:10EEB00087F83030002387F8313007F130031A46E5
:10EEC00010219148FEF716FB012387F82C30002310
:10EED00087F82D3007F12C031A4611218A48FEF7D6
:10EEE00009FB012387F82830002387F8293007F130
:10EEF00028031A4612218448FEF7FCFA012387F8FA
:10EF00002430002387F8253007F124031A46132103
:10EF10007D48FEF7EFFA012387F82030002387F8B9
:10EF2000213007F120031A4601217948FEF7E2FA61
:10EF300001233B7700237B7707F11C031A4602214C
:10EF40007348FEF7D7FA01233B7600237B7607F15F
:10EF500018031A4605216E48FEF7CCFA01233B75CB
:10EF600000237B7507F114031A4606216848FEF753
:10EF7000C1FA01233B7400237B7407F110031A4686
:10EF800007216348FEF7B6FA01233B7300237B7326
:10EF900007F10C031A4608215D48FEF7ABFA01237E
:10EFA0003B7200237B7207F108031A46052159487A
:10EFB000FEF7A0FA01233B7100237B713B1D1A462B
:10EFC00006215448FEF796FA00233B7000237B701D
:10EFD0003B461A461A215048FEF78CFA03220C21B0
:10EFE0004E4805F070FF01220D214C4805F06BFFE3
:10EFF0000B220D21494805F083FF01220E214748CD
:10F0000005F061FF0B220E21444805F079FF012233
:10F010000F21424805F057FF0B220F213F4805F012
:10F020006FFF012210213D4805F04DFF0B221021FA
:10F030003A4805F065FF01221121384805F043FFE9
:10F040000B221121354805F05BFF344B5B6C23F03C
:10F05000807323F00303314A43F003035364012216
:10F0600000212F4805F02FFF012201212C4805F037
:10F070002AFF01220A212A4805F025FF01220B213F
:10F08000274805F020FF01221021254805F01BFF2D
:10F0900001221121224805F016FF012212212048E9
:10F0A00005F011FF012213211D4805F00CFF01227C
:10F0B00002211B4805F007FF01220321184805F033
:10F0C00002FF01220121174805F0FDFE02220A215C
:10F0D000144805F0F8FE134B9B6A23F0807323F06D
:10F0E0006303104A43F06103936202220B211BE089
:10F0F000090038100A0038100B0038100C003810C6
:10F100000D00381000F00F4040F00F40186801006B
:10F1100080F00F40C0F00F4000F10F40009004401D
:10F1200000A0044000B00440684805F0CCFE674BE6
:10F13000DB6A23F0807323F06303644A43F06103C6
:10F14000D36201220221614805F0BDFE04220321A1
:10F150005E4805F0B8FE012205215C4805F0B3FECB
:10F1600001220621594805F0AEFE01220721574829
:10F1700005F0A9FE01220821544805F0A4FE04224E
:10F180000021534805F09FFE04220121504805F05C
:10F190009AFE042202214E4805F095FE0422032126
:10F1A0004B4805F090FE04220421494805F08BFEEF
:10F1B00001220521464805F086FE01220621444829
:10F1C00005F081FE04220721414805F07CFE04225F
:10F1D0000021404805F077FE3E4B1B6823F080730A
:10F1E00023F043033B4A43F043031360042201210D
:10F1F000384805F068FE374B5B6823F0807323F0D6
:10F200004303344A43F0430353600422022131484C
:10F2100005F059FE2F4B9B6823F0807323F04303C6
:10F220002C4A43F04103936001221921294805F03B
:10F230004AFE01221A21274805F045FE254B9B6E08
:10F2400023F0807323F00303224A43F00203936602
:10F25000042203211F4805F036FE1E4BDB6823F015
:10F26000807323F043031B4A43F04303D36004221B
:10F270000421184805F027FE164B1B6923F0807304
:10F2800023F04303134A43F043031361042205218F
:10F29000104805F018FE0F4B5B6923F0807323F0D4
:10F2A00043030C4A43F0430353610B4B03F5805374
:10F2B0000C331B68084923F4402201F580530C33BA
:10F2C0001A6000BF6037BD4680BD00BF00B004407B
:10F2D00000C0044000D004400070044081F00041B0
:10F2E00002E000BF83F0004330B54FEA41044FEA2B
:10F2F000430594EA050F08BF90EA020F1FBF54EAC6
:10F30000000C55EA020C7FEA645C7FEA655C00F061
:10F31000E2804FEA5454D4EB5555B8BF6D420CDD32
:10F320002C4480EA020281EA030382EA000083EAB5
:10F33000010180EA020281EA0303362D88BF30BD55
:10F3400011F0004F4FEA01314FF4801C4CEA1131AB
:10F3500002D0404261EB410113F0004F4FEA03330A
:10F360004CEA133302D0524263EB430394EA050F95
:10F3700000F0A780A4F10104D5F1200E0DDB02FA04
:10F380000EFC22FA05F2801841F1000103FA0EF298
:10F39000801843FA05F359410EE0A5F120050EF15E
:10F3A000200E012A03FA0EFC28BF4CF0020C43FA8F
:10F3B00005F3C01851EBE37101F0004507D54FF09C
:10F3C000000EDCF1000C7EEB00006EEB0101B1F5EC
:10F3D000801F1BD3B1F5001F0CD349085FEA300032
:10F3E0004FEA3C0C04F101044FEA445212F5800F3D
:10F3F00080F09A80BCF1004F08BF5FEA500C50F1DA
:10F40000000041EB045141EA050130BD5FEA4C0CBC
:10F41000404141EB0101013C28BFB1F5801FE9D219
:10F4200091F0000F04BF01460020B1FA81F308BF3C
:10F430002033A3F10B03B3F120020CDA0C3208DD08
:10F4400002F1140CC2F10C0201FA0CF021FA02F1E3
:10F450000CE002F11402D8BFC2F1200C01FA02F153
:10F4600020FA0CFCDCBF41EA0C019040E41AA2BF78
:10F4700001EB0451294330BD6FEA04041F3C1CDA40
:10F480000C340EDC04F11404C4F1200220FA04F060
:10F4900001FA02F340EA030021FA04F345EA03010A
:10F4A00030BDC4F10C04C4F1200220FA02F001FACC
:10F4B00004F340EA0300294630BD21FA04F029464E
:10F4C00030BD94F0000F83F4801306BF81F48011E7
:10F4D0000134013D4EE77FEA645C18BF7FEA655C5A
:10F4E00029D094EA050F08BF90EA020F05D054EA2C
:10F4F000000C04BF1946104630BD91EA030F1EBF31
:10F500000021002030BD5FEA545C05D14000494134
:10F5100028BF41F0004130BD14F580043CBF01F527
:10F52000801130BD01F0004545F0FE4141F470010D
:10F530004FF0000030BD7FEA645C1ABF19461046E8
:10F540007FEA655C1CBF0B46024650EA013406BFE9
:10F5500052EA033591EA030F41F4002130BD00BFA8
:10F5600090F0000F04BF0021704730B54FF4806465
:10F5700004F132044FF000054FF0000150E700BFE6
:10F5800090F0000F04BF0021704730B54FF4806445
:10F5900004F1320410F0004548BF40424FF0000132
:10F5A0003EE700BF42004FEAE2014FEA31014FEA75
:10F5B00002701FBF12F07F4393F07F4F81F06051C4
:10F5C000704732F07F4208BF704793F07F4F04BF0F
:10F5D00041F40021704730B54FF4607401F00045EC
:10F5E00021F000411CE700BF50EA010208BF70474C
:10F5F00030B54FF000050AE050EA010208BF70473D
:10F6000030B511F0004502D5404261EB41014FF4A5
:10F61000806404F132045FEA915C3FF4D8AE4FF0AD
:10F6200003025FEADC0C18BF03325FEADC0C18BF90
:10F63000033202EBDC02C2F1200300FA03FC20FAE1
:10F6400002F001FA03FE40EA0E0021FA02F114442E
:10F65000BDE600BF70B54FF0FF0C4CF4E06C1CEA47
:10F6600011541DBF1CEA135594EA0C0F95EA0C0FB8
:10F6700000F0DEF82C4481EA030621EA4C5123EA2B
:10F680004C5350EA013518BF52EA033541F480115A
:10F6900043F4801338D0A0FB02CE4FF00005E1FB0D
:10F6A00002E506F00042E0FB03E54FF00006E1FB57
:10F6B00003569CF0000F18BF4EF0010EA4F1FF049A
:10F6C000B6F5007F64F5407404D25FEA4E0E6D41DA
:10F6D00046EB060642EAC62141EA55514FEAC520EB
:10F6E00040EA5E504FEACE2EB4F1FD0C88BFBCF567
:10F6F000E06F1ED8BEF1004F08BF5FEA500E50F118
:10F70000000041EB045170BD06F0004646EA0101DD
:10F7100040EA020081EA0301B4EB5C04C2BFD4EB0F
:10F720000C0541EA045170BD41F480114FF0000E08
:10F73000013C00F3AB8014F1360FDEBF002001F076
:10F74000004170BDC4F10004203C35DA0C341BDCF0
:10F7500004F11404C4F1200500FA05F320FA04F0C2
:10F7600001FA05F240EA020001F0004221F00041F6
:10F7700010EBD37021FA04F642EB06015EEA430E69
:10F7800008BF20EAD37070BDC4F10C04C4F1200599
:10F7900000FA04F320FA05F001FA04F240EA02004C
:10F7A00001F0004110EBD37041F100015EEA430E1D
:10F7B00008BF20EAD37070BDC4F1200500FA05F23D
:10F7C0004EEA020E20FA04F301FA05F243EA0203BC
:10F7D00021FA04F001F0004121FA04F220EA0200CB
:10F7E00000EBD3705EEA430E08BF20EAD37070BD11
:10F7F00094F0000F0FD101F00046400041EB0101F1
:10F8000011F4801F08BF013CF7D041EA060195F0D2
:10F81000000F18BF704703F00046520043EB03038C
:10F8200013F4801F08BF013DF7D043EA0603704779
:10F8300094EA0C0F0CEA135518BF95EA0C0F0CD084
:10F8400050EA410618BF52EA4306D1D181EA0301CA
:10F8500001F000414FF0000070BD50EA410606BFC4
:10F860001046194652EA430619D094EA0C0F02D109
:10F8700050EA013613D195EA0C0F05D152EA03364E
:10F880001CBF104619460AD181EA030101F000416C
:10F8900041F0FE4141F470014FF0000070BD41F0B5
:10F8A000FE4141F4780170BD70B54FF0FF0C4CF48F
:10F8B000E06C1CEA11541DBF1CEA135594EA0C0FAE
:10F8C00095EA0C0F00F0A7F8A4EB050481EA030EFB
:10F8D00052EA03354FEA013100F088804FEA0333E2
:10F8E0004FF0805545EA131343EA12634FEA0222B0
:10F8F00045EA111545EA10654FEA00260EF0004171
:10F900009D4208BF964244F1FD0404F5407402D2C2
:10F910005B084FEA3202B61A65EB03055B084FEA53
:10F9200032024FF480104FF4002CB6EB020E75EB50
:10F93000030E22BFB61A754640EA0C005B084FEA78
:10F940003202B6EB020E75EB030E22BFB61A7546F5
:10F9500040EA5C005B084FEA3202B6EB020E75EB40
:10F96000030E22BFB61A754640EA9C005B084FEAB8
:10F970003202B6EB020E75EB030E22BFB61A7546C5
:10F9800040EADC0055EA060E18D04FEA051545EAB4
:10F9900016754FEA06164FEAC30343EA52734FEA5D
:10F9A000C2025FEA1C1CC0D111F4801F0BD141EAD6
:10F9B00000014FF000004FF0004CB6E711F4801F3B
:10F9C00004BF01430020B4F1FD0C88BFBCF5E06F1B
:10F9D0003FF6AFAEB5EB030C04BFB6EB020C5FEA2B
:10F9E000500C50F1000041EB045170BD0EF0004E80
:10F9F0004EEA113114EB5C04C2BFD4EB0C0541EAB2
:10FA0000045170BD41F480114FF0000E013C90E6AE
:10FA100045EA060E8DE60CEA135594EA0C0F08BF72
:10FA200095EA0C0F3FF43BAF94EA0C0F0AD150EA71
:10FA300001347FF434AF95EA0C0F7FF425AF104604
:10FA400019462CE795EA0C0F06D152EA03353FF42C
:10FA5000FDAE1046194622E750EA410618BF52EAA9
:10FA600043067FF4C5AE50EA41047FF40DAF52EA7D
:10FA700043057FF4EBAE12E74FEA4102B2F1E043F7
:10FA800024BFB3F5001CDCF1FE5C0DD901F0004C85
:10FA90004FEAC0024CEA5070B2F1004F40EB8300D5
:10FAA00008BF20F00100704711F0804F21D113F101
:10FAB0003872BCBF01F00040704741F480114FEA3A
:10FAC0005252C2F11802C2F1200C10FA0CF320FAC3
:10FAD00002F018BF40F001004FEAC1234FEAD323E0
:10FAE00003FA0CFC40EA0C0023FA02F34FEA43034A
:10FAF000CCE77FEA625307D150EA01331EBF4FF0D3
:10FB0000FE4040F44000704701F0004040F0FE40ED
:10FB100040F40000704700BF53B94AB9002908BF3C
:10FB200000281CBF4FF0FF314FF0FF3000F06EB9DE
:10FB3000ADF1080C6DE904CE00F006F8DDF804E044
:10FB4000DDE9022304B070472DE9F047089D044623
:10FB50008C46002B40F083808A42174647D9B2FA80
:10FB600082F242B1C2F1200024FA00F091409740A5
:10FB700040EA010C94404FEA1748230CBCFBF8F60E
:10FB80001FFA87FE08FB16C143EA014306FB0EF18C
:10FB9000994209D9FB1806F1FF3080F0198199428A
:10FBA00040F21681023E3B445B1AA4B2B3FBF8F06C
:10FBB00008FB103344EA034400FB0EFEA64509D9B6
:10FBC0003C1900F1FF3380F00581A64540F2028127
:10FBD00002383C4440EA0640A4EB0E0400261DB166
:10FBE000D4400023C5E900433146BDE8F08702B99F
:10FBF000FFDEB2FA82F2002A50D1CB1B4FEA174E39
:10FC00001FFA87F80126B3FBFEFC210C0EFB1C3308
:10FC100041EA034108FB0CF38B4207D979180CF138
:10FC2000FF3002D28B4200F2E9808446C91AA3B2A7
:10FC3000B1FBFEF00EFB101143EA014408FB00F893
:10FC4000A04507D93C1900F1FF3302D2A04500F2CC
:10FC5000D9801846A4EB080440EA0C40BFE78B4269
:10FC600009D9002D00F0B1800026C5E90001304619
:10FC70003146BDE8F087B3FA83F6002E4AD18B42B5
:10FC800002D3824200F2B880841A61EB03010120A2
:10FC90008C46002DA8D0C5E9004CA5E7C2F1200391
:10FCA00020FA03F6974001FA02F04FEA174ED940C6
:10FCB0003043030CB1FBFEF61FFA87F80EFB16115A
:10FCC00043EA014306FB08F1994204FA02F409D918
:10FCD000FB1806F1FF3C80F08D80994240F28A804B
:10FCE000023E3B445B1A81B2B3FBFEF00EFB1033C5
:10FCF00041EA034100FB08F38B4207D9791800F170
:10FD0000FF3C73D28B4271D902383944CB1A40EA96
:10FD1000064678E7C6F1200C03FA06F422FA0CF343
:10FD20001C4320FA0CF701FA06F34FEA144E21FAAD
:10FD30000CF11F433B0CB1FBFEF91FFA84F80EFBDC
:10FD4000191143EA014109FB08FA8A4502FA06F251
:10FD500000FA06F308D9611809F1FF3048D28A4544
:10FD600046D9A9F102092144A1EB0A01BFB2B1FBB6
:10FD7000FEF00EFB101147EA014700FB08F8B845FA
:10FD800007D9E71900F1FF312ED2B8452CD9023836
:10FD9000274440EA0940A7EB0807A0FB02894F452A
:10FDA000C64649461AD317D05DB1B3EB0E0267EBD6
:10FDB000010707FA0CFCF2404CEA0202F740C5E9E1
:10FDC000002700263146BDE8F0872E4628460BE77F
:10FDD0000646E9E61846FDE64345E5D2B8EB020ED5
:10FDE00069EB04010138DFE70846D2E760468DE79A
:10FDF0008146B9E7664675E730464AE7ACF1020C42
:10FE0000394413E702383C4424E700BF704700BF81
:10FE10001FB514461A46094B1B680546D8684CB1F5
:10FE2000074B0091CDE9013406492B4600F00EF84E
:10FE300005F047F9044B1C46F3E700BF38010020EA
:10FE4000B0680100BD680100EB6801000EB403B5A5
:10FE5000014603AB054853F8042B0068019300F0FA
:10FE6000D5F802B05DF804EB03B07047380100200C
:10FE700070B50D4D0D4C641BA4100026A64209D18F
:10FE80000B4D0C4C06F050FD641BA4100026A6423E
:10FE900005D170BD55F8043B98470136EEE755F89B
:10FEA000043B98470136F2E73869010038690100E0
:10FEB000386901004069010037B5002948D051F880
:10FEC000043C0190002BA1F10404B8BFE41800F039
:10FED00085FD204A01981368154633B963601460A4
:10FEE00003B0BDE8304000F07FBDA3420BD92168CC
:10FEF0006218934204BF1A685B68636004BF5218BB
:10FF000022602C60ECE71A465B680BB1A342FAD979
:10FF100011685518A5420BD1246821445418A342F6
:10FF20001160DDD11C685B68536021441160D7E724
:10FF300002D90C230360D3E7256861198B4204BF03
:10FF400019685B68636004BF491921605460C7E7A2
:10FF500003B030BD182C0020F8B5CD1C25F00305EA
:10FF600008350C2D38BF0C25002D064601DBA942B3
:10FF700003D90C2333600020F8BD00F02FFD214988
:10FF80000A6814469CB9204F3B6823B92146304685
:10FF900000F092FA38602946304600F08DFA431C92
:10FFA00023D10C233360304600F01EFDE3E72368C5
:10FFB0005B1B17D40B2B03D923601C44256004E082
:10FFC0006368A2420CBF0B605360304600F00CFD2A
:10FFD00004F10B00231D20F00700C21ACCD01B1A1D
:10FFE000A350C9E722466468CCE7C41C24F003048C
:10FFF000A042E3D0211A304600F05EFA0130DDD194
:020000021000EC
:10000000CFE700BF182C00201C2C00202DE9F04F5A
:100010000D469DB014469846064618B183690BB943
:1000200000F01EFC894B9D421BD175686B6ED90791
:1000300005D4AB899A0502D4A86D05F07FF8AB8989
:100040001B0701D52B69EBB92946304600F096FA1B
:10005000C0B16B6EDC070ED54FF0FF301DB0BDE8B0
:10006000F08F7B4B9D4201D1B568DFE7794B9D4214
:1000700008BFF568DAE7AB899805EDD4A86D05F0FF
:100080005EF8E9E70023099320238DF82930CDF8A5
:100090000C803023DFF8C0818DF82A304FF0010941
:1000A00023469A4613F8012B0AB1252AF9D1BAEB57
:1000B000040B0BD05B4622462946304604F082FFF3
:1000C000013000F0AA80099A5A4409929AF8003047
:1000D000002B00F0A28000234FF0FF32CDE9052372
:1000E0000AF1010A049307938DF853301A9354468A
:1000F000052214F8011B5848F0F78AF9049AD8B978
:10010000D10644BF20238DF85330130744BF2B235F
:100110008DF853309AF800302A2B15D0079A5446A0
:1001200000204FF00A0C214611F8013B303B092B0F
:100130004ED9B0B1079214E0A0EB080309FA03F31B
:1001400013430493A246D2E7039B191D1B68039136
:10015000002BBBBF5B4242F0020207930793B8BF7C
:10016000049223782E2B0CD163782A2B35D1039B54
:100170001A1D1B680392002BB8BF4FF0FF330234E7
:100180000593DFF8E4A0217803225046F0F740F908
:1001900040B14023A0EB0A0003FA00F0049B0343A4
:1001A0000134049314F8011B2C488DF82810062202
:1001B000F0F72EF900283FD0294B1BBB039B0733D8
:1001C00023F0070308330393099B3B44099367E734
:1001D0000CFB02320C460120A5E7002301340593F5
:1001E00019464FF00A0C204610F8012B303A092A24
:1001F00003D9002BC5D00591C3E70CFB01210446B0
:100200000123F0E703AB00932A46164B04A93046BE
:10021000AFF300800746781CD6D16B6ED90705D4A2
:10022000AB899A0502D4A86D04F089FFAB895B06FF
:100230003FF512AF099811E703AB00932A46094B2B
:1002400004A9304600F012F8E4E700BF406801005E
:100250006068010020680100EC680100F668010098
:1002600000000000C54F0100F26801002DE9FF47C2
:100270000C469146277E0C99782F80469A4604F1C9
:10028000430207D8622F0AD8002F00F0D880582FD9
:1002900000F0A38004F1420684F842703AE0A7F12E
:1002A0006303152BF6D801A050F823F005030100D5
:1002B0001903010095020100950201009502010059
:1002C0009502010019030100950201009502010049
:1002D0009502010095020100250401004903010077
:1002E0000704010095020100950201004704010086
:1002F00095020100490301009502010095020100E9
:100300000F0401000B681A1D1B680A6004F1420605
:1003100084F842300123A3E0256808682E0600F126
:1003200004030AD505680B60002D03DA2D236D4206
:1003300084F843305E480A2319E015F0400F056841
:100340000B6018BF2DB2EFE70B682568181D086019
:10035000280601D51D6802E06906FBD51D885448B2
:100360006F2F0CBF08230A23002184F8431066680E
:10037000A660002EA2BF216821F0040121600DB902
:10038000002E4DD01646B5FBF3F103FB1157C75DA8
:1003900006F8017D2F46BB420D46F4D9082B0BD140
:1003A0002368DF0708D5236961689942DEBF3023DF
:1003B00006F8013C06F1FF36921B2261CDF800A041
:1003C0004B4603AA2146404604F00EFE01304CD1B4
:1003D0004FF0FF3004B0BDE8F087354884F8457031
:1003E00023680E681F0656F8045B0E6014D5D90703
:1003F00044BF43F0200323601DB9236823F020038A
:1004000023601023B0E7236843F0200323607823A0
:10041000284884F84530E3E75E0648BFADB2E6E71A
:100420001646BBE70B68266860691D1D0D60350622
:100430001B6801D5186002E07106FBD51880002307
:1004400023611646BAE70B681A1D0A601E686268C7
:1004500000213046EFF7DCFF08B1801B6060636865
:100460002361002384F84330A8E7236932464946D4
:100470004046D0470130ABD023689B0713D4E068D7
:10048000039B9842B8BF1846A4E701233246494669
:100490004046D04701309BD00135E36803995B1A91
:1004A000AB42F2DCEBE7002504F11906F5E700BFEB
:1004B000FD6801000E69010038B5064D00230446B1
:1004C00008462B6001F06CFA431C02D12B6803B183
:1004D000236038BD902C0020F8B50E461446054622
:1004E00018B183690BB900F0BBF9214B9C422BD1A9
:1004F0006C68A369A360A3891A072FD523696BB31E
:1005000023692068C01A6369F6B28342374604DC67
:100510002146284600F026F930BBA368013BA360C2
:1005200023685A1C22601E7063690130834204D024
:10053000A389DB0706D50A2E04D12146284600F000
:1005400011F988B93846F8BD0A4B9C4201D1AC6814
:10055000CFE7094B9C4208BFEC68CAE72146284612
:1005600000F00CF80028CBD04FF0FF37EAE700BFCF
:10057000406801006068010020680100324B70B5DE
:100580001D6806460C4625B1AB6913B9284600F034
:1005900067F92E4B9C420FD16C68A389B4F90C20EB
:1005A00019072CD4DD0611D40923336042F040032F
:1005B000A3814FF0FF303EE0254B9C4201D1AC6857
:1005C000EBE7244B9C4208BFEC68E6E7580712D5DE
:1005D000616B41B104F14403994202D03046FFF708
:1005E0006BFC00236363A38923F02403A38100230E
:1005F000636023692360A38943F00803A38123690F
:100600004BB9A38903F42073B3F5007F03D02146CF
:10061000304600F0A3F9A089B4F90C2010F00103D2
:100620000AD00023A36063695B42A361236943B9D5
:1006300010F08000BAD170BD810758BF6369A36014
:10064000F4E70020F7E700BF380100204068010010
:1006500060680100206801008A892DE9F0410546A3
:1006600010070C4658D44B68002B05DC0B6C002B94
:1006700002DC0020BDE8F081E66A002EF9D00023FC
:1006800012F480522F682B6032D0606DA3895A0714
:1006900005D56368C01A636B0BB1236CC01A0023C5
:1006A0000246E66A216A2846B047431CA38906D160
:1006B00029681D292CD82A4ACA40D60728D50022E5
:1006C0006260D9042269226004D5421C01D12B68E2
:1006D00003B96065616B2F600029CAD004F144033F
:1006E000994202D02846FFF7E7FB00206063C1E78C
:1006F000216A01232846B047411CC7D12B68002B33
:10070000C4D01D2B01D0162B01D12F60B1E7A389D6
:1007100043F04003A381ADE70F69002FA9D09307F1
:100720000E6808BF4B690F6018BF0023A6EB0708CF
:100730008B60B8F1000F9CDD216AA66A43463A46F9
:100740002846B047002806DCA38943F04003A38174
:100750004FF0FF308EE70744A8EB0008E9E700BF41
:100760000100402038B50B6905460C4613B9002539
:10077000284638BD18B183690BB900F071F8144BE5
:100780009C421BD16C68B4F90C30002BEFD0626E28
:10079000D00704D4990502D4A06D04F0CFFC2846FC
:1007A0002146FFF759FF636EDA070546E0D4A389B7
:1007B0009B05DDD4A06D04F0C2FCD9E7054B9C423B
:1007C00001D1AC68DFE7044B9C4208BFEC68DAE774
:1007D000406801006068010020680100002310B536
:1007E0000446C0E90033C0E9043383608181436675
:1007F000C2818361194608225C3004F0C4FB054BBA
:100800006362054BA362054BE362054B24622363DD
:1008100010BD00BFDD510100FF5101003752010042
:100820005B520100014904F069BC00BF650701008B
:10083000014804F083BC00BF9C2C0020014804F058
:100840007EBC00BF9C2C0020014804F077BC00BF98
:10085000972C0020014804F072BC00BF972C0020A8
:1008600010B50446FFF7F0FFA3691BB1BDE81040C7
:10087000FFF7F0BFC4E912332365134B134A1B681B
:10088000A262A34204BF0123A361204600F020F826
:100890006060204600F01CF8A060204600F018F8C8
:1008A0000022E06004216068FFF798FFA068012241
:1008B0000921FFF793FFE06802221221FFF78EFF64
:1008C0000123A361D2E700BF1C68010025080100D5
:1008D000F8B50746FFF7ACFF1E4B1E68B36913B9A6
:1008E0003046FFF7BDFF4836D6E90134013B03D55A
:1008F00033680BB33668F7E7B4F90C50D5B9164B2B
:10090000E36004F15800656604F017FCFFF796FFFA
:10091000C4E90155C4E904552560A56108222946AA
:1009200004F15C0004F02FFBC4E90D55C4E9125535
:100930002046F8BD6834D9E70421384604F0C8FBE6
:10094000044630600028D5D1FFF778FF0C233B60C8
:10095000EEE700BF1C6801000100FFFF8B8973B543
:100960009D0706460C4607D504F147032360236123
:100970000123636102B070BD01AB6A4604F0E0FB85
:10098000009905463046FFF7E7FA48B9B4F90C304C
:100990009A05EFD423F0030343F00203A381E3E7B6
:1009A0000D4BB362A389206043F08003A381009BB9
:1009B0006361019B20615BB1B4F90E10304600F019
:1009C00067F828B1A38923F0030343F00103A3814F
:1009D000A0890543A581CDE725080100014804F061
:1009E000ADBB00BF982C0020014804F0A8BB00BF9D
:1009F000982C0020024B0146186804F0C5BB00BFCC
:100A00003801002038B5074D00230446084611463A
:100A10002B6000F0E3FF431C02D12B6803B123607D
:100A200038BD00BF902C002038B5074D044608465D
:100A3000114600222A601A4604F0AEFC431C02D183
:100A40002B6803B1236038BD902C002038B5064DCB
:100A50000023044608462B6001F038F8431C02D1FD
:100A60002B6803B1236038BD902C002038B5074DAA
:100A700000230446084611462B6004F0DFFC431CAB
:100A800002D12B6803B1236038BD00BF902C002039
:100A900038B5064D0023044608462B6004F0DCFC04
:100AA000431C02D12B6803B1236038BD902C002079
:100AB00038B5074D04460846114600222A601A46FA
:100AC00004F058FC431C02D12B6803B1236038BDED
:100AD000902C002038B5074D0446084611460022E8
:100AE0002A601A4604F0EFFB431C02D12B6803B1C5
:100AF000236038BD902C002008B52DED028BF0EE60
:100B0000408AB0EE608A00F015F820B9B0EE480ACD
:100B1000BDEC028B08BDB0EE480A00F00BF820B126
:100B2000F4EEC88AF1EE10FAF0D5B0EE680ABDEC2A
:100B3000028B08BD10EE103A33F000400ED0A0F545
:100B40000003B3F1FE4F0DD3074B421E9A4207D963
:100B5000A0F1FF40B0FA80F04009704702207047D2
:100B60000320704704207047FEFF7F00D0B52DEDB5
:100B7000028B3B4C8AB0F0EE408A00F027FA94F9E1
:100B800000300133B0EE408A12D0B0EE680A00F0B7
:100B900023FE68B1DFED337AF4EEE78AF1EE10FA66
:100BA00040DCDFED317AF4EEE78AF1EE10FA05D49D
:100BB000B0EE480A0AB0BDEC028BD0BD04232B4A2C
:100BC000009318EE900A002308930192FEF7EAFCC6
:100BD00094F9003000260027022BCDE90401CDE96D
:100BE0000201CDE9066718D0684600F0EBFDA0B120
:100BF000089B002B2ED1DDE90601FEF73DFF08EE34
:100C0000100AB0EE480A0AB0BDEC028BD0BD1849FC
:100C10000020022BCDE90601E6D100F0A9FF222336
:100C20000360E5E70323114A009318EE900A0023BE
:100C300008930192FEF7B6FC94F90030CDE9040167
:100C4000CDE90201002BE2D10A4B4FF06042CDE921
:100C50000623C9E700F08CFF089B0360CBE700BFC9
:100C60009C0100208071B142B5F1CFC280680100C3
:100C70000000F07FFFFFEF47F0B52DED048BB84D7E
:100C80008BB0F0EE408AB0EE608A00F097FA95F9EA
:100C90000040631CB0EE409A33D0B4EE488AF1EEC7
:100CA00010FA2ED6F4EE688AF1EE10FA80F19C80EC
:100CB000DFEDAC9AF4EE698AF1EE10FA27D1B4EECA
:100CC000698AF1EE10FA5FD10123A74A009318EE6A
:100CD000900A002301920893FEF764FC02460B463B
:100CE00018EE100ACDE90223FEF75CFC0022002377
:100CF000CDE90401CDE90623002C00F09580B7EE84
:100D0000009AB0EE490A0BB0BDEC048BF0BD00F0C8
:100D100063FD0446002800F09E80B5EE409AF1EE97
:100D200010FAEED1B0EE680A00F056FD0028E8D0C7
:100D3000B0EE480A00F050FD0028E2D004238A4AB1
:100D4000009318EE900A002301920893FEF72AFC04
:100D500002460B4618EE100ACDE90223FEF722FCEC
:100D600095F9003000260027022BCDE90401CDE9DA
:100D7000066704D0684600F025FD002859D100F030
:100D8000F7FE2223036054E0B0EE480A00F024FD91
:100D90000028B6D0B5EEC08AF1EE10FAB1D5012325
:100DA000714A009318EE900A002301920893FEF70F
:100DB000F9FB02460B4618EE100ACDE90223FEF7B6
:100DC000F1FB95F90030CDE90401002B40F0818062
:100DD00000220023CDE90623684600F0F3FC00283A
:100DE0007ED0089B5BB326E0B5EE408AF1EE10FAA8
:100DF00087D101235C4A009318EE900A00230192E8
:100E00000893FEF7CFFB02460B4618EE100ACDE919
:100E10000223FEF7C7FB554B0022022CCDE904014B
:100E2000CDE906233FF46BAF684600F0CBFC002809
:100E30005BD0089B1BB100F09BFE089B0360DDE9C3
:100E40000601FEF719FE09EE100AB0EE490A0BB0D2
:100E5000BDEC048BF0BDB0EE680A00F0BDFC0028CC
:100E60003FF45BAFB0EE480A00F0B6FC00283FF458
:100E700054AFB4EE499AF1EE10FA80F181803A4B0A
:100E80000894032218EE900ACDE90023FEF78AFBAE
:100E900002460B4618EE100ACDE90223FEF782FB4C
:100EA00095F90030CDE9040123BB314BF5EEC08A42
:100EB0004FF06042F1EE10FACDE9062326D46846E1
:100EC00000F080FC00288CD100F052FE2223036049
:100ED00087E728490020022BCDE906017FF47CAF8B
:100EE00000F046FE212303607BE700F041FE212352
:100EF00003609EE72049F5EEC08A0020F1EE10FA6B
:100F0000CDE9060117D4022BDED0D8E7F6EE007A41
:100F100028EE278AB0EE480A00F072FCB4EE480AC8
:100F2000F1EE10FA18D0154995F900304FF06040F5
:100F3000CDE90601E7E7F6EE007A28EE278AB0EE63
:100F4000480A00F05DFCB4EE480AF1EE10FA03D056
:100F5000084B0022CDE9062395F90030D3E700BF06
:100F60009C01002000000000886801000000F03FA4
:100F7000FFFFEF470000F0FF0000F07FFFFFEFC72B
:100F8000114B0894012218EE900ACDE90023FEF7D8
:100F900009FB02460B4618EE100ACDE90223FEF7C4
:100FA00001FB95F90040CDE90401002C3FF410AF9E
:100FB000C9EEA97A17EE900AFEF7F4FA022CCDE9F1
:100FC00006018DD008E700BF8868010010EE103AD6
:100FD00023F00042B2F1FF4F57D84FEAD37100F02F
:100FE00098806448834253DC002BC0F28B80624BB4
:100FF0009A4252D9614B9A4200F29E80604B614AFC
:1010000003EB810393ED004A02EB8102C1F101037E
:1010100030EE444A92ED007A5B1A34EE470ADFED77
:101020005A7ADFED5A4A9FED5A5ADFED5A5A9FED30
:101030005A6A60EE006AE6EEA74AF0EE407AA4EE45
:10104000A65AE5EE265AA5EEA66AE6EE667AF0EE18
:10105000676A002B47D0B0EE006A60EE275A76EE42
:10106000676A13F17D0F85EEA60AF7EE007A37EE78
:10107000400A30EE440A37EEC00A51DB10EE102A67
:1010800002EBC35300EE103A704730EE000A70478F
:101090009FED420A20EE000A7047B2F1465F0AD285
:1010A000DFED3E7A70EE277AB7EE007AF4EEC77A7B
:1010B000F1EE10FA5ADC60EE007A9FED335ADFED64
:1010C000335A9FED336ADFED336A9FED337AE7EEF3
:1010D000855AA7EEA56AE7EE866AA7EEA67AF0EE35
:1010E000406AE7EEC76AB0EE007A36EEC77A60EE85
:1010F000266AB7EE006AC6EE877A37EEC00A36EE89
:10110000400A7047264B9A427FF671AF9FED250A41
:101110007047DFED247A002918BFB0EE670A7047E8
:1011200010EE102A643302EBC353DFED1F7A00EE9A
:10113000103A20EE270A70471C4B9FED1D7A9FED59
:101140001D6ADFED1D6A03EB8103D3ED007AE0EE4B
:10115000077AB0EE404AFDEEE77AB8EEE77A17EE8E
:10116000903AA7EE464A27EE267A56E730EE070A6F
:10117000704700BF1772B1421872B13E9115853F9A
:1011800098680100A06801004CBB31330EEADDB560
:1011900055B38A38610B36BBABAA2A3ECAF24971F5
:1011A000B5F1CF42000000000000800D9068010002
:1011B0003BAAB83F8071313FD1F717372DE9F0478F
:1011C00010EE904A34F000482DED028B15D010EE51
:1011D000105A25F00047B7F1FF4F10EE109A06DDC8
:1011E000BDEC028BBA48BDE8F04700F003BBB8F194
:1011F000FF4F08DDB7F17E5FF2D1B7EE000ABDEC1C
:10120000028BBDE8F087002D10EE906AC0F2F680E8
:101210004FF0000AB8F1FF4F00F00481B8F17E5F93
:1012200000F02A81B6F1804F00F03F81B6F17C5F7B
:1012300000EE105A40F00381B9F1000F80F23A81BC
:1012400000F0C2FAB7F1FF4F00F00B81002F00F061
:101250000481B7F17E5F00F0FA804FEAD972013A5B
:101260005AEA020300F02C81B8F19A4F40F3528100
:10127000984B9F4240F35F82974B9F4200F301815E
:10128000F7EE007A30EE670ADFED946ADFED947ACC
:10129000DFED945A9FED946AB5EE007AE0EE476A6E
:1012A000B6EE007AA6EEC07AF0EE476A20EE007A3B
:1012B00027EE267A67EEC77AE0EE257AF0EE676AC7
:1012C000E0EE066A16EE903A23F47F6323F00F03F4
:1012D00007EE103AA0EE467A06EE903A77EEC77A1D
:1012E00026F47F6626F00F0607EE104A06EE106A17
:1012F00067EE877A37EE466A07EE106AE6EE267AE0
:101300000AF1FF3A5AEA020326EE877AB7EE000A9C
:1013100077EE876ABFEE006A16EE903A0CBFB0EE29
:10132000468AB0EE408A002B23F0004240F3B98198
:10133000B2F1864F00F3F88100F0EB81B2F17C5FEF
:1013400000F3BB810022104623F47F6323F00F03D8
:1013500006EE103ADFED656ADFED655A9FED653AFE
:10136000DFED653A9FED652A9FED654ADFED654A41
:101370009FED655A36EE477AF0EE002A77EEC77A8F
:1013800026EE267AA7EEA57AF7EE005AF0EE477A17
:10139000A6EE037A67EE076AF0EE471AE6EE431A06
:1013A000B0EE636AA6EE826A77EEE17AA6EE264A8E
:1013B000E7EE277AE4EE264AA4EEA65AB0EE456A96
:1013C000B0EE475AA6EE665AF0EE456A36EEE26A8D
:1013D00027EE055AC5EE066A76EEE77A37EEC77A4B
:1013E00035EEC70A10EE103A1344B3F5000FC0F201
:1013F000BA8100EE103A20EE080A00E7B8F1974FE4
:101400001ADAB8F17E5F0ADB4FEAE853C3F19603BC
:1014100048FA03F202FA03F3434500F03D814FF02E
:10142000000AFBE6B7F17E5F3FF4E7AE2FDD002E4A
:101430002ADB00EE104AE2E64FF0020AEAE600F08C
:10144000C3F9B7F1FF4F02D0002F7FF402AF002E97
:10145000BCBFF7EE007A87EE800AB9F1000FBFF645
:10146000CEAEA7F17E5757EA0A0340F00E8170EE28
:10147000407A87EEA70AC2E6002E0FDB00EE105A74
:10148000BDE6002E00F35A819FED200AB7E6002E3C
:10149000FADA07EE904AB1EE670AB0E607EE105AA4
:1014A000F7EE007A87EE870AA9E607EE905A27EE54
:1014B000A70AA4E6BDEC028BBDE8F04700F07EB9B8
:1014C00007EE905A77EEE77A87EEA70A97E600BF15
:1014D00034630100F7FF7F3F0700803FABAAAA3EBD
:1014E0003BAAB83F70A5EC3600AAB83F8CBEBF350A
:1014F0001872313F0072313F0EEADDB54CBB31331B
:1015000055B38A38610B36BBABAA2A3E00000000F7
:101510000000804B19F0FF4F40F0F9805FED047A36
:1015200060EE277A6FF0170117EE907A8F48FB155F
:10153000C7F316077F3B87420B4447F07E5140F3C9
:10154000DE808B48874240F3FE80DFED8A4A01331C
:10155000A1F50001F0EE643A0020B7EE006A06EE55
:10156000901A76EE867AB7EE007A87EE278A4910CF
:1015700041F0005101F58021014436EEC67A07EEB4
:10158000901A27EE082A77EEC65A9FED7B4A7B49D0
:10159000DFED7B8A9FED7B0ADFED7B0A9FED7B1AF7
:1015A000DFED7B1ADFED7B2A9FED7B3A9FED7B5AC7
:1015B00022EE026A12EE100A76EEE56AF0EE445A66
:1015C000E6EE285A084004EE100AA4EE677AF0EE20
:1015D000407AE5EE867AA4EE667AE7EE860A67EE52
:1015E000086AB0EE417AA0EE867A72EE047AE7EEEF
:1015F000061A67EEA67A26EE066AF0EE085AE6EEBE
:10160000217AB0EE656AA4EE046A07EE103A36EE6F
:10161000276AB8EEC77A16EE103A0B4006EE103A7B
:1016200076EE655AE4EE445A77EEE57A67EE827A12
:10163000E6EE867AF0EE675AE4EE065A15EE903A38
:101640000B4006EE903AE4EE466A05EE903A77EEED
:10165000E67A67EEA27AE5EE837A77EEA37AF0EE89
:10166000676AE5EE856A76EEA46A76EE876A16EE1C
:10167000903A0B4006EE903A36EEC77A37EE647A2F
:10168000A5EEC57A77EEC77A2AE6BAF1010F7FF4A4
:10169000B6ADB1EE400AB2E502F00102C2F1020AB3
:1016A000BCE53F498A4257DC7FF448AE76EEC76A14
:1016B000F4EEE76AF1EE10FA4EDAD2154FF40001BB
:1016C0007E3A41FA02F21A44C2F3C751354C7F39CF
:1016D0000C41C2F3160022EA040206EE902A37EE0D
:1016E000667AC1F1170140F400000841002B77EE43
:1016F000876AB8BF404216EE903AC20524E6DFED95
:101700001D4A0020F0EE643AB7EE006A27E7002198
:101710000CE79FED256A76EEC76A37EE866AB4EE6F
:10172000E66AF1EE10FAC8DDDFED207A28EE270A2E
:1017300020EE270A63E5002EBFF6A6AE9FED1B0A3A
:1017400020EE000A5BE5DFED1A4ADFED1A3A4FF4AE
:101750000010B7EE086A02E7DFED177A28EE270AD5
:1017600020EE270A4BE500F0A9F844E671C41C00FE
:10177000D6B35D000000000055326C3E00F0FFFF64
:1017800042F1533E05A38B3EABAAAA3EB76DDB3EAA
:101790009A99193F4F38763FA0C39D360038763F5F
:1017A00000001643FFFF7F003CAA3833CAF249719C
:1017B00000C0153FDCCFD1356042A20DB1EEC00AAA
:1017C000704700BF0020704710EE103A23F000432E
:1017D00000EE103A704700BF82B08DED010A01980B
:1017E00020F00040B0F1FF4FACBF0020012002B05C
:1017F000704700BF9FED010A704700BF0000C07F27
:1018000010EE101AC1F3C753A3F17F02162A21F07C
:10181000004328DC33B310B4002A83B04FEAD17000
:1018200027DB244B1341194218D05C0811EA5303FB
:1018300007D04FF4001321EA040113410B4300EEDB
:10184000103A1D4B03EB8000D0ED007A37EE800A92
:101850008DED010A9DED010A30EE670A03B05DF8D7
:10186000044B70477047B3F1FF4FFBD330EE000AD3
:101870007047C1F316035B420F4A5B0A090D03F47C
:1018800080030905194302EB8002D2ED006A07EEDE
:10189000901A36EEA77A8DED017ADDED017A77EEBA
:1018A000E67A17EE903A23F0004343EAC07300EE65
:1018B000103AD3E7FFFF7F00A868010082B08DEDEA
:1018C000010A019B33F000422AD0B2F1FF4F23D22C
:1018D00013F0FF4F28D19DED017ADFED2A7A2A4BD4
:1018E00067EE277A9842CDED017A37DB019BC3F38F
:1018F000C752193A0244FE2A1ADD9FED240A9FEDD1
:10190000247A019B002BF0EE407AB8BFB0EE470A74
:1019100020EE270A02B0704730EE000A02B070478E
:101920009DED010A02B07047D20D0244FE2AE4DCAC
:10193000002A0BDC12F1160F17DA4CF250339842E2
:10194000DBDC9FED140A9FED147ADAE723F0FF4306
:1019500043EAC25300EE103A02B070479FED0D0A01
:10196000DDED017A27EE800AD8E7193223F0FF4334
:1019700043EAC253DFED097A07EE103A27EE270A51
:10198000CCE700BF0000004CB03CFFFFCAF2497139
:10199000CAF249F16042A20D6042A28D00000033FC
:1019A00070B50C4D2B680BB90B4B2B6003302E68B8
:1019B00020F003043444204600F0AEF810B92C6047
:1019C000304670BD00F0D4F80C2303604FF0FF36B2
:1019D000F6E700BF202C0020A02C0020062930B5FF
:1019E0000CBF044D044D182420462946ABBE0446C6
:1019F000204630BD23000200260002002DE9F04FF2
:101A0000234E336885B0002B3FD1DFF898A0CDF886
:101A100004A04FF00309CDF80C90012402930DF1BE
:101A2000040820464146ABBE05461A4FCDF804A037
:101A30000423CDF80C903D60029320464146ABBE96
:101A40008346154DCDF804A00823CDF80C90C5F8B9
:101A500000B0029320464146ABBE04460F4A2868B8
:101A60001460013404BF2B6813600D4B12684FF0F3
:101A7000FF3199611962396819600021C3E90201D7
:101A8000C3E9042159600123336005B0BDE8F08F3C
:101A9000242C00202C2C0020302C0020282C00206E
:101AA000342C00201F690100042810B5044601D918
:101AB000002010BDFFF7A2FF034850F83420013288
:101AC000F6D000EBC400F4E7342C002038B505460E
:101AD000FFF7EAFF044630B900F04AF80923036033
:101AE0004FF0FF3038BD013D012D09D8094B9A68F0
:101AF0001B699A4204D14FF0FF3303600020F1E7E5
:101B0000206803F06BFC0028ECD14FF0FF3323601A
:101B1000E8E700BF342C0020044B23B1984234BFC7
:101B20000020012070471846704700BFA03C0020ED
:101B300010B5054C237833B9044B13B10448AFF307
:101B400000800123237010BD5C2C002000000000E9
:101B50005869010008B5034B1BB103490348AFF3B3
:101B6000008008BD00000000602C002058690100C2
:101B7000014B1868704700BF3801002008B5FAF71C
:101B800099FF08BD08B5FAF7A3FF08BD08B5FAF735
:101B9000ADFF08BD08B5FAF7B7FF08BD08B5FAF7FD
:101BA000C1FF08BD08B5FAF7CBFF08BD08B5FAF7C5
:101BB000D5FF08BD08B5FAF7DFFF08BD08B5FAF78D
:101BC000E9FF08BD08B5FAF7F3FF08BD08B5FAF755
:101BD000FDFF08BD08B5FBF707F808BD08B5FBF722
:101BE00011F808BD08B5FBF71BF808BD08B5FBF7F1
:101BF00025F808BD08B5EEF736FB08BD08B5EEF7C9
:101C000032FB08BD08B5EEF72EFB08BD08B5EEF7B0
